:020000040800F2
:100000000080012059240408B9130008CD1300080A
:100010006D160008851600089D16000800000000F7
:10002000000000000000000000000000B5160008FD
:10003000C916000800000000DD16000801DD0008F8
:10004000B5240408B5240408B524040831DD0008EB
:10005000B5240408B5240408B5240408B52404080C
:10006000B5240408B5240408B5240408B5240408FC
:10007000B5240408B5240408B5240408B5240408EC
:10008000B5240408B5240408B5240408B5240408DC
:10009000B5240408B5240408B5240408B5240408CC
:1000A000B5240408B5240408B5240408B5240408BC
:1000B0003FDD0008B5240408B5240408B52404086D
:1000C000B5240408B5240408B5240408B52404089C
:1000D000B52404084BDD000857DD000863DD000887
:1000E000B5240408B5240408B5240408B52404087C
:1000F000B5240408B5240408B5240408B52404086C
:10010000B5240408B5240408B5240408B52404085B
:100110006FDD00087BDD0008B5240408B524040861
:10012000B5240408B5240408B5240408B52404083B
:1001300000000000000000000000000000000000BF
:1001400000000000000000000000000000000000AF
:10015000000000000000000000000000000000009F
:10016000000000000000000000000000000000008F
:10017000000000000000000000000000000000007F
:10018000000000000000000000000000000000006F
:10019000000000000000000000000000000000005F
:1001A000000000000000000000000000000000004F
:1001B000000000000000000000000000000000003F
:1001C000000000000000000000000000000000002F
:1001D000000000000000000000000000000000001F
:0401E0005FF8E0F1F3
:1001E800EC46A0E8F05F4FF000007047B0E8F05F21
:1001F800E546080008BF0120704700BF80EA010CEF
:100208001CF0030F37D110F0030C20F0030021F08D
:10021800030150F8042B08BF51F8043B0ED08CF0B2
:10022800030C6FF07F434FEACC0C23FA0CFC51F817
:10023800043B42EA0C0243EA0C0300BFA2F1013C72
:100248009A4201BF2CEA020C1CF0803F50F8042BA4
:1002580051F8043BF2D04FEA02604FEA122201281B
:1002680028BFB0EB036F08BF1B0AF4D003F0FF03ED
:10027800000EC01A704710F0030F0AD010F8012BB7
:1002880011F8013B012A28BF9A42F4D0A2EB0300DF
:1002980070474DF8045D50F8042B01F0030521F078
:1002A800030151F8043B022D26D04DD822F07F459A
:1002B800B5EB132FA2F1013C2CEA020C0DD11CF076
:1002C800803C08BF51F8043B0AD185EA0205B5EB2A
:1002D800036F0CD150F8042BE8E74FEA13235BE0D7
:1002E8003CF07F4C54D10B784FEA126554E04FEA4A
:1002F800126503F0FF034FE04FEA0245A2F1013C0B
:100308004FEA15452CEA020CB5EB134F18D11CF037
:10031800803C08BF51F8043B07D185EA0205B5EBDC
:10032800034F09D150F8042BE6E75FEA0C4C2FD1B4
:100338000B884FEA12452FE04FEA03434FEA124574
:100348004FEA134328E000BF02F0FF05B5EB136F37
:10035800A2F1013C2CEA020C0DD11CF0803C08BF34
:1003680051F8043B0AD185EA0205B5EB032F0AD1FF
:1003780050F8042BE8E74FEA13630DE012F0FF0F83
:1003880006D051F8043B4FEA122523F07F4303E0DF
:100398004FF0000020BC704705F0FF0203F0FF009B
:1003A800012828BF904204BF2D0A1B0AF4D0A2EBF3
:1003B800000020BC704700BF844641EA000313F0E8
:1003C800030349D1403A23D30B6803604B68436069
:1003D8008B688360CB68C3600B6903614B694361B9
:1003E8008B698361CB69C3610B6A03624B6A4362A1
:1003F8008B6A8362CB6AC3620B6B03634B6B436389
:100408008B6B8363CB6BC36340304031403ADBD2A4
:1004180030320BD30B6803604B6843608B68836092
:10042800CB68C36010301031103AF3D20C3205D3C8
:1004380051F8043B40F8043B043AF9D2043208D09E
:10044800D2071CBF11F8013B00F8013B01D30B8810
:1004580003806046704700BF082A13D38B07B1D0CA
:1004680010F00303AED0C3F10403D21ADB071CBF9C
:1004780011F8013B00F8013BA4D331F8023B20F806
:10048800023B9FE7043AD9D3013A11F8013B00F83F
:10049800013BF9D20B7803704B7843708B788370EB
:1004A8006046704781F0004102E000BF83F00043DE
:1004B80030B54FEA41044FEA430594EA050F08BFF7
:1004C80090EA020F1FBF54EA000C55EA020C7FEABB
:1004D800645C7FEA655C00F0E2804FEA5454D4EB38
:1004E8005555B8BF6D420CDD2C4480EA020281EA02
:1004F800030382EA000083EA010180EA020281EA3A
:100508000303362D88BF30BD11F0004F4FEA01318B
:100518004FF4801C4CEA113102D0404261EB41019A
:1005280013F0004F4FEA03334CEA133302D0524220
:1005380063EB430394EA050F00F0A780A4F10104DC
:10054800D5F1200E0DDB02FA0EFC22FA05F2801816
:1005580041F1000103FA0EF2801843FA05F35941FC
:100568000EE0A5F120050EF1200E012A03FA0EFC7B
:1005780028BF4CF0020C43FA05F3C01851EBE371A5
:1005880001F0004507D54FF0000EDCF1000C7EEBC2
:1005980000006EEB0101B1F5801F1BD3B1F5001F00
:1005A8000CD349085FEA30004FEA3C0C04F101041F
:1005B8004FEA445212F5800F80F09A80BCF1004F48
:1005C80008BF5FEA500C50F1000041EB045141EACA
:1005D800050130BD5FEA4C0C404141EB0101013C93
:1005E80028BFB1F5801FE9D291F0000F04BF014682
:1005F8000020B1FA81F308BF2033A3F10B03B3F154
:1006080020020CDA0C3208DD02F1140CC2F10C02E3
:1006180001FA0CF021FA02F10CE002F11402D8BF41
:10062800C2F1200C01FA02F120FA0CFCDCBF41EA0D
:100638000C019040E41AA2BF01EB0451294330BDDC
:100648006FEA04041F3C1CDA0C340EDC04F11404B9
:10065800C4F1200220FA04F001FA02F340EA030090
:1006680021FA04F345EA030130BDC4F10C04C4F1D6
:10067800200220FA02F001FA04F340EA03002946B6
:1006880030BD21FA04F0294630BD94F0000F83F400
:10069800801306BF81F480110134013D4EE77FEAE3
:1006A800645C18BF7FEA655C29D094EA050F08BF2F
:1006B80090EA020F05D054EA000C04BF1946104610
:1006C80030BD91EA030F1EBF0021002030BD5FEA54
:1006D800545C05D14000494128BF41F0004130BD7C
:1006E80014F580043CBF01F5801130BD01F00045D0
:1006F80045F0FE4141F470014FF0000030BD7FEA43
:10070800645C1ABF194610467FEA655C1CBF0B463D
:10071800024650EA013406BF52EA033591EA030F54
:1007280041F4002130BD00BF90F0000F04BF00214C
:10073800704730B54FF4806404F132044FF000057F
:100748004FF0000150E700BF90F0000F04BF0021F8
:10075800704730B54FF4806404F1320410F000455E
:1007680048BF40424FF000013EE700BF42004FEA59
:10077800E2014FEA31014FEA02701FBF12F07F43D6
:1007880093F07F4F81F06051704732F07F4208BF8D
:10079800704793F07F4F04BF41F40021704730B594
:1007A8004FF4607401F0004521F000411CE700BFE0
:1007B80050EA010208BF704730B54FF000050AE063
:1007C80050EA010208BF704730B511F0004502D564
:1007D800404261EB41014FF4806404F132045FEA66
:1007E800915C3FF4D8AE4FF003025FEADC0C18BF0F
:1007F80003325FEADC0C18BF033202EBDC02C2F101
:10080800200300FA03FC20FA02F001FA03FE40EA92
:100818000E0021FA02F11444BDE600BF70B54FF096
:10082800FF0C4CF4E06C1CEA11541DBF1CEA135574
:1008380094EA0C0F95EA0C0F00F0DEF82C4481EADC
:10084800030621EA4C5123EA4C5350EA013518BFFC
:1008580052EA033541F4801143F4801338D0A0FBE9
:1008680002CE4FF00005E1FB02E506F00042E0FB96
:1008780003E54FF00006E1FB03569CF0000F18BF9C
:100888004EF0010EA4F1FF04B6F5007F64F5407444
:1008980004D25FEA4E0E6D4146EB060642EAC621D7
:1008A80041EA55514FEAC52040EA5E504FEACE2E44
:1008B800B4F1FD0C88BFBCF5E06F1ED8BEF1004F47
:1008C80008BF5FEA500E50F1000041EB045170BDC3
:1008D80006F0004646EA010140EA020081EA030107
:1008E800B4EB5C04C2BFD4EB0C0541EA045170BD03
:1008F80041F480114FF0000E013C00F3AB8014F17D
:10090800360FDEBF002001F0004170BDC4F10004C5
:10091800203C35DA0C341BDC04F11404C4F1200546
:1009280000FA05F320FA04F001FA05F240EA0200A1
:1009380001F0004221F0004110EBD37021FA04F6D7
:1009480042EB06015EEA430E08BF20EAD37070BD91
:10095800C4F10C04C4F1200500FA04F320FA05F0F0
:1009680001FA04F240EA020001F0004110EBD370F2
:1009780041F100015EEA430E08BF20EAD37070BD62
:10098800C4F1200500FA05F24EEA020E20FA04F33B
:1009980001FA05F243EA020321FA04F001F00041EA
:1009A80021FA04F220EA020000EBD3705EEA430E5B
:1009B80008BF20EAD37070BD94F0000F0FD101F08A
:1009C8000046400041EB010111F4801F08BF013CC3
:1009D800F7D041EA060195F0000F18BF704703F001
:1009E8000046520043EB030313F4801F08BF013D88
:1009F800F7D043EA0603704794EA0C0F0CEA135544
:100A080018BF95EA0C0F0CD050EA410618BF52EAFD
:100A18004306D1D181EA030101F000414FF0000003
:100A280070BD50EA410606BF1046194652EA430611
:100A380019D094EA0C0F02D150EA013613D195EA85
:100A48000C0F05D152EA03361CBF104619460AD1CD
:100A580081EA030101F0004141F0FE4141F47001D7
:100A68004FF0000070BD41F0FE4141F4780170BDC7
:100A780070B54FF0FF0C4CF4E06C1CEA11541DBF2C
:100A88001CEA135594EA0C0F95EA0C0F00F0A7F82E
:100A9800A4EB050481EA030E52EA03354FEA01315B
:100AA80000F088804FEA03334FF0805545EA13136E
:100AB80043EA12634FEA022245EA111545EA106536
:100AC8004FEA00260EF000419D4208BF964244F1CD
:100AD800FD0404F5407402D25B084FEA3202B61AEC
:100AE80065EB03055B084FEA32024FF480104FF4C0
:100AF800002CB6EB020E75EB030E22BFB61A754634
:100B080040EA0C005B084FEA3202B6EB020E75EBC6
:100B1800030E22BFB61A754640EA5C005B084FEA2E
:100B28003202B6EB020E75EB030E22BFB61A7546FB
:100B380040EA9C005B084FEA3202B6EB020E75EB06
:100B4800030E22BFB61A754640EADC0055EA060EC7
:100B580018D04FEA051545EA16754FEA06164FEA0A
:100B6800C30343EA52734FEAC2025FEA1C1CC0D1B6
:100B780011F4801F0BD141EA00014FF000004FF043
:100B8800004CB6E711F4801F04BF01430020B4F104
:100B9800FD0C88BFBCF5E06F3FF6AFAEB5EB030CBC
:100BA80004BFB6EB020C5FEA500C50F1000041EBB9
:100BB800045170BD0EF0004E4EEA113114EB5C0486
:100BC800C2BFD4EB0C0541EA045170BD41F4801159
:100BD8004FF0000E013C90E645EA060E8DE60CEA61
:100BE800135594EA0C0F08BF95EA0C0F3FF43BAF7E
:100BF80094EA0C0F0AD150EA01347FF434AF95EA35
:100C08000C0F7FF425AF104619462CE795EA0C0F18
:100C180006D152EA03353FF4FDAE1046194622E7E5
:100C280050EA410618BF52EA43067FF4C5AE50EABF
:100C380041047FF40DAF52EA43057FF4EBAE12E7AF
:100C48004FF0FF3C06E000BF4FF0010C02E000BF90
:100C58004FF0010C4DF804CD4FEA410C7FEA6C5C73
:100C68004FEA430C18BF7FEA6C5C1BD001B050EA16
:100C7800410C0CBF52EA430C91EA030F02BF90EA01
:100C8800020F0020704710F1000F91EA030F58BFC0
:100C9800994208BF90422CBFD8176FEAE37040F022
:100CA800010070474FEA410C7FEA6C5C02D150EAC0
:100CB800013C07D14FEA430C7FEA6C5CD6D152EA7B
:100CC800033CD3D05DF8040B704700BF8446104640
:100CD80062468C461946634600E000BF01B5FFF73F
:100CE800B7FF002848BF10F1000F01BD4DF808ED0F
:100CF800FFF7F4FF0CBF012000205DF808FB00BFE0
:100D08004DF808EDFFF7EAFF34BF012000205DF839
:100D180008FB00BF4DF808EDFFF7E0FF94BF012086
:100D280000205DF808FB00BF4DF808EDFFF7CEFF87
:100D380094BF012000205DF808FB00BF4DF808EDC6
:100D4800FFF7C4FF34BF012000205DF808FB00BF97
:100D58004FEA410C7FEA6C5C02D150EA013C0AD1AF
:100D68004FEA430C7FEA6C5C02D152EA033C02D1A1
:100D78004FF0000070474FF0010070474FEA410202
:100D880012F5001215D211D56FF47873B3EB6252D5
:100D980012D94FEAC12343F0004343EA505311F0FC
:100DA800004F23FA02F018BF404270474FF000008E
:100DB800704750EA013005D111F0004008BF6FF0CC
:100DC800004070474FF00000704700BF4A0011D242
:100DD80012F5001211D20DD56FF47873B3EB62528D
:100DE8000ED44FEAC12343F0004343EA505323FA99
:100DF80002F070474FF00000704750EA013002D10E
:100E08004FF0FF3070474FF0000070474FEA410243
:100E1800B2F1E04324BFB3F5001CDCF1FE5C0DD950
:100E280001F0004C4FEAC0024CEA5070B2F1004F9A
:100E380040EB830008BF20F00100704711F0804F9D
:100E480021D113F13872BCBF01F00040704741F462
:100E580080114FEA5252C2F11802C2F1200C10FA66
:100E68000CF320FA02F018BF40F001004FEAC1234A
:100E78004FEAD32303FA0CFC40EA0C0023FA02F3EE
:100E88004FEA4303CCE77FEA625307D150EA0133C4
:100E98001EBF4FF0FE4040F44000704701F0004094
:100EA80040F0FE4040F40000704700BF80F0004072
:100EB80002E000BF81F0004142001FBF5FEA41032A
:100EC80092EA030F7FEA226C7FEA236C6AD04FEA2A
:100ED8001262D2EB1363C1BFD2184140484041406F
:100EE800B8BF5B42192B88BF704710F0004F40F421
:100EF800000020F07F4018BF404211F0004F41F43D
:100F0800000121F07F4118BF494292EA030F3FD008
:100F1800A2F1010241FA03FC10EB0C00C3F120031B
:100F280001FA03F100F0004302D5494260EB4000AA
:100F3800B0F5000F13D3B0F1807F06D340084FEA15
:100F4800310102F10102FE2A51D2B1F1004F40EB0A
:100F5800C25008BF20F0010040EA03007047490072
:100F680040EB0000013A28BFB0F5000FEDD2B0FA0F
:100F780080FCACF1080CB2EB0C0200FA0CF0AABF32
:100F880000EBC25052421843BCBFD04018437047D0
:100F980092F0000F81F4000106BF80F400000132D6
:100FA800013BB5E74FEA41037FEA226C18BF7FEAAD
:100FB800236C21D092EA030F04D092F0000F08BFEF
:100FC8000846704790EA010F1CBF0020704712F0D6
:100FD8007F4F04D1400028BF40F00040704712F115
:100FE80000723CBF00F50000704700F0004343F07A
:100FF800FE4040F4000070477FEA226216BF0846B0
:101008007FEA23630146420206BF5FEA412390EA72
:10101800010F40F4800070474FF0000304E000BF68
:1010280010F0004348BF40425FEA000C08BF704719
:1010380043F0964301464FF000001CE050EA0102DD
:1010480008BF70474FF000030AE000BF50EA0102F2
:1010580008BF704711F0004302D5404261EB4101DF
:101068005FEA010C02BF84460146002043F0B64304
:1010780008BFA3F18053A3F50003BCFA8CF2083A29
:10108800A3EBC25310DB01FA02FC634400FA02FC32
:10109800C2F12002BCF1004F20FA02F243EB020039
:1010A80008BF20F00100704702F1200201FA02FC9B
:1010B800C2F1200250EA4C0021FA02F243EB02008E
:1010C80008BF20EADC7070474FF0FF3C06E000BF25
:1010D8004FF0010C02E000BF4FF0010C4DF804CDB9
:1010E8004FEA40024FEA41037FEA226C18BF7FEAC9
:1010F800236C11D001B052EA530C18BF90EA010FCB
:1011080058BFB2EB030088BFC81738BF6FEAE17059
:1011180018BF40F0010070477FEA226C02D15FEAF5
:10112800402C05D17FEA236CE4D15FEA412CE1D061
:101138005DF8040B704700BF844608466146FFE728
:101148000FB5FFF7C9FF002848BF10F1000F0FBD0A
:101158004DF808EDFFF7F4FF0CBF012000205DF803
:1011680008FB00BF4DF808EDFFF7EAFF34BF012088
:1011780000205DF808FB00BF4DF808EDFFF7E0FF21
:1011880094BF012000205DF808FB00BF4DF808ED72
:10119800FFF7D2FF94BF012000205DF808FB00BFD5
:1011A8004DF808EDFFF7C8FF34BF012000205DF8B7
:1011B80008FB00BF53B94AB9002908BF00281CBF63
:1011C8004FF0FF314FF0FF3000F0E2B8ADF1080CFE
:1011D8006DE904CE50F0C4F8DDF804E0DDE902233F
:1011E80004B0704700F1340191E838009C46A646E7
:1011F8004CF8045D90E8FF0FE54600BD90EC210B2C
:10120800704700BF80EC210B704700BF90EC200BAB
:10121800704700BF80EC200B704700BFD0EC200B5C
:10122800704700BFC0EC200B704700BFF0EC020114
:10123800F0EC0211F0EC0221F0EC0231F0EC02418A
:10124800F0EC0251F0EC0261F0EC0271F0EC02817A
:10125800F0EC0291F0EC02A1F0EC02B1F0EC02C16A
:10126800F0EC02D1F0EC02E1F0EC02F1704700BFC3
:10127800E0EC0201E0EC0211E0EC0221E0EC0231CA
:10128800E0EC0241E0EC0251E0EC0261E0EC0271BA
:10129800E0EC0281E0EC0291E0EC02A1E0EC02B1AA
:1012A800E0EC02C1E0EC02D1E0EC02E1E0EC02F19A
:1012B800704700BFB0FC0181B0FC0191B0FC01A1F6
:1012C800B0FC01B1704700BFA0FC0181A0FC0191F6
:1012D800A0FC01A1A0FC01B1704700BFEC4600B51D
:1012E8002DE900502DE9FF1F4FF000032DE90C00F8
:1012F80001A950F0EDFADDF840E012B0704700BFE8
:10130800EC4600B52DE900502DE9FF1F4FF0000312
:101318002DE90C0001A950F01BFBDDF840E012B0EC
:10132800704700BFEC4600B52DE900502DE9FF1FBE
:101338004FF000032DE90C0001A950F029FBDDF85E
:1013480040E012B0704700BFEC4600B52DE90050F0
:101358002DE9FF1F4FF000032DE90C0001AB50F001
:10136800EBFADDF840E012B0704700BFEC4600B57C
:101378002DE900502DE9FF1F4FF000032DE90C0067
:1013880001AA50F05FFBDDF840E012B0704700BFE3
:10139800704700BF80B400AF72B600BFBD4680BCC6
:1013A800704780B500AF0CF01DFD00BF80BD000088
:1013B80080B500AF0249022041F034FA00BF80BD79
:1013C8009823050880B500AFFFF7E4FFA34807603E
:1013D800A348C0F800E0864B1B681A46854B1A6084
:1013E800854B00221A7013E0824B1B68824A1278E0
:1013F80011461B68814A42F821307E4B1B68103326
:101408007C4A13607C4B1B780133DAB27A4B1A7032
:10141800794B1B78042BE7D9754B1B681A4678491A
:10142800022041F0FFF9774B1B681A4676490220E3
:1014380041F0F8F9704B00221A7012E06E4B1B78DD
:101448005A1C6D4B1B7819466C4B53F821306F4969
:10145800022041F0E7F9684B1B780133DAB2664B9A
:101468001A70654B1B78042BE8D9694BDB6A694A0B
:101478001360684B1B6803F00103002B03D0664917
:10148800022041F0CFF9634B1B6803F08043002B27
:1014980000F09A805E4B9B6A604A13605F4B1B6842
:1014A800DBB2002B03D05E49022041F0BBF95B4B55
:1014B8001B6803F47F43002B40D0584B1B6803F490
:1014C8007F43002B0AD0524B5B6B564A1360554B37
:1014D8001B681A465449022041F0A4F94F4B1B6877
:1014E80003F48053002B05D05049022041F09AF9AB
:1014F800FFF757FF494B1B6803F40063002B05D027
:101508004B49022041F08EF9FFF74BFF434B1B6814
:1015180003F40073002B05D04649022041F082F9FC
:10152800FFF73FFF3D4B1B6803F48073002B05D08A
:101538004149022041F076F9FFF733FF374B1B682A
:10154800B3F5803F40D3354B1B6803F40003002BF1
:101558000AD02F4B5B6B394A1360384B1B681A460D
:101568003749022041F05EF92C4B1B6803F48013C5
:10157800002B05D03349022041F054F9FFF711FF41
:10158800264B1B6803F40023002B05D02E490220AC
:1015980041F048F9FFF705FF204B1B6803F40033BF
:1015A800002B05D02949022041F03CF9FFF7F9FE4C
:1015B8001A4B1B6803F48033002B05D02449022002
:1015C80041F030F9FFF7EDFE124B1B6803F0804342
:1015D800002B05D01F49022041F024F9FFF7E1FE56
:1015E8001D49022041F01EF9FFF7DBFE00BF80BD58
:1015F8006416002070ED002068ED002050160020D1
:10160800A423050868160020B8230508CC2305087C
:1016180000ED00E058ED0020E02305086CED002007
:10162800F02305085CED0020202405084024050867
:101638007C240508C42405081425050864ED002049
:10164800682505088C250508D025050814260508F1
:1016580064260508B8260508EC2605086416002047
:101668006816002080B500AF0349022041F0DAF87F
:10167800FFF797FE00BF80BD0027050880B500AFC3
:101688000349022041F0CEF8FFF78BFE00BF80BD72
:101698001427050880B500AF0349022041F0C2F8BD
:1016A800FFF77FFE00BF80BD2027050880B500AF8B
:1016B8000249022041F0B6F800BF80BD2C2705087A
:1016C80080B500AF0249022041F0ACF800BF80BDF0
:1016D8003827050880B500AF0249022041F0A2F87A
:1016E80000BF80BD4C27050880B58CB000AF78607E
:1016F80039600023FB620023BB6200237B62002366
:101708003B620023FB617B68934A934213D07B685A
:10171800924A93420FD07B68914A93420BD07B68E0
:10172800904A934207D07B688F4A934203D0B821EE
:101738008E4809F0E9F83B681B68002B04D03B6829
:101748001B688B4A934203D9B921884809F0DCF811
:101758003B689B88002B08D03B689B88B3F5805F6B
:1017680003D0BA21814809F0CFF83B68DB88002B09
:1017780012D03B68DB88B3F5805F0DD03B68DB880F
:10178800B3F5005F08D03B68DB88B3F5405F03D052
:10179800BB21764809F0B8F83B681B89002B0DD0AF
:1017A8003B681B89B3F5806F08D03B681B89B3F58C
:1017B800C06F03D0BC216D4809F0A6F83B685B896F
:1017C8001A464FF6F3731340002B03D13B685B892D
:1017D800002B03D1BD21654809F096F83B689B8929
:1017E800002B12D03B689B89B3F5807F0DD03B68F6
:1017F8009B89B3F5007F08D03B689B89B3F5407F90
:1018080003D0BE21594809F07FF83B689B89002B1B
:101818000FD07B68504A93420BD07B684F4A934263
:1018280007D07B684E4A934203D0C2214F4809F043
:101838006BF87B68FB617B681B8A9BB2FB62FA6A68
:101848004CF6FF731340FB623B68DB881A46FB6A61
:101858001343FB62FB6A9AB27B681A827B689B8996
:101868009BB2FB62FA6A4EF6F3131340FB623B68C5
:101878009A883B681B8913439AB23B685B89134378
:101888009BB21A46FB6A1343FB62FB6A9AB27B68F7
:101898009A817B689B8A9BB2FB62FA6A4FF6FF4388
:1018A8001340FB623B689B891A46FB6A1343FB6241
:1018B800FB6A9AB27B689A8207F10803184601F01E
:1018C800ABFAFB69244A934202D17B69BB6201E00F
:1018D8003B69BB627B689B899BB21BB2002B0CDA0D
:1018E800BA6A13469B0013449A001A443B681B6863
:1018F8005B00B2FBF3F37B620BE0BA6A13469B0012
:1019080013449A001A443B681B689B00B2FBF3F32C
:101918007B627B6A174AA2FB03235B091B01FB62FC
:10192800FB6A1B09642202FB03F37A6AD31A3B623F
:101938007B689B899BB21BB2002B1DDA3B6ADB00DC
:1019480032330C4AA2FB03235B0903F00703FA6A4C
:101958001343FB621CE000BF003801400044004014
:1019680000480040004C0040005000405C2705083B
:1019780020AA44001F85EB513B6A1B013233084AF9
:10198800A2FB03235B0903F00F03FA6A1343FB620C
:10199800FB6A9AB27B681A8100BF3037BD4680BDAA
:1019A8001F85EB5180B483B000AF78607B684FF43B
:1019B80016521A607B6800229A807B680022DA80BF
:1019C8007B6800221A817B680C225A817B6800227E
:1019D8009A8100BF0C37BD4680BC704780B582B085
:1019E80000AF78600B46FB707B681D4A934214D0A9
:1019F8007B681C4A934210D07B681B4A93420CD0E8
:101A08007B681A4A934208D07B68194A934204D0EB
:101A18004FF4B171174808F077FFFB78002B07D017
:101A2800FB78012B04D040F26311124808F06CFFD8
:101A3800FB78002B08D07B689B899BB243F400534A
:101A48009AB27B689A8107E07B689B899BB223F4F2
:101A580000539AB27B689A8100BF0837BD4680BDA3
:101A6800003801400044004000480040004C00405D
:101A7800005000405C27050880B586B000AF78604C
:101A88000B467B8013467B7000233B610023FB6081
:101A98000023BB6000237B617B684C4A934214D0CF
:101AA8007B684B4A934210D07B684A4A93420CD0D9
:101AB8007B68494A934208D07B68484A934204D0DD
:101AC80040F28911464808F01FFF7B88282B25D053
:101AD8007B8840F22772934220D07B8840F22662AE
:101AE80093421BD07B8840F22552934216D07B88C4
:101AF80040F22442934211D07B8840F6460293423A
:101B08000CD07B8840F66A12934207D07B88602B02
:101B180004D04FF4C571324808F0F6FE7B78002BEC
:101B280007D07B78012B04D040F28B112C4808F0A9
:101B3800EBFE7B8840F66A12934210D17B68234AF9
:101B480093420CD07B68224A934208D07B68214A92
:101B5800934204D040F28F11214808F0D5FE7B68EB
:101B68007B617B88DBB25B09DBB23B617B8803F07E
:101B78001F03FB600122FB6802FA03F3BB603B69A9
:101B8800012B03D17B690C337B6109E03B69022B94
:101B980003D17B6910337B6102E07B6914337B617D
:101BA8007B78002B06D07B6919687B69BA680A4381
:101BB8001A6006E07B691968BB68DA437B690A40EA
:101BC8001A6000BF1837BD4680BD00BF003801400D
:101BD8000044004000480040004C004000500040D5
:101BE8005C27050880B582B000AF78600B467B8023
:101BF8007B68154A934214D07B68144A934210D0EC
:101C08007B68134A93420CD07B68124A934208D0EF
:101C18007B68114A934204D040F253210F4808F0E0
:101C280073FE7B88B3F5007F04D34FF415710B481E
:101C380008F06AFE7B88C3F308039AB27B689A802F
:101C480000BF0837BD4680BD003801400044004051
:101C580000480040004C0040005000405C27050848
:101C680080B582B000AF78607B68114A934214D087
:101C78007B68104A934210D07B680F4A93420CD07D
:101C88007B680E4A934208D07B680D4A934204D081
:101C98004FF419710B4808F037FE7B689B889BB29C
:101CA800C3F308039BB218460837BD4680BD00BF82
:101CB800003801400044004000480040004C00400B
:101CC800005000405C27050880B586B000AF7860FA
:101CD8000B467B800023FB6000237B610023BB60F5
:101CE8000023FB747B68554A934214D07B68544A9E
:101CF800934210D07B68534A93420CD07B68524A77
:101D0800934208D07B68514A934204D040F2C131D3
:101D18004F4808F0F9FD7B88282B2ED07B8840F2AD
:101D28002772934229D07B8840F22662934224D0BE
:101D38007B8840F2255293421FD07B8840F2244290
:101D480093421AD07B8840F64602934215D07B888E
:101D580040F66A12934210D07B88B3F5587F0CD0B6
:101D68007B88B3F5187F08D07B88B3F5B07F04D0A3
:101D780040F2C231364808F0C7FD7B8840F66A1247
:101D8800934210D17B682D4A93420CD07B682C4A31
:101D9800934208D07B682B4A934204D040F2C63164
:101DA8002B4808F0B1FD7B88DBB25B09DBB2BB6076
:101DB8007B8803F01F037B6101227B6902FA03F32E
:101DC8007B61BB68012B07D17B689B899BB21A4654
:101DD8007B6913407B6111E0BB68022B07D17B68EC
:101DE8001B8A9BB21A467B6913407B6106E07B68BD
:101DF8009B8A9BB21A467B6913407B617B881B0ACE
:101E08009BB2FB600122FB6802FA03F3FB607B686C
:101E18001B889BB21A46FB681340FB607B69002B4A
:101E280005D0FB68002B02D00123FB7401E00023DE
:101E3800FB74FB7C18461837BD4680BD003801404E
:101E48000044004000480040004C00400050004062
:101E58005C27050880B584B000AF78600B467B80AE
:101E68000023FB810023BB817B682C4A934214D05A
:101E78007B682B4A934210D07B682A4A93420CD045
:101E88007B68294A934208D07B68284A934204D049
:101E980040F20A41264808F037FD7B8840F2266266
:101EA800934213D07B8840F2255293420ED07B8810
:101EB80040F64602934209D07B8840F66A12934264
:101EC80004D040F20B411A4808F01EFD7B8840F60A
:101ED8006A12934210D17B68104A93420CD07B68F7
:101EE8000F4A934208D07B680E4A934204D040F2CE
:101EF8000F410F4808F008FD7B881B0AFB81FB890E
:101F0800012202FA03F3BB81BB89DB439AB27B68E7
:101F18001A8000BF1037BD4680BD00BF00380140A1
:101F28000044004000480040004C00400050004081
:101F38005C27050880B586B000AF786000237B6118
:101F480000233B610F23FB607B68DB78002B07D005
:101F58007B68DB78012B03D07521334808F0D4FC6B
:101F68007B685B780F2B03D976212F4808F0CCFCCF
:101F78007B689B780F2B03D977212B4808F0C4FC8A
:101F88007B68DB78002B3AD0284BDB68DB431B0AE5
:101F980003F007037B617B69C3F104033B61FA68C3
:101FA8007B6922FA03F3FB607B685B781A463B691E
:101FB80002FA03F37B617B689B781A46FB6813403F
:101FC8007A6913437B617B691B017B61184A7B68D3
:101FD8001B787969C9B213440A4683F800237B68E1
:101FE8001B7803F01F0312497A6812785209D2B29B
:101FF8001046012202FA03F341F820300FE07B6813
:102008001B7803F01F030A497A6812785209D2B282
:10201800104601229A4000F1200341F8232000BF16
:102028001837BD4680BD00BFE427050800ED00E075
:1020380000E100E080B584B000AF78600023FB6069
:102048007B68002B0AD07B68012B07D07B68022BAA
:1020580004D040F203110A4808F056FC094B1B68EB
:10206800FB60FB6803F03803FB60FA687B68134386
:10207800FB60044AFB68136000BF1037BD4680BD93
:10208800602805080020024080B582B000AF786063
:102098007B68102B07D07B68002B04D040F22F11EF
:1020A800094808F031FC094B1B68084A23F0100363
:1020B8001360064B1A6805497B6813430B6000BF21
:1020C8000837BD4680BD00BF6028050800200240D3
:1020D80080B400AF074B084A5A60064B074A5A605B
:1020E800044B054A5A64034B044A5A6400BFBD4670
:1020F80080BC70470020024023016745AB89EFCDC3
:1021080080B400AF074B1B69064A43F08003136194
:10211800044B1B6D034A43F08003136500BFBD46A3
:1021280080BC70470020024080B584B000AF786062
:102138000423FB737B68B3F1006F03D37B682E4ADB
:10214800934204D940F2A7112C4808F0DDFB7B68C4
:102158002B4A934225D24FF4302000F04BFA034625
:10216800FB73FB7B042B41D1264B1B69254A43F0AB
:1021780002031361234A7B685361224B1B69214A7E
:1021880043F0400313614FF4302000F033FA034664
:10219800FB731C4B1A691B4941F6FD7313400B6115
:1021A80024E04FF4302000F047FA0346FB73FB7B32
:1021B800042B1BD1134B1B6D124A43F0020313650A
:1021C800104A7B6853650F4B1B6D0E4A43F0400362
:1021D80013654FF4302000F02FFA0346FB73094BC8
:1021E8001A6D084941F6FD7313400B65FB7B1846D1
:1021F8001037BD4680BD00BFFEFF0F0860280508E8
:10220800FFFF07080020024080B582B000AFA52379
:10221800FB8004237B7100F039F90346002B01D0C1
:102228000023FB804FF4302000F0C2F903467B7195
:102238007B79042B45D1254B254A9A60234B254AA7
:102248009A60224B1B69214A43F0200313611F4BFC
:102258001B691E4A43F0400313614FF4302000F01D
:10226800A7F903467B717B79042B20D1174B1A6998
:10227800164941F6DF7313400B61144B1B69134A6F
:1022880043F010031361144AFB8813804FF4005085
:1022980000F08EF903467B717B79052B11D00B4B2F
:1022A8001A690A4941F6EF7313400B6109E07B791B
:1022B800052B06D0054B1A69044941F6EF73134004
:1022C8000B617B7918460837BD4680BD0020024067
:1022D80023016745AB89EFCD00F8FF1F80B584B0B7
:1022E80000AF78600B467B800423FB737B68B3F1F7
:1022F800006F03D37B68254A934204D940F25E31CC
:10230800234808F001FB4FF4005000F051F9034650
:10231800FB737B681F4A934219D2FB7B042B2FD196
:102328001D4B1B691C4A43F0010313617B687A88C3
:102338001A804FF4005000F05DF90346FB73164B0A
:102348001A69154941F6FE7313400B6118E0FB7BCF
:10235800042B15D1104B1B6D0F4A43F00103136575
:102368007B687A881A804FF4005000F065F90346BC
:10237800FB73094B1A6D084941F6FE7313400B6550
:10238800FB7B18461037BD4680BD00BFFEFF0F0817
:1023980060280508FFFF07080020024080B584B0C8
:1023A80000AF0346FB710423FB73FB79002B07D0B6
:1023B800FB79012B04D040F21D412F4808F0A4FA04
:1023C8004FF4302000F0F4F80346FB73FB7B042B3A
:1023D8004CD12A4B2A4A9A60284B2A4A9A60274BA2
:1023E8001B69264A43F020031361244B1B69234AC7
:1023F80043F0400313614FF4302000F0D9F803464E
:10240800FB73FB7B042B27D11C4B1A691B4941F634
:10241800DF7313400B61194B1B69184A43F0100313
:102428001361FB79002B03D0174B00221A8002E0BE
:10243800154BA5221A804FF4302000F0B9F8034656
:10244800FB73FB7B052B11D00C4B1A690B4941F62A
:10245800EF7313400B6109E0FB7B052B06D0074B9C
:102468001A69064941F6DF7313400B61FB7B184676
:102478001037BD4680BD00BF602805080020024017
:1024880023016745AB89EFCD00F8FF1F80B483B007
:1024980000AF0023FB71084BDB6903F00203002B3C
:1024A80002D00123FB7101E00023FB71FB79184680
:1024B8000C37BD4680BC70470020024080B582B012
:1024C80000AF78607B6823F0004323F03503002BCE
:1024D80002D17B68002B04D140F2A751084808F0CC
:1024E80013FA7B68002B03DA064A7B68D36402E0A0
:1024F800044A7B68D36000BF0837BD4680BD00BF73
:10250800602805080020024080B483B000AF04238F
:10251800FB71114BDB6803F00103012B02D101238E
:10252800FB7113E00C4BDB6803F00403002B02D0B3
:102538000223FB710AE0084BDB6803F01003002B51
:1025480002D00323FB7101E00423FB71FB791846D9
:102558000C37BD4680BC70470020024080B483B071
:1025680000AF0423FB71114BDB6C03F00103012B5B
:1025780002D10123FB7113E00C4BDB6C03F0040365
:10258800002B02D00223FB710AE0084BDB6C03F03E
:102598001003002B02D00323FB7101E00423FB711D
:1025A800FB7918460C37BD4680BC704700200240B6
:1025B80080B584B000AF78600423FB73FFF7A4FFF5
:1025C8000346FB7306E0FFF79FFF0346FB737B6838
:1025D800013B7B60FB7B012B02D17B68002BF2D196
:1025E8007B68002B01D10523FB73FB7B1846103752
:1025F800BD4680BD80B584B000AF78600423FB730E
:10260800FFF782FF0346FB7306E0FFF77DFF0346F3
:10261800FB737B68013B7B60FB7B012B02D17B68F2
:10262800002BF2D17B68002B01D10523FB73FB7BC8
:1026380018461037BD4680BD80B584B000AF7860BD
:102648000423FB73FFF78AFF0346FB7306E0FFF7DB
:1026580085FF0346FB737B68013B7B60FB7B012B9B
:1026680002D17B68002BF2D17B68002B01D10523B6
:10267800FB73FB7B18461037BD4680BD80B582B022
:1026880000AF78607B683F4A93421BD07B683E4A24
:10269800934217D07B683D4A934213D07B683C4AEB
:1026A80093420FD07B683B4A93420BD07B683A4AEF
:1026B800934207D07B68394A934203D06F21384848
:1026C80008F022F97B682F4A934208D1012104209F
:1026D80000F0CCFC0021042000F0C8FC4EE07B6830
:1026E800294A934208D10121082000F0BFFC0021AB
:1026F800082000F0BBFC41E07B68244A934208D1E3
:102708000121102000F0B2FC0021102000F0AEFCE6
:1027180034E07B681E4A934208D10121202000F052
:10272800A5FC0021202000F0A1FC27E07B68194AC5
:10273800934208D10121402000F098FC002140205C
:1027480000F094FC1AE07B68134A934208D10121F7
:10275800802000F08BFC0021802000F087FC0DE039
:102768007B680E4A934209D101214FF4807000F032
:102778007DFC00214FF4807000F078FC00BF083722
:10278800BD4680BD00080140000C0140001001401A
:102798000014014000180140001C014000200140C5
:1027A800E828050880B588B000AF78603960002354
:1027B800FB6100233B610023BB610023FB60002316
:1027C8007B610023BB607B68824A93421BD07B6895
:1027D800814A934217D07B68804A934213D07B6822
:1027E8007F4A93420FD07B687E4A93420BD07B6826
:1027F8007D4A934207D07B687C4A934203D0B2213A
:102808007B4808F081F83B68DB78002B1FD03B68D9
:10281800DB78042B1BD03B68DB78282B17D03B6870
:10282800DB78482B13D03B68DB78142B0FD03B6840
:10283800DB78102B0BD03B68DB781C2B07D03B6870
:10284800DB78182B03D0B321694808F05DF83B68A2
:102858001B88002B03D1B421654808F055F83B6864
:10286800DB7803F00F03FB613B68DB7803F01003B0
:10287800002B15D03B689B78012B0BD03B689B78CD
:10288800022B07D03B689B78032B03D0BB21584809
:1028980008F03AF83B689B781A46FB691343FB61DA
:1028A8003B681B88DBB2002B44D07B681B687B61CC
:1028B8000023BB6138E00122BB6902FA03F3FB6025
:1028C8003B681B881A46FB6813403B613A69FB6802
:1028D8009A4226D1BB699B00FB600F22FB6802FA73
:1028E80003F3BB60BB68DB437A6913407B61FA6919
:1028F800FB6802FA03F37A6913437B613B68DB7870
:10290800282B05D10122BB699A407B685A6108E0EF
:102918003B68DB78482B04D10122BB699A407B686D
:102928001A61BB690133BB61BB69072BC3D97B68DB
:102938007A691A603B681B88FF2B46D97B685B68FD
:102948007B610023BB613AE0BB690833012202FACC
:1029580003F3FB603B681B881A46FB6813403B6126
:102968003A69FB689A4227D1BB699B00FB600F223A
:10297800FB6802FA03F3BB60BB68DB437A69134068
:102988007B61FA69FB6802FA03F37A6913437B6196
:102998003B68DB78282B05D1BB69083301229A40B4
:1029A8007B685A613B68DB78482B05D1BB690833E3
:1029B80001229A407B681A61BB690133BB61BB691C
:1029C800072BC1D97B687A695A6000BF2037BD469A
:1029D80080BD00BF00080140000C0140001001400C
:1029E8000014014000180140001C01400020014073
:1029F800E828050880B582B000AF78607B68134A84
:102A080093421CD07B68124A934218D07B68114AC3
:102A1800934214D07B68104A934210D07B680F4AC7
:102A280093420CD07B680E4A934208D07B680D4ACB
:102A3800934204D04FF49A710B4807F065FF7B6806
:102A48009B689BB218460837BD4680BD0008014008
:102A5800000C014000100140001401400018014022
:102A6800001C014000200140E828050880B584B01A
:102A780000AF78600B467B800023FB737B68364A87
:102A880093421CD07B68354A934218D07B68344AFD
:102A9800934214D07B68334A934210D07B68324A01
:102AA80093420CD07B68314A934208D07B68304A05
:102AB800934204D04FF4A2712E4807F025FF7B887B
:102AC800012B39D07B88022B36D07B88042B33D05E
:102AD8007B88082B30D07B88102B2DD07B88202B2F
:102AE8002AD07B88402B27D07B88802B24D07B88DA
:102AF800B3F5807F20D07B88B3F5007F1CD07B881E
:102B0800B3F5806F18D07B88B3F5006F14D07B883D
:102B1800B3F5805F10D07B88B3F5005F0CD07B885D
:102B2800B3F5804F08D07B88B3F5004F04D040F24E
:102B38004511104807F0E8FE7B68DA687B88134087
:102B4800002B02D00123FB7301E00023FB73FB7B06
:102B580018461037BD4680BD00080140000C0140F2
:102B6800001001400014014000180140001C014001
:102B780000200140E828050880B582B000AF7860E1
:102B88000B467B807B68174A93421CD07B68164AA9
:102B9800934218D07B68154A934214D07B68144A34
:102BA800934210D07B68134A93420CD07B68124A38
:102BB800934208D07B68114A934204D040F26911CD
:102BC8000F4807F0A1FE7B88002B04D14FF4B571A4
:102BD8000B4807F099FE7A887B681A6100BF0837AE
:102BE800BD4680BD00080140000C014000100140B6
:102BF8000014014000180140001C01400020014061
:102C0800E828050880B582B000AF78600B467B8065
:102C18007B68174A93421CD07B68164A934218D0A7
:102C28007B68154A934214D07B68144A934210D0AB
:102C38007B68134A93420CD07B68124A934208D0AF
:102C48007B68114A934204D040F279110F4807F08B
:102C58005BFE7B88002B04D14FF4BD710B4807F055
:102C680053FE7A887B685A6100BF0837BD4680BD2D
:102C780000080140000C0140001001400014014010
:102C880000180140001C014000200140E828050808
:102C980080B582B000AF78600B467B8013467B70AE
:102CA8007B683B4A93421CD07B683A4A934218D0CF
:102CB8007B68394A934214D07B68384A934210D0D3
:102CC8007B68374A93420CD07B68364A934208D0D7
:102CD8007B68354A934204D040F28D11334807F09F
:102CE80013FE7B88012B39D07B88022B36D07B885A
:102CF800042B33D07B88082B30D07B88102B2DD029
:102D08007B88202B2AD07B88402B27D07B88802B60
:102D180024D07B88B3F5807F20D07B88B3F5007FF3
:102D28001CD07B88B3F5806F18D07B88B3F5006F13
:102D380014D07B88B3F5805F10D07B88B3F5005F33
:102D48000CD07B88B3F5804F08D07B88B3F5004F53
:102D580004D04FF4C771154807F0D6FD7B78002BD7
:102D680007D07B78012B04D040F28F110F4807F071
:102D7800CBFD7B78002B03D07A887B681A6102E050
:102D88007A887B685A6100BF0837BD4680BD00BF9E
:102D980000080140000C01400010014000140140EF
:102DA80000180140001C014000200140E8280508E7
:102DB80080B584B000AF78600023FB607B68002B8F
:102DC80014D07B68B3F5806F10D07B68B3F5A06F23
:102DD8000CD07B68B3F5C06F08D07B68B3F5E06FA3
:102DE80004D040F27E210A4807F08EFD094B5B684B
:102DF800FB60FB6823F4E063FB60FA687B681343BD
:102E0800FB60044AFB68536000BF1037BD4680BDB5
:102E1800702905080010024080B487B000AF7860C0
:102E280000237B6100233B610023FB600023BB6020
:102E38004F4B5B6803F00C037B617B69082B11D057
:102E48007B69082B3AD87B69002B03D07B69042B5C
:102E580004D033E07B68474A1A6033E07B68454A10
:102E68001A602FE0424B5B6803F470133B61404BE0
:102E78005B6803F48033FB603B699B0C02333B6166
:102E8800FB68002B06D13B693B4A03FB02F27B68D7
:102E98001A6017E0364B5B6803F40033002B06D04A
:102EA8003B69354A03FB02F27B681A600AE03B691A
:102EB800304A03FB02F27B681A6003E07B682D4A04
:102EC8001A6000BF2A4B5B6803F0F0037B617B69E3
:102ED8001B097B61294A7B6913441B78DBB2BB6001
:102EE8007B681A68BB68DA407B685A60204B5B686D
:102EF80003F4E0637B617B691B0A7B611F4A7B6982
:102F080013441B78DBB2BB607B685A68BB68DA4045
:102F18007B689A60164B5B6803F460537B617B693E
:102F2800DB0A7B61154A7B6913441B78DBB2BB6003
:102F38007B685A68BB68DA407B68DA600C4B5B6870
:102F480003F440437B617B699B0B7B610C4A7B6983
:102F580013441B78DBB2BB607B68DA68BB68B2FBE2
:102F6800F3F27B681A6100BF1C37BD4680BC70470E
:102F78000010024000127A0000093D000000002005
:102F88001000002080B582B000AF78600B46FB705F
:102F98007A68164B1340002B02D17B68002B04D1B2
:102FA80040F24A41124807F0AFFCFB78002B07D0EB
:102FB800FB78012B04D040F24B410D4807F0A4FCEC
:102FC800FB78002B06D00B4B9A690A497B681343A0
:102FD8008B6106E0074B9A697B68DB430549134020
:102FE8008B6100BF0837BD4680BD00BF0200C0FF2F
:102FF800702905080010024080B582B000AF7860E3
:103008000B46FB707A68164B1340002B02D17B6885
:10301800002B04D140F26941124807F075FCFB7897
:10302800002B07D0FB78012B04D040F26A410D48F1
:1030380007F06AFCFB78002B06D00B4BDA690A49CB
:103048007B681343CB6106E0074BDA697B68DB4397
:1030580005491340CB6100BF0837BD4680BD00BF9E
:1030680000360181702905080010024080B582B041
:1030780000AF78600B46FB707A68164B1340002B44
:1030880002D17B68002B04D140F2A441124807F01A
:103098003BFCFB78002B07D0FB78012B04D040F2D7
:1030A800A5410D4807F030FCFB78002B06D00B4BF0
:1030B800DA680A497B681343CB6006E0074BDA6895
:1030C8007B68DB4305491340CB6000BF0837BD462A
:1030D80080BD00BF0200C0FF702905080010024033
:1030E80080B584B000AF786039600023FB817B68CD
:1030F800684A934243D07B68B3F1804F3FD07B68E6
:10310800654A93423BD07B68644A934237D07B68D8
:10311800634A934233D07B68624A93422FD07B68DC
:10312800614A93422BD07B68604A934227D07B68E0
:103138005F4A934223D07B685E4A93421FD07B68E4
:103148005D4A93421BD07B685C4A934217D07B68E8
:103158005B4A934213D07B685A4A93420FD07B68EC
:10316800594A93420BD07B68584A934207D07B68F0
:10317800574A934203D0E721564807F0C5FB3B68FE
:103188005B88002B13D03B685B88102B0FD03B6803
:103198005B88202B0BD03B685B88402B07D03B68B3
:1031A8005B88602B03D0E8214A4807F0ADFB3B68F9
:1031B800DB88002B0DD03B68DB88B3F5807F08D017
:1031C8003B68DB88B3F5007F03D0E921414807F06D
:1031D8009BFB7B681B88FB817B682E4A934213D03C
:1031E8007B68324A93420FD07B68B3F1804F0BD093
:1031F8007B68294A934207D07B68284A934203D0C8
:103208007B68274A934208D1FB8923F07003FB812E
:103218003B685A88FB891343FB817B68214A9342A8
:103228000CD07B68204A934208D0FB8923F4407372
:10323800FB813B68DA88FB891343FB817B68FA8949
:103248001A803B689A887B689A853B681A887B68ED
:103258001A857B680F4A93420FD07B68134A9342C2
:103268000BD07B68184A934207D07B68174A934271
:1032780003D07B68164A934204D13B681B7A1A46EE
:103288007B681A867B6801229A8200BF1037BD4688
:1032980080BD00BF002C0140000400400008004031
:1032A800000C0040001000400014004000340140B1
:1032B800004C0140005001400054014000180040FB
:1032C800001C004000200040004001400044014034
:1032D80000480140F829050880B582B000AF786041
:1032E8000B46FB707B68354A934244D07B68B3F148
:1032F800804F40D07B68324A93423CD07B68314A49
:10330800934238D07B68304A934234D07B682F4A46
:10331800934230D07B682E4A93422CD07B682D4A4A
:10332800934228D07B682C4A934224D07B682B4A4E
:10333800934220D07B682A4A93421CD07B68294A52
:10334800934218D07B68284A934214D07B68274A56
:10335800934210D07B68264A93420CD07B68254A5A
:10336800934208D07B68244A934204D040F2293122
:10337800224807F0C9FAFB78002B07D0FB78012B0D
:1033880004D040F22A311D4807F0BEFAFB78002B22
:1033980008D07B681B889BB243F001039AB27B6814
:1033A8001A8007E07B681B889BB223F001039AB25E
:1033B8007B681A8000BF0837BD4680BD002C0140DD
:1033C8000004004000080040000C004000100040CD
:1033D8000014004000340140004C014000500140FE
:1033E8000054014000180040001C0040002000402C
:1033F800004001400044014000480140F829050808
:1034080080B582B000AF78600B467B8013467B7036
:103418007B683D4A934244D07B68B3F1804F40D0EB
:103428007B683A4A93423CD07B68394A934238D009
:103438007B68384A934234D07B68374A934230D00D
:103448007B68364A93422CD07B68354A934228D011
:103458007B68344A934224D07B68334A934220D015
:103468007B68324A93421CD07B68314A934218D019
:103478007B68304A934214D07B682F4A934210D01D
:103488007B682E4A93420CD07B682D4A934208D021
:103498007B682C4A934204D040F26B312A4807F0EB
:1034A80033FA7B8803F47F43002B02D17B88002BFF
:1034B80004D14FF45B71244807F026FA7B78002B7F
:1034C80007D07B78012B04D040F26D311E4807F0FD
:1034D8001BFA7B78002B08D07B689B899AB27B8883
:1034E80013439AB27B689A8109E07B689B899AB2F8
:1034F8007B88DB439BB213409AB27B689A8100BFFA
:103508000837BD4680BD00BF002C014000040040C4
:1035180000080040000C004000100040001400406B
:1035280000340140004C014000500140005401406B
:1035380000180040001C00400020004000400140EE
:103548000044014000480140F829050880B582B0D0
:1035580000AF78600B467B807B682F4A934244D04B
:103568007B68B3F1804F40D07B682C4A93423CD0B3
:103578007B682B4A934238D07B682A4A934234D0DE
:103588007B68294A934230D07B68284A93422CD0E2
:103598007B68274A934228D07B68264A934224D0E6
:1035A8007B68254A934220D07B68244A93421CD0EA
:1035B8007B68234A934218D07B68224A934214D0EE
:1035C8007B68214A934210D07B68204A93420CD0F2
:1035D8007B681F4A934208D07B681E4A934204D0F6
:1035E80040F677211C4807F08FF97B8803F47F4366
:1035F800002B02D17B88002B04D140F67821164895
:1036080007F082F97B88DB439AB27B681A8200BF95
:103618000837BD4680BD00BF002C014000040040B3
:1036280000080040000C004000100040001400405A
:1036380000340140004C014000500140005401405A
:1036480000180040001C00400020004000400140DD
:103658000044014000480140F829050880B500AF42
:10366800194B1B68184A43F001031360164B5A683C
:103678001549164B13404B60134B1B68124A23F035
:10368800847323F4803313600F4B1B680E4A23F4B2
:10369800802313600C4B5B680B4A23F4FE035360D2
:1036A800094B4FF41F029A60094B00221A60094B1C
:1036B80000221A6000F084F800F010F8064B4FF072
:1036C80000629A6000BF80BD001002400000FFF851
:1036D8007CED002078ED002000ED00E080B485B09E
:1036E80000AF0023FB600023BB6000237B602F4BEF
:1036F8005B6803F00C03FB60FB68082B11D0FB68C8
:10370800082B3AD8FB68002B03D0FB68042B04D0A5
:1037180033E0274B274A1A6033E0254B254A1A60C5
:103728002FE0224B5B6803F47013BB601F4B5B6890
:1037380003F480337B60BB689B0C0233BB607B68FF
:10374800002B06D1BB681C4A02FB03F3184A13601E
:1037580017E0164B5B6803F40033002B06D0BB68F8
:10376800154A02FB03F3124A13600AE0BB68114AC8
:1037780002FB03F30E4A136003E00D4B0D4A1A6077
:1037880000BF0A4B5B681B0903F00F030B4AD35CAD
:10379800DBB2FB60064B1A68FB6822FA03F3044AA3
:1037A800136000BF1437BD4680BC7047001002404C
:1037B8001400002000127A0000093D0018000020C3
:1037C80080B500AF00F002F800BF80BD80B582B0C0
:1037D80000AF00237B6000233B603F4B1B683E4AE1
:1037E80043F4803313603C4B1B6803F400333B60A5
:1037F8007B6801337B603B68002B03D17B68B3F5A2
:10380800A06FF0D1344B1B6803F40033002B02D0B7
:1038180001233B6001E000233B603B68012B4FD153
:103828002E4B1B682D4A43F0100313602B4B1B686B
:103838002A4A23F003031360284B1B68274A43F0E6
:1038480002031360244B244A5B685360224B224ACC
:103858005B685360204B5B681F4A43F48063536086
:103868001D4B5B681C4A23F47C1353601A4B5B683E
:10387800194A43F4E8135360174B1B68164A43F080
:103888008073136000BF144B1B6803F00073002B98
:10389800F9D0114B5B68104A23F0030353600E4BB9
:1038A8005B680D4A43F00203536000BF0A4B5B6834
:1038B80003F00C03082BF9D1094B01221A6007E029
:1038C800084B01221A60064B00221A6000F00CF81F
:1038D80000BF0837BD4680BD0010024000200240EE
:1038E80078ED00207CED002080B483B000AF002389
:1038F8007B6000233B60424B01221A60414B1B68EE
:10390800404A23F4803313603E4B1B683D4A43F022
:10391800010313603B4B1B6803F002033B607B68A9
:1039280001337B603B68002B03D17B68B3F5A06F44
:10393800F0D1344B1B6803F00203002B02D00123A3
:103948003B6001E000233B603B68012B4FD12E4BCD
:103958001B682D4A43F0100313602B4B1B682A4A3F
:1039680023F003031360284B1B68274A43F0020324
:103978001360244B234A5B685360224B214A5B68DF
:103988005360204B5B681F4A43F4806353601D4BB0
:103998005B681C4A23F47C1353601A4B5B68194A12
:1039A80043F4E0135360174B1B68164A43F08073C7
:1039B800136000BF134B1B6803F00073002BF9D092
:1039C800104B5B680F4A23F0030353600D4B5B6891
:1039D8000C4A43F00203536000BF0A4B5B6803F0D4
:1039E8000C03082BF9D1094B02221A6002E0074B9D
:1039F80003221A6000BF0C37BD4680BC704700BF69
:103A08007CED0020001002400020024078ED0020EC
:103A180080B500AF00214FF47B7000F0AAF802F0E7
:103A2800C3F8FCE780B58EB000AF002000F0D0F8F6
:103A3800034687F8373066233B723B1D1A46002140
:103A4800002008F0B7FAD7F80930B3F1FF3F30D0BB
:103A5800D7F80930184A536097F83730164A9360F8
:103A6800164B002242F001029A730022DA730022F8
:103A78001A7400225A74114B002242F002021A7181
:103A880000225A710D4B00229A720022DA7200222B
:103A98001A7300225A73094B00229A710022DA71B4
:103AA80000221A7200225A7203494FF47B7000F008
:103AB8006FF802F079F8FCE790ED0020A8ED0020FF
:103AC80080B58EB000AF012000F082F8034687F879
:103AD800373067233B723B1D1A460021002008F04F
:103AE80069FAD7F80930B3F1FF3F34D0D7F8093075
:103AF8001A4A536097F83730184A9360184B0022D7
:103B080042F001021A7700225A7700229A7700229F
:103B1800DA77134B002242F002029A740022DA7418
:103B28000F4B002242F001021A7600225A76002238
:103B38009A760022DA760A4B002242F001021A75C0
:103B480000225A7500229A750022DA7503494FF44B
:103B58007B7000F02DF802F027F8FCE780ED0020DC
:103B6800A8ED002080B500AF01F0EAFF02F01CF8D4
:103B7800FCE780B582B000AF03463960FB80FB8864
:103B88003968184602F0D8FE00BF0837BD4680BD28
:103B980080B582B000AF03463960FB80FB883A6885
:103BA800194600200AF01CFC00BF0837BD4680BD3E
:103BB80080B582B000AF03463960FB80FB883A6865
:103BC800194601200AF00CFC00BF0837BD4680BD2D
:103BD80080B588B000AF0346FB710023BB820A237F
:103BE800FB8207F10803BB6107F1140319460120A2
:103BF80009F032FEFB79002B04D107F108030433E6
:103C0800FB6103E007F108030933FB61FB691B78DB
:103C1800DC2B0DD0FB691B78D92B09D0FB691B78ED
:103C2800C72B05D9FB691B78E52B01D8012300E0D8
:103C38000023002B01D1C82301E0FB691B7818463B
:103C48002037BD4680BD80B483B000AF786039604E
:103C58007B68002B05DD7A683B689A4201DC01230A
:103C680000E0002318460C37BD4680BC70470000B2
:103C780080B582B000AF786039607B68002B1BD0BC
:103C88007B68002B29DB7B68B3F57B7F25DC7B68B1
:103C9800B3F57A7F21DD7B68A3F2E933032B1CD8C7
:103CA80001A252F823F000BFCB3C0008D33C000827
:103CB800DB3C0008C13C0008386800F0FDF803460A
:103CC800F6E0386801F09EFE07E0386801F0B5FEBE
:103CD80003E0386801F0A8FE00BF7B68013B342B85
:103CE80000F2E58001A252F823F000BFC93D0008A8
:103CF800D33D0008B73E0008B73E0008B73E0008AD
:103D0800B73E0008B73E0008B73E0008B73E0008B7
:103D1800DD3D0008E73D0008F13D0008FB3D0008D7
:103D2800053E00080F3E0008193E0008233E000823
:103D3800B73E0008B73E0008373E00083F3E00087F
:103D4800B73E00082D3E0008493E0008B73E00086F
:103D5800B73E0008B73E0008B73E0008B73E000867
:103D6800B73E00085D3E0008673E0008533E000865
:103D7800713E0008B73E0008B73E0008B73E00088D
:103D8800B73E0008B73E0008853E00087B3E0008A5
:103D98008F3E0008B73E0008B73E0008B73E00084F
:103DA800B73E0008B73E0008B73E0008B73E000817
:103DB800993E0008B73E0008A33E0008AD3E000843
:103DC800386800F0AFF8034672E0386800F0DEF9B2
:103DD80003466DE0386800F0FDFC034668E038688B
:103DE80000F08EFB034663E0386800F011FE0346DE
:103DF8005EE0386800F0B7FB034659E0386800F029
:103E0800A3FC034654E0386800F0F6FB03464FE095
:103E1800386800F024FC03464AE0386800F06DFD7D
:103E2800034645E0386800F05BFE034640E000F0DA
:103E38003DFE03463CE0386800F0C6FE034637E026
:103E4800386800F08FFE034632E0386800F0F6FE6E
:103E580003462DE0386800F025FF034628E038685F
:103E680000F0FCFF034623E0386800F063FF0346D8
:103E78001EE0386801F034FB034619E0386801F0A9
:103E880023FC034614E0386801F024FD03460FE0E4
:103E9800386801F0F7FA03460AE0386801F012F8CA
:103EA800034605E0386801F011FA034600E00123F3
:103EB80018460837BD4680BD80B58AB000AF786027
:103EC8007B683B623B6ADB69FB6100237B6221E024
:103ED8007A6AFB69134401337B617A6AFB6913448C
:103EE8000133FB6007F10803184601F06BFD034638
:103EF800002B0CD1BB69D3F80620BB6922F08002E5
:103F0800C3F8062007F10803184601F06FFD7B6A25
:103F180001337B627B6A0F2BDADD002318462837D2
:103F2800BD4680BD80B58CB000AF78607B68BB6251
:103F3800BB6ADB6901337B62BB6A002283F83820E5
:103F4800002283F83920002283F83A20002283F8DF
:103F58003B207B6A7B617B6A6433FB6007F1080363
:103F6800184601F02FFDF862FB6A002B40F0038130
:103F7800BB6A002283F8CA20002283F8CB200022E3
:103F880083F8CC20002283F8CD20BB69D3F80A300F
:103F980003F48053002B17D0BB69D3F80A20BB6900
:103FA80022F48052C3F80A20BB6A002242F00202BF
:103FB80083F8CA20002283F8CB20002283F8CC2083
:103FC800002283F8CD20D0E0BB69D3F8063003F493
:103FD8008073002B20D1BB69D3F8063003F48063CB
:103FE800002B01D03EF02CFABB69D3F80620BB6940
:103FF80022F48062C3F80620BB6A002242F0020263
:1040080083F8CA20002283F8CB20002283F8CC2032
:10401800002283F8CD20A8E0BB6A002242F001020A
:1040280083F8CA20002283F8CB20002283F8CC2012
:10403800002283F8CD20BB69D3F8063003F48063EF
:10404800002B07D1BB6AD3F8CA3043F02002BB6A01
:10405800C3F8CA20BB6A20333B62BB6A2433FB61C6
:104068003B6A00221A60FB6900221A60BB6A0022C0
:1040780083F8B220002283F8B320002283F8B4200A
:10408800002283F8B520BB69D3F8063003F040035B
:10409800002B05D13B6A1B6843F004023B6A1A6097
:1040A800BB69D3F80A3003F00403002B05D03B6A40
:1040B8001B6843F008023B6A1A60BB69D3F80A30F0
:1040C80003F00103002B2CD0BB69D3F80A3003F0AE
:1040D8003003002B25D03B6A1B6843F002023B6A81
:1040E8001A60BB699A7D3B6A04331A60BB69D3F8CE
:1040F8000A3003F40073002B13D0BB69D3F80A30DD
:1041080003F00403002B06D1FB691B6843F400721B
:10411800FB691A6005E0FB691B6843F48072FB6960
:104128001A60BB69D3F81120BB6942F00402C3F8D6
:104138001120BB69D3F8113003F00103002B05D01F
:104148003B6A1B6843F001023B6A1A60BB69D3F8FB
:10415800113003F00203002B06D03B6A1B6843F0C2
:1041680010023B6A1A6000E000BF07F10803184616
:1041780001F03CFC05E00323FB62BB6AFA6AC3F862
:10418800CA20FB6A18463037BD4680BD80B590B05E
:1041980000AF78607B68FB62FB6ADB690133BB6256
:1041A80000233B6300237B63FB6A002283F8CA2059
:1041B800002283F8CB20002283F8CC20002283F849
:1041C800CD20BB6ABB61BB6AC8333B6107F10C03F6
:1041D800184601F0F7FB0346002B40F08681FB6987
:1041E8007B627B6AD3F8063023F080027B6AC3F8CF
:1041F80006207B6AD3F80A3003F08003002B29D10C
:10420800FB6ADB6A03F08003002B11D07B6AD3F8CA
:10421800063003F02003002B01D101233B637B6AA6
:10422800D3F8063043F020027B6AC3F8062017E073
:104238007B6AD3F8063003F02003002B01D001235A
:104248003B637B6AD3F8063023F020027B6AC3F80D
:10425800062005E007F10C03184601F0C7FB4AE108
:10426800FB6ADB6A03F00103002B11D07B6AD3F8E9
:10427800063003F00103002B01D101233B637B6A65
:10428800D3F8063043F001027B6AC3F8062027E022
:104298007B6AD3F8063003F00103002B01D0012319
:1042A8003B637B6AD3F8063023F001027B6AC3F8CC
:1042B8000620FB6ADB6A03F00203002B10D17B6A3D
:1042C800D3F8063003F00203002B09D07B6AD3F839
:1042D800063023F002027B6AC3F8062001233B6301
:1042E800FB6ADB6A03F01003002B11D07B6AD3F85A
:1042F800063003F40073002B01D101233B637B6A72
:10430800D3F8063043F400727B6AC3F8062010E045
:104318007B6AD3F8063003F40073002B01D0012325
:104328003B637B6AD3F8063023F400727B6AC3F8D8
:104338000620FB6ADB6A03F00203002B57D07B6A76
:10434800D3F8063003F00203002B01D101233B63AD
:104358007B6AD3F8063043F002027B6AC3F8062072
:10436800FB6ADB6A03F00403002B2ED07B6AD3F8C8
:10437800063003F00403002B01D101233B637B6A61
:10438800D3F8063043F004027B6AC3F80620FB6AC0
:10439800DB6A03F00803002B3AD17B6AD3F80A30B2
:1043A80003F00203002B33D17B6AD3F80A3043F0C1
:1043B80001027B6AC3F80A207B6AD3F80A3043F00B
:1043C80001027B6AC3F80A2022E07B6AD3F8063030
:1043D80003F00403002B01D001233B637B6AD3F86D
:1043E800063023F004027B6AC3F8062010E07B6ADB
:1043F800D3F8063003F00403002B01D001233B63FC
:104408007B6AD3F8063023F004027B6AC3F80620DF
:10441800FB6ADB6A03F00803002B12D07B6AD3F82F
:10442800063003F00803002B02D14FF0FF333B6343
:104438007B6AD3F8063043F008027B6AC3F806208B
:1044480011E07B6AD3F8063003F00803002B02D092
:104458004FF0FF333B637B6AD3F8063023F0080242
:104468007B6AC3F80620FB6A1B6CDAB27B6A5A7156
:10447800FB6ADB6A03F04003002B28D07B6A3D33DC
:10448800FB637B6A00229A730023BB631CE0FB6B0F
:104498001B68002B03D1FB6B5B68002B0ED001223D
:1044A800BB6B02FA03F33B627B6A9B7B5AB23B6AA3
:1044B8005BB213435BB2DAB27B6A9A73FB6B21334C
:1044C800FB63BB6B0133BB63BB6B072BDFDD07F102
:1044D8000C03184601F08AFA3B6B002B0BD0FB6AE1
:1044E800DB69184601F041FA05E003237B63FB6AA8
:1044F8007A6BC3F8CA207B6B18464037BD4680BD2F
:1045080080B586B000AF78607B687B6107F10C03EB
:104518001946072001F0CAFBFB6803F00103002BD2
:104528000DD07B69002283F8CA20002283F8CB20B3
:10453800002283F8CC20002283F8CD200EE07B698E
:10454800002242F0010283F8CA20002283F8CB201F
:10455800002283F8CC20002283F8CD2000231846BF
:104568001837BD4680BD80B58AB000AF78607B68DB
:104578003B6200237B623B6ADB690133BB61BB6939
:1045880003F596733B6107F10C03184601F01AFA1C
:104598000346002B29D1FB69D3F80A3003F0020344
:1045A800002B0FD13B6A002242F0010283F8CA2097
:1045B800002283F8CB20002283F8CC20002283F845
:1045C800CD200CE03B6A002283F8CA20002283F841
:1045D800CB20002283F8CC20002283F8CD2007F1DD
:1045E8000C03184601F002FA01E003237B627B6AA0
:1045F80018462837BD4680BD80B586B000AF7860C4
:104608007B687B6107F10C031946072001F04EFB1C
:10461800FB6803F00203002B0DD07B69002283F8AE
:10462800CA20002283F8CB20002283F8CC20002265
:1046380083F8CD200EE07B69002242F0010283F866
:10464800CA20002283F8CB20002283F8CC20002245
:1046580083F8CD20002318461837BD4680BD80B5A5
:104668008AB000AF78607B683B6200237B623B6A5C
:10467800DB690133BB61BB6903F5C8733B6107F1B3
:104688000C03184601F09EF90346002B55D1FB692F
:10469800D3F80A3003F40063002B24D0FB69D3F865
:1046A800063003F00103002B0FD03B6A002242F0D2
:1046B800010283F8CA20002283F8CB20002283F865
:1046C800CC20002283F8CD2031E03B6A002283F819
:1046D800CA20002283F8CB20002283F8CC200022B5
:1046E80083F8CD2023E0FB69D3F80A3003F00803F0
:1046F800002B0FD13B6A002242F0010283F8CA2046
:10470800002283F8CB20002283F8CC20002283F8F3
:10471800CD200CE03B6A002283F8CA20002283F8EF
:10472800CB20002283F8CC20002283F8CD2007F18B
:104738000C03184601F05AF901E003237B627B6AF7
:1047480018462837BD4680BD80B58AB000AF78606E
:104758007B683B6200237B623B6ADB690133BB6198
:10476800BB6903F5FA733B6107F10C03184601F0C6
:1047780029F90346002B26D1FB69DB7B002B0FD1DF
:104788003B6A002242F0010283F8CA20002283F823
:10479800CB20002283F8CC20002283F8CD200CE027
:1047A8003B6A002283F8CA20002283F8CB2000222B
:1047B80083F8CC20002283F8CD2007F10C0318469B
:1047C80001F014F901E003237B627B6A184628375D
:1047D800BD4680BD80B58AB000AF78607B683B621B
:1047E80000237B623B6ADB690133BB61BB6903F56C
:1047F80016733B6107F10C03184601F0E3F8034612
:10480800002B64D1FB69D3F8063003F48063002BD6
:104818004CD0FB69D3F8063003F00203002B47D1D4
:10482800FB69D3F80A3003F00103002B42D0FB697F
:104838009B7B002B40D1FB69D3F80A3003F080033F
:10484800002B3BD1FB69DB7B002B37D1FB69D3F80D
:104858000A3003F03003002B15D0FB69D3F80A3077
:1048680003F00403002B07D0FB69D3F8063003F0EC
:104878002003002B07D124E0FB69D3F8063003F0AE
:104888002003002B1CD13B6A002283F8CA20002297
:1048980083F8CB20002283F8CC20002283F8CD2097
:1048A80007F10C03184601F0A1F821E000BF08E069
:1048B80000BF06E000BF04E000BF02E000BF00E068
:1048C80000BF07F10C03184601F090F801E003233C
:1048D8007B623B6A002242F0010283F8CA20002270
:1048E80083F8CB20002283F8CC20002283F8CD2047
:1048F8007B6A18462837BD4680BD80B58AB000AFB0
:1049080078607B683B6200237B623B6A002242F04E
:10491800010283F8CA20002283F8CB20002283F802
:10492800CC20002283F8CD203B6ADB690133BB61D0
:10493800BB6903F52F733B6107F10C03184601F0BF
:1049480041F80346002B5CD1FB69D3F80A3003F029
:104958004003002B35D0FB69D3F8063003F480639D
:10496800002B30D0FB69D3F80A3003F00103002B89
:104978002BD0FB69D3F80A3003F08003002B26D133
:10498800FB69D3F8063003F00103002B21D0FB6943
:10499800D3F8063003F00203002B1CD03B6A002238
:1049A80083F8CA20002283F8CB20002283F8CC2089
:1049B800002283F8CD2007F10C03184601F016F801
:1049C80021E000BF08E000BF06E000BF04E000BF30
:1049D80002E000BF00E000BF3B6A002242F0010293
:1049E80083F8CA20002283F8CB20002283F8CC2049
:1049F800002283F8CD2007F10C03184600F0F6FFDB
:104A080001E001237B627B6A18462837BD4680BDDA
:104A180080B58AB000AF78607B683B6200237B6218
:104A28003B6A002242F0010283F8CA20002283F880
:104A3800CB20002283F8CC20002283F8CD203B6ACB
:104A4800DB6901337B617B6903F54873FB6007F120
:104A58000803184600F0B6FF0346002B1FD14E236B
:104A6800FB61BB69D3F80620FB691340002B10D10A
:104A7800BB699B7B002B0CD03B6A002283F8CA20C1
:104A8800002283F8CB20002283F8CC20002283F870
:104A9800CD2007F10803184600F0A8FF01E0032322
:104AA8007B627B6A18462837BD4680BD80B582B0D8
:104AB80000AF3B461946072001F0F8F83B6823F0A1
:104AC80001033B603B6843F004033B603B461946E7
:104AD800062001F0EBF8002318460837BD4680BDD4
:104AE80080B58AB000AF78607B68FB6100233B62C9
:104AF800FB69DB6901337B617B6903F56173FB60EB
:104B080007F10803184600F05DFF0346002B22D189
:104B1800BB69D3F8063003F48063002B0BD13DF05A
:104B28008FFCBB69D3F80620BB6942F48062C3F8E6
:104B3800062001233B6207F10803184600F056FFE0
:104B48003B6A002B04D0FB69DB69184600F00DFFB7
:104B580000237B6201E003237B627B6A18462837C7
:104B6800BD4680BD80B58AB000AF78607B683B6287
:104B78003B6ADB690133BB61BB6903F57A733B614F
:104B880007F10C03184600F01DFF0346002B14D153
:104B9800FB69D3F80620FB6942F00202C3F806203D
:104BA80000237B6207F10C03184600F01FFF3B6AE5
:104BB800DB69184600F0D9FE01E003237B627B6ABB
:104BC80018462837BD4680BD80B58AB000AF7860EA
:104BD8007B683B623B6ADB690133BB61BB6903F2FB
:104BE8004C433B6107F10C03184600F0EBFE03460B
:104BF800002B1CD100237B62FB69D3F80A20FB69D8
:104C080022F00302C3F80A20FB69D3F80620FB69E7
:104C180042F00802C3F8062007F10C03184600F01A
:104C2800E5FE3B6ADB69184600F09FFE01E00323BE
:104C38007B627B6A18462837BD4680BD80B58AB03E
:104C480000AF78607B683B623B6ADB690133BB611C
:104C5800BB6903F596633B6107F10C03184600F046
:104C6800B1FE0346002B16D13DF0EAFBFB69D3F8F1
:104C78000620FB6922F48062C3F8062000237B62C9
:104C880007F10C03184600F0B1FE3B6ADB691846D1
:104C980000F06BFE01E003237B627B6A184628372D
:104CA800BD4680BD80B588B000AF78607B68FB6189
:104CB800FB69DB6901337B6107F10803184600F0E3
:104CC80081FE0346002B30D1BB69D3F80A30BA699C
:104CD80023F4006323F00A03C2F80A30BB69D3F84F
:104CE800063003F00203002B0DD0BB69D3F80A206D
:104CF800BB6942F00102C3F80A2007F1080318460D
:104D080000F074FE0CE0BB69D3F80A20BB6922F0FE
:104D18003002C3F80A2007F10803184600F066FEBF
:104D2800FB69DB69184600F020FE0023184620378F
:104D3800BD4680BDB0B588B000AF78607B68FB61C8
:104D4800FB69DB6901337B617B6903F21453FB6008
:104D580007F10803184600F035FE0346002B78D10A
:104D6800FB691B6C002B6ADDFB691B6C082B66DC7E
:104D7800FB69D3F8A240D3F8A650B969FB691B6C4C
:104D88005A1E13465B0113440B443833D3F80530DD
:104D98001846FBF7D9FC02460B4620462946FBF786
:104DA800A5FF0346002B4AD0FB69D3F89A40D3F8F5
:104DB8009E50B969FB691B6C5A1E13465B0113446C
:104DC8000B443833D3F809301846FBF7BDFC0246CC
:104DD8000B4620462946FBF789FF0346002B2ED0B9
:104DE800FB69D3F8AA10B869FB691B6C5A1E1346F5
:104DF8005B011344034445331B7899421FD1BB69B7
:104E08009B7B5AB2FB691B6C013B012101FA03F33E
:104E18005BB2DB435BB213405AB2BB69D2B29A733E
:104E2800BB69DB7B5AB2FB691B6C013B012101FAB0
:104E380003F35BB213435AB2BB69D2B2DA7307F118
:104E48000803184600F0D2FDFB69DB69184600F03C
:104E58008CFD002318462037BD46B0BD80B58AB00A
:104E680000AF78607B683B623B6ADB690133BB61FA
:104E7800BB6903F596633B6107F10C03184600F024
:104E8800A1FD0346002B16D13DF0DAFAFB69D3F8F1
:104E98000A20FB6922F04002C3F80A2000237B6243
:104EA80007F10C03184600F0A1FD3B6ADB691846C0
:104EB80000F05BFD01E003237B627B6A184628371C
:104EC800BD4680BD2DE9B04F9CB000AFF863FB6BC9
:104ED8003B660023BB663B6EDB6901333B653B6D7C
:104EE80003F5AF63BB6407F14403184600F06AFD9D
:104EF8000346002B40F0E2810023FB667B6DD3F86C
:104F08000A3003F00403002B03D0FB6E43F00103C7
:104F1800FB667B6DD3F80A3003F03003002B10D00A
:104F28007B6DD3F80A3003F01003002B04D0FB6E1E
:104F380043F00803FB6608E0FB6E43F00403FB66DE
:104F480003E0FB6E43F00203FB667B6DD3F80A3087
:104F580003F48063002B03D0FB6E43F01003FB6661
:104F68003A6EFB6EC2F8AE303A6E002343F0070388
:104F780082F8C630002382F8C730002382F8C83090
:104F8800002382F8C9307B6D5B7D1A463B6EC3F8FF
:104F9800C2207B6D9B7D1A463B6EC3F8B2207B6DA9
:104FA800DB7D1A463B6EC3F8B6207B6D5B79002B20
:104FB80003D07B6D5B79082B02D97A6D012353717D
:104FC8007B6DD3F8063003F02003002B0CD0796DED
:104FD8007B6D5B795A1E13465B0113440B443833CF
:104FE800D3F809307B660BE0796D7B6D5B795A1ECF
:104FF80013465B0113440B443833D3F805307B6602
:10500800FB6E03F00803002B00F0B5807B6D9B69F5
:10501800002B02DD7B6E002B1CD13B6E002283F837
:10502800BA20002283F8BB20002283F8BC2000228B
:1050380083F8BD203B6E002283F8BE20002283F84F
:10504800BF20002283F8C020002283F8C120022359
:10505800BB662DE17B6D9B691A463B6EC3F8BA208F
:105068003B6ED3F8BA3000229A46934652465B46C6
:105078004FF000004FF00001990041EA9271900052
:1050880002460B4612EB0A0443EB0B054FF00002F5
:105098004FF00003EB0043EA5473E20014461D4648
:1050A800B4EB0A0865EB0B094FF000024FF0000360
:1050B8004FEA091343EA18734FEA081290469946D3
:1050C80018EB0A03BB6049EB0B03FB604FF00002CF
:1050D8004FF00003D7E9024529460B01204629462F
:1050E800044643EA147301460A01796E4908002010
:1050F800B962F862D7E90A4521465118396029464C
:1051080043EB01017960D7E90034C7E916347B6EB7
:1051180000223B627A62D7E90823D7E91601FCF737
:1051280049F802460B46C7E91623D7E91623012B8F
:105138001CD33B6E002283F8BA20002283F8BB20E0
:10514800002283F8BC20002283F8BD203B6E002299
:1051580083F8BE20002283F8BF20002283F8C020F5
:10516800002283F8C1200223BB66A1E0BA6D3B6E22
:10517800C3F8BE209CE0FB6E03F00403002B7DD037
:105188007B6DDB69002B02DD7B6E002B1CD13B6E37
:10519800002283F8BA20002283F8BB20002283F87B
:1051A800BC20002283F8BD203B6E002283F8BE207D
:1051B800002283F8BF20002283F8C020002283F851
:1051C800C1200223BB6673E07B6DDB691A463B6E28
:1051D800C3F8BE203B6ED3F8BE300022BB61FA6133
:1051E8007B6E00223B617A61D7E906342246D7E913
:1051F8000489414601FB02F24D4618462146034602
:1052080003FB05F3134402464146A2FB01217963DF
:105218003A637A6B13447B6342F210724FF00003D7
:10522800D7E90C01FBF7C6FF02460B46C7E9162370
:10523800D7E91623012B1CD33B6E002283F8BA2032
:10524800002283F8BB20002283F8BC20002283F8C8
:10525800BD203B6E002283F8BE20002283F8BF20C9
:10526800002283F8C020002283F8C1200223BB66F5
:105278001EE0BA6D3B6EC3F8BA2019E03B6E0022FF
:1052880083F8BA20002283F8BB20002283F8BC20D0
:10529800002283F8BD203B6E002283F8BE20002246
:1052A80083F8BF20002283F8C020002283F8C120A1
:1052B80007F14403184600F099FB01E00323BB669D
:1052C800BB6E18467037BD46BDE8B08F80B58AB052
:1052D80000AF78607B683B623B6AA03302330022F0
:1052E8001A7000225A7000229A700022DA70002286
:1052F8001A7100225A7100229A710022DA713B6AEF
:10530800A033063B00221A7000225A7000229A70BD
:105318000022DA7000221A7100225A7100229A7152
:105328000022DA7100237B623B6ADB6901337B610F
:105338007B6903F2DC53FB6007F10803184600F0B1
:1053480041FB0346002B40F09680BB699B7B1846C7
:1053580000F014FBF861FB695A1C3B6A1A64FB698C
:10536800002B02DBFB69072B33DD3B6AA0330233DA
:1053780000221A7000225A7000229A700022DA70F5
:1053880000221A7100225A7100229A710022DA71E1
:105398003B6AA033063B00221A7000225A70002292
:1053A8009A700022DA7000221A7100225A710022C3
:1053B8009A710022DA713B6A002283F8AA2000223F
:1053C80083F8AB20002283F8AC20002283F8AD20BC
:1053D8004BE0B969FA6913465B0113440B4438334F
:1053E800D3F805301846FBF79FF902460B46396A91
:1053F800A03102310A604B60B969FA6913465B0152
:1054080013440B443833D3F809301846FBF78CF9AA
:1054180002460B46396AA03106390A604B60B96901
:10542800FA6913465B0113440B4445331B78C82BB8
:105438000FD13B6A002262F0370283F8AA200022CB
:1054480083F8AB20002283F8AC20002283F8AD203B
:105458000BE0B969FA6913465B0113440B44453301
:105468001B781A463B6AC3F8AA2007F108031846B6
:1054780000F0BCFA01E003237B627B6A18462837F8
:10548800BD4680BD80B58AB000AF78607B683B625E
:105498003B6ADB690133BB61BB6903F5C8633B61E8
:1054A80007F10C03184600F08DFA0346002B10D1C3
:1054B800FB69DB7B184600F061FA03465A1C3B6A1D
:1054C8001A6400237B6207F10C03184600F08EFA79
:1054D80001E003237B627B6A18462837BD4680BDFE
:1054E80090B58BB000AF78607B687B627B6ADB69C4
:1054F80001333B623B6A7B617B6903F2A463FB6017
:1055080007F10803184600F05DFA0346002B40F047
:10551800D6807B6A1B6C08211846FEF794FB03466D
:10552800002B06D107F10803184600F05FFA0223A2
:10553800C6E0BB69D3F80A3003F08003002B19D00A
:105548003CF07EFFBB69D3F80620BB6922F0170246
:10555800C3F80620BB69D3F80A20BB6922F0C10250
:10556800C3F80A20BB69D3F80620BB6942F04002A1
:10557800C3F80620B9697B6A1B6C5A1E13465B0187
:10558800134438330B440533FB61796AD1F8722030
:10559800D1F87630104619464BF0C4FE02460B4649
:1055A800F969103107390A604B60796AD1F87A20B5
:1055B800D1F87E30104619464BF0B4FE02460B4631
:1055C800F969203107390A604B60796AD1F882207D
:1055D800D1F88630104619464BF0A4FE02460B4619
:1055E800F969103101310A604B607B6AD3F86E307B
:1055F80003F08103002B03D0BB6930221A740DE03D
:105608007B6AD3F86E3003F00403002B03D0BB6928
:1056180032221A7402E0BB6933221A74796AD1F80B
:105628008A20D1F88E3010461946FBF7C1F8024699
:105638000B46BC69104619464BF074FE02460B46F1
:1056480004F1300103390A604B60796AD1F892207D
:10565800D1F8963010461946FBF7AAF802460B46D1
:10566800BC69104619464BF05DFE02460B4604F134
:1056780040010B390A604B607B6A1B6C002B14DD00
:105688007B6A1B6C082B10DCBB69DB7B5AB27B6A1C
:105698001B6C013B012101FA03F35BB2DB435BB2F4
:1056A80013405AB2BB69D2B2DA7307F1080318463D
:1056B80000F09CF97B6ADB69184600F056F9002374
:1056C80018462C37BD4690BD90B58DB000AF7860B8
:1056D8007B68BB62BB6ADB6901337B627B6ABB6147
:1056E800BB6903F5E1633B6107F10C03184600F061
:1056F80069F90346002B40F0E8800023FB62BB6A8F
:105708001B6C002B03DDBB6A1B6C082B04DDFB69DB
:10571800012283F82C2005E0BB6A1A6CFB69D2B21F
:1057280083F82C20F969FB6993F82C305A1E13462C
:105738005B01134438330B4405333B62BB6A1B6A75
:1057480003F00103002B1ED0FB69D3F80620FB6988
:1057580042F02002C3F80620FB69D3F80A20FB694F
:1057680042F00402C3F80A20FB693A6A52689A6256
:10577800B96ACA6C0B6DFC6910461946FBF726FB23
:10578800034623621DE0FB69D3F80620FB6922F07B
:105798002002C3F80620FB69D3F80A20FB6922F02F
:1057A8000402C3F80A20FB693A6A12689A62B96A65
:1057B8004A6D8B6DFC6910461946FBF707FB0346DB
:1057C8002362B96ACA6D0B6EFC6910461946FBF76D
:1057D800FDFA03466362BB6A1B6A03F04003002BB1
:1057E8004FD00123FB62BB6AD86C196D4FF00002E1
:1057F8004FF00003FBF77AFA0346002B14D0BB6A7C
:10580800D86D196E4FF000024FF00003FBF76EFAE7
:105818000346002B08D0FB69D3F80620FB6922F069
:105828001502C3F8062043E0BB6A1B6C002B0ED19F
:10583800BB6A002242F0010283F84020002283F86C
:105848004120002283F84220002283F843203CF0C4
:10585800F7FDFB69DB7B5AB2BB6A1B6C013B01217C
:1058680001FA03F35BB213435AB2FB69D2B2DA739B
:10587800FB69D3F80A20FB6942F08002C3F80A20CA
:1058880016E0BB6A1B6A03F02003002B08D0FB69F3
:10589800D3F80620FB6942F01002C3F8062007E09F
:1058A800FB69D3F80620FB6922F01002C3F8062032
:1058B80007F10C03184600F099F8FB6A002B04D096
:1058C800BB6ADB69184600F050F8002318463437E5
:1058D800BD4690BD80B58AB000AF78607B687B62BA
:1058E8007B6A9B683B623B6ABB61BB6903F5E1630A
:1058F8003B6107F10C03184600F064F80346002BDF
:105908002DD17B6ADB68B3F5FC7F1DD1FB69D3F829
:10591800063003F08003002B1AD13CF091FDFB699F
:10592800D3F80620FB6942F08002C3F80620FB6921
:10593800D3F80620FB6922F48062C3F80620796850
:10594800C92005F0D9FC03E07968C92005F0D4FC2A
:1059580007F10C03184600F049F8002301E04FF462
:105968007A7318462837BD4680BD80B483B000AF2F
:10597800786000BF0C37BD4680BC704780B485B0E6
:1059880000AF78600023FB600023BB6010E00122B9
:10599800BB6802FA03F31A467B681340002B01D058
:1059A800FB6809E0FB680133FB60BB680133BB603F
:1059B800BB68072BEBDD002318461437BD4680BCB7
:1059C8007047000080B584B000AF78607B68FB60EA
:1059D800FB68054A1A607968282000F067F90346D1
:1059E80018461037BD4680BD802A050880B582B0AC
:1059F80000AF786079682B2000F058F900BF0837AD
:105A0800BD4680BD80B483B000AF78607B68002B52
:105A180002D07B68034A1A6000BF0C37BD4680BCC1
:105A2800704700BF802A050880B483B000AF786053
:105A380000BF0C37BD4680BC704780B483B000AF50
:105A4800786000BF0C37BD4680BC704780B584B015
:105A580000AFF860B9607A603B60234B1B78002B7D
:105A680004D000F0A1F8204B00221A70FB68012B2B
:105A780006D13A687968B86806F09CFA03462FE0C0
:105A8800FB68022B09D1BB689BB27A6891B23A686D
:105A9800184605F00FFF034622E0FB68642B09D186
:105AA800BB689BB27A6891B23A68184606F066F805
:105AB800034615E0FB68082B06D13A687968B86890
:105AC80005F04EF903460BE0FB68652B07D17B68B0
:105AD8009BB23968184607F0BFFE034600E0012371
:105AE80018461037BD4680BDA0ED002080B5A6B091
:105AF80000AF652387F8683007F164031A46002170
:105B0800002006F057FAD7F86930184639F046FFF2
:105B18003B460A49184642F0DBFD00237B663B46BC
:105B2800C7F8813039F030FF07F164031A460121C4
:105B380006F040FA00BF9837BD4680BD942A050894
:105B480080B500AF174B00221A703CF0DBFD03F064
:105B58004DFC00214FF47B7007F07EFE00224FF4CD
:105B68007B71002006F00AF800224FF47B710020B8
:105B780006F020FA00224FF47B71002005F09AFE0F
:105B8800FFF7B4FF00220021002005F0E9F804F037
:105B980081FD08F069F900F059F803F0EBFD00BF4A
:105BA80080BD00BFA0ED002080B500AF3CF024FD13
:105BB80000BF80BD80B483B000AF03463A60FB806D
:105BC8000B46BB80032318460C37BD4680BC704784
:105BD80080B500AF08F066F90A4B1B8801339AB20A
:105BE800084B1A80074B1B88B3F57A7F07D1064B01
:105BF8001B680133044A1360024B00221A8000BF5D
:105C080080BD00BF6C16002070160020B0B485B0AF
:105C180000AFF860B9607A600A4B1B6800221C4626
:105C28001546BB68C3E90045064B1B68064A02FBDC
:105C380003F31A46BB689A60002318461437BD461A
:105C4800B0BC70477016002040420F0080B582B08B
:105C580000AF00237B600FE03CF050F8014610488D
:105C68007A6813469B0013449A011344034418337B
:105C780019607B6801337B607B681F2BECDD094B67
:105C880000221A6000F0AAFA074B00221A60044B9F
:105C980010221A60002318460837BD4680BD00BF91
:105CA8007816002074160020303F002080B584B09C
:105CB80000AF786039607B6840F2EB32934200F0C5
:105CC80028817B68B3F57B7F80F228817B6840F26E
:105CD800EA32934200F018817B6840F2EA3293423C
:105CE80000F31C817B6840F2E932934200F007819F
:105CF8007B6840F2E932934200F310817B685B2BAA
:105D080000F3BC807B68042BC0F208817B68043BED
:105D1800572B00F2038101A252F823F0BD5E000860
:105D2800C75E0008A95E0008B35E0008955E00081B
:105D38009F5E0008255F0008255F0008255F0008B2
:105D4800255F0008255F0008255F0008255F00081B
:105D5800255F0008255F0008255F0008255F00080B
:105D6800255F0008255F0008255F0008255F0008FB
:105D7800255F0008255F0008255F0008255F0008EB
:105D8800255F0008255F0008255F0008255F0008DB
:105D9800255F0008255F0008255F0008255F0008CB
:105DA800255F0008255F0008255F0008DB5E000806
:105DB800255F0008255F0008D15E0008255F000800
:105DC800255F0008255F0008255F0008ED5E0008D4
:105DD800E55E0008255F0008255F0008255F0008CC
:105DE800255F0008255F0008255F0008255F00087B
:105DF800255F0008255F0008255F0008255F00086B
:105E0800255F0008255F0008255F0008255F00085A
:105E1800255F0008255F0008255F0008255F00084A
:105E2800255F0008255F0008255F0008255F00083A
:105E3800255F0008255F0008255F0008255F00082A
:105E4800255F0008255F0008255F0008255F00081A
:105E5800255F0008255F0008255F0008255F00080A
:105E6800255F0008255F0008255F0008255F0008FA
:105E7800255F0008F75E0008FF5E00087B68C82BF6
:105E88004CD1386800F060F8F8604EE0386800F0EF
:105E9800B9F8F86049E0386800F0D4F8F86044E0F0
:105EA800386800F08BF8F8603FE0386800F098F840
:105EB800F8603AE0386800F05DF8F86035E0386876
:105EC80000F06AF8F86030E0386800F0DBF8F86055
:105ED8002BE0386800F04AF9F86026E000F07EF917
:105EE800F86022E0386800F091F9F8601DE000F0F1
:105EF800CFFAF86019E000F0D2FAF86015E03868D7
:105F080000F0D4FA002319E0386800F015FB0023EC
:105F180014E0386800F0DCFA00230FE0094B1B6836
:105F28000133084A1360012308E0FB68002B04D002
:105F3800044B1B680133034A1360FB68184610378B
:105F4800BD4680BD343F002080B485B000AF786086
:105F58007B68FB60FB68054A1A60054AFB685A6063
:105F6800002318461437BD4680BC704778160020B9
:105F7800385C012080B485B000AF78607B68FB6036
:105F8800FB681B68034A5360002318461437BD4654
:105F980080BC70477816002080B485B000AF786068
:105FA8007B68FB60044B5A68FB681A60002318463C
:105FB8001437BD4680BC70477816002080B485B081
:105FC80000AF78607B68FB60FB681B68034A13605E
:105FD800002318461437BD4680BC70477816002049
:105FE80080B485B000AF78607B68FB60044B1A68AA
:105FF800FB681A60002318461437BD4680BC7047FA
:106008007816002080B485B000AF78607B68FB60AC
:10601800FB681B68FA6852680949013341F8332064
:10602800FB681B68FA68926805490133DB000B447A
:106038005A60002318461437BD4680BC704700BF1D
:106048007816002080B485B000AF78607B68FB606C
:10605800FB681B680A4A013352F83320FB685A6010
:10606800FB681B68064A0133DB0013445A68FB6867
:106078009A60002318461437BD4680BC704700BF9D
:106088007816002080B584B000AF78607B68FB602C
:10609800FB681B691B68002B01D106230CE0FB6819
:1060A8001B691B68012118463BF0A2FE0346002B22
:1060B80001D1002300E0062318461037BD4680BDF5
:1060C80080B586B000AF786000237B6126497A6886
:1060D80013469B0013449A0113440B4418331B685E
:1060E800BB60BB68002B05D13CF0AAF94FF0FF3329
:1060F8007B6133E000233B610523FB6012E0012153
:10610800B8683BF0C7FE0346002B0CBF01230023F1
:10611800DBB23B613B69002B04D105203BF0ECFE70
:106128003CF08EF93B69002B04D1FB685A1EFA60DB
:10613800002BE4DC3B69002B10D13CF081F90121F4
:10614800B8683BF00FFE0346002B02D13CF078F90B
:1061580004E03CF075F94FF0FF337B617B6918462A
:106168001837BD4680BD00BF7816002080B586B0C0
:1061780000AF78607B687B617B69DB683B613B696A
:10618800002B02DD3B69202B0ADD7B6900221A7493
:1061980000225A7400229A740022DA74022316E04C
:1061A8003B69013BFB60F868FFF78AFF0346002B59
:1061B8000CD1FA6813469B0013449A011344183310
:1061C800054A1A447B691A61002300E00423184633
:1061D8001837BD4680BD00BF7816002080B586B050
:1061E80000AF00237B6109E07B690133FB603B461C
:1061F800184600F00BF87B6901337B617B691F2B24
:10620800F2DD002318461837BD4680BD80B487B03C
:1062180000AF78607B683B613B69DB685A1E1346B8
:106228009B0013449A0113441833984A1344FB60A3
:106238003B69DB68DBB2013BDAB2FB681A71FB68C9
:1062480000225A71FB6800229A710022DA7100223A
:106258001A7200225A72FB68002242F004029A72F3
:106268000022DA7200221A7300225A73FB68002295
:106278009A73FB680022DA73FB6800221A74FB68C1
:1062880000225A7400229A740022DA7400221A75C5
:10629800FB680F225A75FB6800229A75FB6800227A
:1062A8001A7600225A7600229A760022DA76FB685D
:1062B80000221A7700225A7700229A770022DA778A
:1062C800FB68002283F82020002283F82120002286
:1062D80083F82220002283F82320FB68002283F819
:1062E8002420002283F82520002283F8262000227B
:1062F80083F82720FB68002283F82820002283F8EF
:106308002920002283F82A20002283F82B20FB680A
:10631800002283F82C20FB6840330B3B00221A70C4
:1063280000225A7000229A700022DA7000221A7134
:1063380000225A7100229A710022DA71FB68303308
:10634800033B00221A7000225A7000229A70002221
:10635800DA7000221A7100225A7100229A71002202
:10636800DA7100237B6174E0F9687A6913465B018E
:1063780013440B44383300225A7100229A710022C8
:10638800DA7100221A72F9687A6913465B011344BC
:106398000B44383300225A7200229A720022DA72B1
:1063A80000221A73F9687A6913465B0113440B4497
:1063B800453300221A70F9687A6913465B01134461
:1063C8000B44403310330A3B00221A7000225A70E3
:1063D80000229A700022DA7000221A7100225A7183
:1063E80000229A710022DA71F9687A6913465B0112
:1063F80013440B44483310330A3B00221A7000221E
:106408005A7000229A700022DA7000221A71002253
:106418005A7100229A710022DA71F9687A69134672
:106428005B0113440B44503310330A3B00221A70AB
:1064380000225A7000229A700022DA7000221A7123
:1064480000225A7100229A710022DA717B690133A5
:106458007B617B69072B87DDFB68D3F8063003F483
:106468008072FB68C3F80620FB6800229A7200223B
:1064780042F01002DA7200221A7300225A730023C3
:1064880018461C37BD4680BC704700BF78160020F0
:1064980080B400AF00231846BD4680BC704780B466
:1064A80000AF00231846BD4680BC704780B483B057
:1064B80000AF78607B68002B02D07B68034A1A60C3
:1064C80000BF0C37BD4680BC704700BFA42A050832
:1064D80080B483B000AF786000BF0C37BD4680BC85
:1064E8007047000080B582B000AF002039F05EFE32
:1064F80078600D49786839F001FF78600B49786851
:1065080039F037FE78600A49786839F032FE7860E9
:10651800502303220749786839F058FE78607B6871
:1065280018460837BD4680BDB42A0508BC2A0508A8
:10653800E02A05080C2B050880B582B000AF78600A
:10654800FFF7D0FF0346184639F07AFD03461B2BA8
:1065580005D0502B02D100F007F800BFF0E700BFCC
:106568000837BD4680BD00002DE9F04FADB004AF3F
:106578000023C7F89C30D7F89C300133194670487F
:1065880039F06AFAD7F89C301A4692001A449301F7
:106598001A4418326B4B1344C7F88C30D7F88C3038
:1065A8005B79002B0AD0D7F88C305B79082B05D89B
:1065B800D7F88C305B79C7F8903002E00123C7F830
:1065C8009030D7F88C3093F82C30002B0CD0D7F8BB
:1065D8008C3093F82C30082B06D8D7F88C3093F8E9
:1065E8002C30C7F8943002E00123C7F89430D7F86C
:1065F8008C30D3F806301946534839F02DFAD7F8BD
:106608008C30D3F80A301946504839F025FAD7F8B3
:106618008C30D3F8113019464D4839F01DFAD7F8A7
:1066280090104C4839F018FAD7F894104A4839F0C5
:1066380013FAD7F88C309A6913469B0013445B0011
:10664800DA179A46934607F15802032301930A235F
:1066580000930F235046594607F000FD034619469C
:106668003E4839F0F9F9D7F88C30DB69DA173B6323
:106678007A6307F15802032301930A2300930F2337
:10668800D7E90C0107F0EAFC03461946344839F00B
:10669800E3F9D7F88C309B6A0022BB62FA6207F1F3
:1066A800580203230193062300930F23D7E90A0115
:1066B80007F0D4FC034619462A4839F0CDF9D7F833
:1066C8008C301B6A00223B627A6207F1580202236F
:1066D80001930A2300930F23D7E9080107F0BEFCB2
:1066E80003461946204839F0B7F9D7F88C305B6A69
:1066F8000022BB61FA6107F15802032301930A23C0
:1067080000930F23D7E9060107F0A8FC03461946B2
:10671800164839F0A1F9D7F88C309B7B19461448F4
:1067280039F09AF9D7F88C30DB7B1946114839F0E3
:1067380093F9114839F0CEF90023C7F89830B5E03D
:10674800242B050878160020382B0508542B05083B
:10675800702B0508882B0508A42B0508C02B0508F5
:10676800DC2B0508F82B0508142C0508302C050827
:106778004C2C0508682C0508842C0508D7F8983097
:1067880003F10109D7F88C10D7F8982013465B015C
:1067980013440B443833D3F8093000223B617A6143
:1067A80007F1680203230193062300930F23D7E917
:1067B800040107F053FC8046D7F88C10D7F89820CE
:1067C80013465B0113440B443833D3F805300022D9
:1067D800BB60FA6007F17802032301930623009354
:1067E8000F23D7E9020107F039FC0646D7F88C10C9
:1067F800D7F8982013465B0113440B4445331B78A4
:106808007B60D7F88C10D7F8982013465B011344A7
:106818000B444033D3F80600D3F80A1007F15802A6
:10682800032301930A2300930F2307F017FC05465F
:10683800D7F88C10D7F8982013465B0113440B4403
:106848005033D3F80600D3F80A1007F148020223A0
:1068580001930A2300930F2307F000FC0446D7F89E
:106868008C10D7F8982013465B0113440B44483327
:10687800D3F80600D3F80A1007F13802022301936F
:106888000A2300930F2307F0E9FB034603930294BE
:1068980001957B680093334642464946244839F0BF
:1068A800DBF8D7F898300133C7F89830D7F8983024
:1068B800072B7FF763AF1F4839F00CF9002039F038
:1068C80082F90346C7F88830D7F888302D2B19D0BD
:1068D800D7F888302D2B3FF74EAED7F888301B2BD2
:1068E80021D0D7F888302B2B1CD1D7F89C30013316
:1068F800C7F89C30D7F89C301F2B10DD0023C7F851
:106908009C300CE0D7F89C30013BC7F89C30D7F896
:106918009C30002B05DA1F23C7F89C3001E000BF2C
:1069280029E600BF27E600BFA437BD46BDE8F08FC3
:10693800C82C0508F02C050880B582B000AF0346C6
:106948003960FB80FB88B3F57B7F0BD0B3F57B7F89
:1069580010DC40F2E93293420BD040F2EA32934223
:1069680003D007E000F00AF804E0002002F01CFC65
:1069780000E000BF0837BD4680BD000080B592B07A
:1069880000AFC84B01221A70002387F8463077E021
:1069980097F94630C44A8C2101FB03F3134418339A
:1069A80000225A7000229A7097F94630BE4A8C210C
:1069B80001FB03F3134400221A7097F94630BA4AD0
:1069C8008C2101FB03F31344863300221A7097F9D4
:1069D8004630B54A8C2101FB03F313448733002268
:1069E8001A7097F94630B04A8C2101FB03F313441F
:1069F800853300221A7097F94630AB4A8C2101FB87
:106A080003F31344883300221A6097F94630A64AE4
:106A18008C2101FB03F3134418330022DA7100229E
:106A28001A7297F94630A04A8C2101FB03F31344EC
:106A380018330022DA7000221A7100225A710022DB
:106A48009A7197F94630984A8C2101FB03F3134455
:106A58001833B3F8073098B297F946308C2202FB06
:106A680003F31833904A134403331A46012105F0FF
:106A780085F897F94630DBB20133DBB287F8463048
:106A880097F94630012B83DD884B00221A70692361
:106A98003B713B461A460021002005F08BFA03465D
:106AA800002B1ED102E0FFF77FF8FCE7D7F805308E
:106AB8009AB27D4BA3F81920012002F0F3FA03469D
:106AC8001A467B49784841F003FE68233B713B46F0
:106AD8001A460021002005F06DFA0346002B02D06B
:106AE800E1E700BFDFE7D7F805309AB26E4BA3F8AD
:106AF800A520022002F0D6FA03461A466C496D48D2
:106B080041F0E6FD02F0C6F90323BB860123FB86AC
:106B1800694BBB6307F134031946012006F09CFE5C
:106B2800654B1B88022B02D9634B00221A80002375
:106B380087F847307EE1FFF737F897F94730DBB23F
:106B48000133DBB287F8473097F8473003F0010389
:106B580087F8473097F84720584B1A7097F947300D
:106B68008C2202FB03F3504A13443B643B6C93F8BA
:106B78008630062B00F24C8101A252F823F000BFA8
:106B8800A56B0008EB6B0008216D00087B6C000802
:106B9800A36D0008E96D0008C96C00083B6CB3F8E8
:106BA80019309BB207F13F021146184602F05EFA0F
:106BB8000346002B40F0318197F83F30022B40F01C
:106BC8002C8100BF00E000BF3B6C022283F88520C7
:106BD8003B6C002283F887203B6C012283F88620D7
:106BE8001BE13B6CB3F819309BB207F13F02114629
:106BF800184602F03BFA0346002B40F0108197F844
:106C08003F30022BDFD03B6C93F8852097F83F305C
:106C18001344DAB23B6C83F8852097F83F30032B96
:106C280004D13B6C022283F88620F8E03B6C93F891
:106C38008730622B18D83B6C93F887305A1CD1B236
:106C48003A6C82F88710194697F83F203B6C0B4442
:106C580083F821203B6C93F887301A463B6C134429
:106C6800002283F82120DAE03B6C032283F8862097
:106C7800D5E03B6CB3F819309BB207F13F021146DF
:106C8800184602F0F3F90346002B40F0CA8097F843
:106C98003F30032B40F0C5803B6C062283F88620EA
:106CA800BFE000BF383F00203C3F0020A2ED00209D
:106CB800F42C0508C83F0020A4ED002080430020E4
:106CC8003B6CB3F819309BB207F13F0211461846E6
:106CD80002F0CCF90346002B40F0A5803B6C002263
:106CE80083F887203B6C052283F886203B6C0022C2
:106CF80042F00A02DA7600221A7700225A77002236
:106D08009A773B6CB3F81F3098B23B6C1B331A462A
:106D1800032104F033FF86E03B6CB3F819309BB2D3
:106D280007F13F021146184602F0A0F90346002B6E
:106D38007BD13B6C002283F887203B6C93F885203D
:106D480097F83F301344DAB23B6C83F885203B6CEC
:106D580093F8853003F07F03002B04D13B6C0422A9
:106D680083F8862003E03B6C052283F886203B6C81
:106D7800002242F00A02DA7600221A7700225A77B5
:106D880000229A773B6CB3F81F3098B23B6C1B33E8
:106D98001A46032104F0F2FE47E03B6C1B33184609
:106DA80002F0B3F90346002B41D13B6C002283F873
:106DB8008620254B1B68254A13603B6CB3F81930B5
:106DC80098B23B6C21330022194600F0BFF81E4BE5
:106DD8001A681E4B1B68D21A3B6CC3F8882026E041
:106DE8003B6C1B33184602F090F90346002B20D168
:106DF8003B6C002283F88620154904203BF012FDE5
:106E08003B6CB3F819309BB2184602F09FF810E0BB
:106E18003B6C002283F886200CE000BF0AE000BF2C
:106E280008E000BF06E000BF04E000BF02E000BFCA
:106E380000E000BF074B1B78002B7FF47CAE064BAD
:106E480001221A7000BFFDE720EE00207C430020DD
:106E5800002D0508383F0020393F002080B584B058
:106E680000AF78600B467B80374B00221A800123E5
:106E7800FB817B681B78413B0A2B5FD801A252F843
:106E880023F000BFE56E0008F16E0008FD6E0008F3
:106E9800096F0008156F0008D96E0008C56E000854
:106EA800216F00082D6F0008396F0008B96E0008BF
:106EB800786800F04DFB0346FB813FE07B8818466D
:106EC80002F022F864203BF017F806F08BFF35E05B
:106ED800786800F0FBFB0346FB812FE0786800F040
:106EE80037FE0346FB8129E0786800F0B3FF0346CC
:106EF800FB8123E0786801F0B5FB0346FB811DE0C8
:106F0800786801F01FFC0346FB8117E0786801F000
:106F1800B7FC0346FB8111E0786801F03BFD0346AE
:106F2800FB810BE0786801F081FD0346FB8105E0F9
:106F3800786801F037FE0346FB8100BFFB891846DD
:106F48001037BD4680BD00BFE441002080B584B045
:106F580000AF03463960FB8013467B711F4B1B68EB
:106F6800002B04D13AF0CAFE03461C4A13601B4B9F
:106F78001B68002B08D0194B1B68012118463AF0F2
:106F8800F1FE0346002B05D0FB88184601F0DEFF12
:106F980003461FE0FB8819463868FFF75FFF034682
:106FA800FB81FB89002B02D07B79002B04D1FB8865
:106FB800184601F0EDFF06E0094B00221A80FB8815
:106FC800184601F0C3FF054B1B68012118463AF02B
:106FD8000FFFFB8918461037BD4680BDA04300202F
:106FE800E441002080B485B000AF78600B46FB70A8
:106FF8001346BB70FB78FB7310E0FB7B7A68134485
:107008001B782F2B05D9FB7B7A6813441B78392B07
:1070180001D900230AE0FB7B0133FB73FA78BB78C4
:107028001344DBB2FA7B9A42E7D30123184614379C
:10703800BD4680BC7047000080B584B000AF786062
:10704800786841F01FFEF8607B681B78413B0A2B8B
:1070580000F2E68001A252F823F000BF897100080F
:1070680055710008D1700008D1700008F17000084F
:107078009F700008C370000835710008157100087A
:10708800BD71000891700008FB68012B0CBF01233B
:107098000023DBB2C5E0FB68022B0BD17B68013310
:1070A8001B78312B04D07B6801331B78452B01D129
:1070B800012300E00023DBB2B3E0FB68012B0CBF27
:1070C80001230023DBB2ACE0FB68032B09D10222C9
:1070D80001217868FFF786FF0346002B01D00123C2
:1070E80000E00023DBB29CE0FB68022B0BD17B683D
:1070F80001331B7819464D4841F02AFC0346002B02
:1071080001D0012300E00023DBB28AE0FB68042BF6
:1071180009D1032201217868FFF764FF0346002B99
:1071280001D0012300E00023DBB27AE0FB68072BE3
:1071380009D1062201217868FFF754FF0346002B86
:1071480001D0012300E00023DBB26AE0FB68042BD6
:1071580013D1022201217868FFF744FF0346002B70
:107168000BD07B6803331B78522B04D07B68033326
:107178001B78432B01D1012300E00023DBB250E050
:10718800FB68112B13D1102201217868FFF72AFF21
:107198000346002B0BD07B6804331B781946244820
:1071A80041F0D6FB0346002B01D0012300E0002369
:1071B800DBB236E0FB68052B10D103220121786889
:1071C800FFF710FF0346002B08D07B6804331B78B9
:1071D800522B0CBF01230023DBB222E0FB68112BEA
:1071E8001BD1032201217868FFF7FCFE0346002B20
:1071F80013D07B6804331B7819460E4841F0A8FB6E
:107208000346002B09D00C2205217868FFF7EAFE17
:107218000346002B01D0012300E00023DBB200E08D
:10722800002318461037BD4680BD00BF142D050841
:107238001C2D0508242D050880B5A0B000AF034615
:107248003960FB80002387F87F30002387F87E3081
:10725800002387F87D30002387F872303AF088FEE3
:10726800B86700237B67002387F8733007F10C03A6
:1072780064220021184641F0FBFAAD4838F02AFC98
:10728800FEF792FC97F87F30052B11D13AF070FE8B
:1072980002467B6FD31A40F2ED22934208D90023AD
:1072A80087F87F30002387F87D30002387F8733014
:1072B8003AF05EFE0246BB6FD31A4EF65F22934247
:1072C80008D93B68002B01D002F056F9994838F0EC
:1072D80001FC29E107F17202FB881146184601F00A
:1072E800C5FE0346002B40F017813AF041FEB8670F
:1072F80097F87F30002B0CD197F872301B2B08D1F0
:107308003B68002B01D002F037F98B4838F0E2FBDC
:107318000AE197F87F30052B00F2EE8001A252F8BF
:1073280023F000BF45730008EB7300085974000888
:1073380001750008117500088F73000897F87230FE
:10734800022B0BD1022387F87E30002387F87D308B
:1073580000233B73012387F87F30DFE03B68002B75
:1073680000F0DC8097F872301D2B40F0D7800523A1
:1073780087F87F30002387F87D30012387F8733042
:10738800BB6F7B67CAE097F87D30102B07D897F85A
:107398007D306A4AD25C97F872309A4202D0002354
:1073A80087F8733097F87D30013387F87D3097F888
:1073B80072301E2B40F0B48097F87330002B06D043
:1073C80097F87D30112B02D15D4838F083FB0023FC
:1073D80087F87F30002387F87D30002387F87330E3
:1073E8009EE097F87230022B08D1022387F87E308E
:1073F800002387F87D3000233B7394E097F87220D0
:1074080097F87E30134487F87E3097F87230032B54
:1074180003D1022387F87F3085E097F87D30622B0F
:1074280012D897F87D305A1C87F87D2097F872207B
:1074380080333B4403F8742C97F87D3080333B4409
:10744800002203F8742C6EE0032387F87F306AE08B
:1074580097F8722097F87E30134487F87E3000231F
:1074680087F87F3097F87E3003F07F03002B04D035
:10747800FB88184601F06AFD55E007F10C03314915
:107488001846F8F7BBFE0346002B0CD1FB881846BC
:1074980001F03AFD3B68002B01D002F06DF8264858
:1074A80038F018FB40E03B68002B10D007F10C03C4
:1074B80025491846F8F7A2FE0346002B07D1FB889A
:1074C800184601F021FD214838F004FB2CE007F1B3
:1074D8000C031846FFF7B0FD0346002B04D1FB88C8
:1074E800184601F033FD1EE007F10C01FB8801226C
:1074F8001846FFF72BFD16E097F87230032B11D1D1
:10750800042387F87F300DE0FB88184601F01EFD44
:10751800002387F87F3006E000BFB1E600BFAFE682
:1075280000BFADE600BFABE68037BD4680BD00BFFB
:10753800282D0508382D05084C2D0508AC2D050803
:107548005C2D05088C2D0508942D05089C2D050833
:1075580080B59EB002AF78604E4BFB660023009367
:107568004D4B4E4A4E49F86E41F0B2F8F86E41F074
:1075780089FB03460133FA6E1344FB6607F10803DF
:107588001946002001F0CAFE07F108020023454908
:10759800F86E41F09DF8F86E41F074FB0346013334
:1075A800FA6E1344FB6600223F49F86E41F090F8EA
:1075B800F86E41F067FB03460133FA6E1344FB662D
:1075C80007F108031946012001F0A8FE07F1080297
:1075D80000233449F86E41F07BF8F86E41F052FB15
:1075E80003460133FA6E1344FB6600222E49F86EF7
:1075F80041F06EF8F86E41F045FB03460133FA6E30
:107608001344FB667B6801337B607B681B78452BE2
:1076180034D1264B1B88012B08D0022B0DD0002318
:10762800234A2049F86E41F053F80DE00023214A1F
:107638001C49F86E41F04CF806E000231E4A19492F
:10764800F86E41F045F800BFF86E41F01BFB0346A9
:107658000133FA6E1344FB66184B1A68184B1B6803
:10766800002100911749F86E41F032F8F86E41F0A8
:1076780009FB03460133FA6E1344FB66FB6E054AA9
:107688009B1A9AB2104B1A80002318467037BD46D1
:1076980080BD00BF54400020C02D0508C42D05083A
:1076A800CC2D0508E82D0508F02D0508A4ED0020CF
:1076B800FC2D0508082E05081C2E05089C00002036
:1076C80094000020342E0508E441002080B584B0E1
:1076D80000AF7860284BFB60FB685A1CFA603022C8
:1076E8001A7026490720FEF7E1FAFB6830221A7063
:1076F800224B1B6803F01003002B06D0FB681B7895
:1077080043F00403DAB2FB681A700021CC2003F0BE
:10771800F3FD0346002B06D0FB681B7843F00803F3
:10772800DAB2FB681A70164B1B7803F00103002BC2
:1077380006D0FB681B7843F00103DAB2FB681A70C5
:10774800FB680133FB607B6801331B78452B04D150
:10775800F86800F017F803460AE07B6801331B78E5
:10776800312B04D1F86800F0D7F8034600E0012374
:1077780018461037BD4680BD54400020984300206D
:10778800A2ED002080B584B000AF78600023FB60D4
:10779800ACE0FB6801335D4AD3605C492820FEF702
:1077A80085FA0346002B40F091807B6830221A70DE
:1077B800564B1B69D3F8063003F04003002B06D064
:1077C8007B681B7843F00103DAB27B681A704F4B71
:1077D8001B69D3F8063003F00403002B06D07B683E
:1077E8001B7843F00203DAB27B681A70474B1B69B7
:1077F800D3F8063003F01003002B06D07B681B7803
:1078080043F00403DAB27B681A70404B1B69D3F863
:107818000A3003F00203002B07D13C4B1B69D3F855
:10782800063003F00803002B06D07B681B7843F072
:107838000803DAB27B681A707B6801337B607B6867
:1078480030221A70314B1B69D3F8063003F001035C
:10785800002B06D07B681B7843F00103DAB27B6803
:107868001A702A4B1B69D3F8063003F48063002B87
:1078780006D07B681B7843F00203DAB27B681A7083
:10788800224B1B69D3F8063003F00203002B06D005
:107898007B681B7843F00403DAB27B681A701B4BD1
:1078A8001B69D3F80A3003F00103002B06D07B686C
:1078B8001B7843F00803DAB27B681A707B680133DF
:1078C8007B6012492B20FEF7F1F909E07B685A1C0E
:1078D8007A6030221A707B685A1C7A6030221A70DB
:1078E8007B6800221A70FB680133FB60FB681F2B62
:1078F8007FF74FAF064841F0C5F903469AB2054BEA
:107908001A80002318461037BD4680BD84430020E6
:1079180054400020E441002080B584B000AF786076
:107928000023FB60FEE0FB680133864AD36085498B
:107938002820FEF7BBF90346002B40F0E380814B7B
:107948001B69D3F8063003F48073002B00F0CB805A
:107958007B6880221A707B4B1B69D3F8063003F4CE
:107968000073002B06D07B681B7843F01003DAB253
:107978007B681A70734B1B69D3F8063003F0400319
:10798800002B06D07B681B7843F00103DAB27B68D2
:107998001A706C4B1B69D3F8063003F00403002BF4
:1079A80006D07B681B7843F00203DAB27B681A7052
:1079B800644B1B69D3F8063003F01003002B06D084
:1079C8007B681B7843F00403DAB27B681A705D4B5E
:1079D8001B69D3F80A3003F00203002B07D1594B77
:1079E8001B69D3F8063003F00803002B06D07B6828
:1079F8001B7843F00803DAB27B681A707B6801339E
:107A08007B607B6800221A704E4B1B69D3F80630E6
:107A180003F00103002B07D17B681B7863F06F0329
:107A2800DAB27B681A701EE0464B1B695B7903F07B
:107A38000F03BB60BB68002B02DDBB68082B07DDAA
:107A48007B681B7863F06F03DAB27B681A700AE010
:107A58007B681B785AB2BB681B015BB213435BB2ED
:107A6800DAB27B681A70374B1B69D3F8063003F01B
:107A78000103002B06D07B681B7843F00103DAB2C0
:107A88007B681A702F4B1B69D3F8063003F48063A8
:107A9800002B06D07B681B7843F00203DAB27B68C0
:107AA8001A70284B1B69D3F8063003F00203002B29
:107AB80006D07B681B7843F00403DAB27B681A703F
:107AC800204B1B69D3F80A3003F00103002B06D0C2
:107AD8007B681B7843F00803DAB27B681A707B680E
:107AE80001337B6009E07B685A1C7A6080221A7037
:107AF8007B685A1C7A6080221A7012492B20FEF784
:107B0800D5F809E07B685A1C7A6080221A707B6875
:107B18005A1C7A6080221A707B6800221A70FB68EF
:107B28000133FB60FB681F2B7FF7FDAE064841F071
:107B3800A9F803469AB2054B1A8000231846103755
:107B4800BD4680BD8443002054400020E44100200D
:107B580080B588B000AF78607B6801337B60786857
:107B680001F054F90346FB73FB7B002B00F06B819B
:107B7800FB7B202B00F267817B6802337B607B688C
:107B88001B78303BBB737B6801337B607B681B7859
:107B9800FB77FB7F452B19D17B6801337B607B68C2
:107BA8001B78FB777B6801337B6079680A2001F0DA
:107BB80049F9B8617B680A337B6079680A2001F06B
:107BC80041F978617B680A337B6012E07B68013396
:107BD8007B607968062001F035F9B8617B68063367
:107BE8007B607968062001F02DF978617B6806339F
:107BF8007B607B681B78303BDBB21B017B737B6847
:107C080001331B78303BDBB25AB297F90D3013437E
:107C18005BB27B730023FB7402233B82FB7B8C4AA1
:107C2800D3608B492820FEF741F80346002B40F02B
:107C3800D3800123FB74864B1B69D3F8063003F409
:107C48008063002B00F0F180814B1B69D3F806306C
:107C580003F04803002B40F0E8807D4B1B69BA69AC
:107C68009A617B4B1B697A69DA61FB7F392B0AD1F0
:107C7800774B1B69D3F80A20754B1B6942F0400209
:107C8800C3F80A20B2E0724B1B69D3F8063003F040
:107C98000203002B40F0CB806D4B1B69D3F80A30F0
:107CA80003F00103002B40F0C280694B1B69D3F835
:107CB8000A30674A126923F48E6323F00403C2F87A
:107CC8000A30BB7B0F2B12D1614B1B6900229A75BE
:107CD8005F4B1B69D3F80A205D4B1B6942F4806235
:107CE800C3F80A205A4B1B697A7BDA7507E0584BB0
:107CF8001B69BA7B9A75564B1B690022DA75FB7FA4
:107D0800342B32D1524B1B69002242F03F021A76C3
:107D1800002242F042025A76002242F00F029A767E
:107D28000022DA764A4B1B69002242F03F021A779A
:107D3800002242F042025A77002242F00F029A775C
:107D48000022DA77424B1B69D3F8063003F0200390
:107D5800002B41D03E4B1B69D3F80A203C4B1B69D2
:107D680042F00402C3F80A2036E0FB7F302B0AD128
:107D7800374B1B69D3F80A20354B1B6942F01402B4
:107D8800C3F80A2028E0FB7F312B0AD1304B1B694E
:107D9800D3F80A202E4B1B6942F01002C3F80A20C0
:107DA8001AE0FB7F322B0AD1294B1B69D3F80A2032
:107DB800274B1B6942F02402C3F80A200CE0FB7F22
:107DC800332B36D1224B1B69D3F80A20204B1B6971
:107DD80042F02002C3F80A201D4B1B69D3F80A2081
:107DE8001B4B1B6942F00102C3F80A20184B1B69A0
:107DF800002283F82020002283F82120002283F823
:107E08002220002283F82320114B1B69002283F8CB
:107E18002420002283F82520002283F8262000222F
:107E280083F8272000233B8204E000BF02E000BF64
:107E380000E000BFFB7C002B03D005492B20FDF799
:107E480035FF3B8A00E0022318462037BD4680BD37
:107E580084430020F0B58BB004AF78607B680133B1
:107E68007B6000237B827B8A5A1C7A821A467B6855
:107E78001978984B99547B685A1C7B8A591C7982CB
:107E880019461278934B5A54786800F0BFFF03469E
:107E9800FB75FB7D202B00F2CF837B6802337B6070
:107EA8007B681B78432B25D1FB7D8B4AD3608A499D
:107EB8002820FDF7FBFE0346002B17D1864B1B69D4
:107EC800D3F80620844B1B6922F04002C3F8062031
:107ED800814B1B69D3F80A207F4B1B6922F03002C3
:107EE800C3F80A207C492B20FDF7E0FE7B4B0022DB
:107EF8001A80AAE37B681B78452B40F09382FB7DB0
:107F0800754AD36074492820FDF7D0FE0346002B3C
:107F180040F07C82704B1B69D3F8063003F04003B5
:107F2800002B05D06C4B1B6993F82C30FB6003E0E9
:107F3800694B1B695B79FB60FB68002B02DDFB6802
:107F4800082B01DD0123FB60634B1969FB685A1E8E
:107F580013465B01134438330B440533BB604CE2D2
:107F68007B6801337B607B8AB3F5B87F04D35A49B9
:107F78002B20FDF79BFE66E37B681B78243B322BA6
:107F880000F23B8201A252F823F000BF878000086C
:107F9800038400080384000803840008038400089D
:107FA800038400080384000803840008038400088D
:107FB800038400080384000803840008038400087D
:107FC800038400080384000803840008038400086D
:107FD800038400080384000803840008038400085D
:107FE800038400080384000803840008038400084D
:107FF800038400080384000803840008038400083D
:10800800038400080384000803840008038400082C
:1080180003840008038400080384000861800008C2
:10802800038400080384000803840008EB82000826
:108038003982000803840008038400087782000856
:108048000384000803840008ED8000087D8300088D
:1080580003840008B18000087B8A5A1C7A821A4679
:108068001C4B48219954FB68DAB27B8A591C7982E7
:10807800194602F13003DAB2164B5A54BDE17B8A35
:108088005A1C7A821A46134B242199547B8A114A26
:108098009818114B1B691B6A1A46114940F018FBC6
:1080A8007B8A0A337B82A8E17B8A5A1C7A821A4629
:1080B800084B562199547B8A064A9818064B1B6927
:1080C8005B6A1A46064940F003FB7B8A0A337B82C7
:1080D80093E100BF5440002084430020E441002085
:1080E800442E05087B8A5A1C7A821A469A4B5321D9
:1080F80099547B8A984A3021D154984B1B69D3F8FC
:10810800063003F04003002B08D07B8A924AD25CE9
:108118007B8A42F00102D1B28F4AD1548F4B1B693E
:10812800D3F8063003F00403002B08D07B8A8A4A70
:10813800D25C7B8A42F00202D1B2874AD154874B83
:108148001B69D3F8063003F01003002B08D07B8A94
:10815800814AD25C7B8A42F00402D1B27E4AD15471
:108168007E4B1B69D3F80A3003F00203002B07D1BA
:108178007A4B1B69D3F8063003F00803002B08D0AC
:108188007B8A754AD25C7B8A42F00802D1B2724A75
:10819800D1547B8A01337B827B8A6F4A3021D15448
:1081A8006E4B1B69D3F8063003F00103002B08D08F
:1081B8007B8A694AD25C7B8A42F00102D1B2664A64
:1081C800D154664B1B69D3F8063003F48063002B47
:1081D80008D07B8A604AD25C7B8A42F00202D1B224
:1081E8005D4AD1545D4B1B69D3F8063003F0020396
:1081F800002B08D07B8A584AD25C7B8A42F0040262
:10820800D1B2554AD154554B1B69D3F80A3003F003
:108218000103002B08D07B8A4F4AD25C7B8A42F04C
:108228000802D1B24C4AD1547B8A01337B82E4E004
:108238007B8A5A1C7A821A46474B4D219954474BE0
:108248001B69D3F8063003F02003002B07D07B8A84
:108258005A1C7A821A46404B30219954CDE07B8AC9
:108268005A1C7A821A463C4B31219954C5E07B8AC4
:108278005A1C7A821A46384B50219954374B1B693D
:1082880093F82C30002B0DD1344B1B6993F82C300C
:10829800082B07D97B8A304A13443149184640F0E5
:1082A80017FA1AE02D4B1B69D3F8063003F02003A8
:1082B800002B09D07B8A284A9818BB685B681A4645
:1082C800284940F005FA08E07B8A234A9818BB68D9
:1082D8001B681A46234940F0FBF97B8A06337B82E8
:1082E8008BE07B8A5A1C7A821A461B4B4C21995484
:1082F8001A4B1B69D3F80A3003F02003002B13D064
:108308007B8A154A9818154B1B69DB69164A82FB4C
:1083180003129114DA178A1A144901FB02F29A1A05
:10832800134940F0D5F912E07B8A0B4A98180B4B99
:108338001B699B690C4A82FB03129114DA178A1A8B
:108348000A4901FB02F29A1A094940F0C1F97B8AED
:1083580006337B8251E000BF544000208443002054
:108368004C2E0508542E050883DE1B4340420F009F
:108378005C2E05087B8A5A1C7A821A468E4B542139
:1083880099548E4B1B691B7C2F2B04D98B4B1B6973
:108398001B7C332B07D97B8A5A1C7A821A46864B58
:1083A8003021995408E0854B1A697B8A591C7982D7
:1083B8001946127C804B5A547B8A7F4A03EB020C85
:1083C800BB68D3F80940D3F80D50B968D1F8192023
:1083D800D1F81D30BE68D6F81100D6F81510CDE9D1
:1083E8000201CDE9002322462B467549604640F03C
:1083F8006FF97B8A1E337B8200BF7B681B78002B5A
:108408007FF4AEAD6D492B20FDF750FC7B8A6A4A9C
:108418000021D154684840F035FC03469AB2694BB4
:108428001A8012E17B681B78522B63D1FB7D634A6B
:10843800D36062492820FDF739FC0346002B40F041
:10844800FD805E4B1B6993F82C30002B0BD05B4BE7
:108458001B6993F82C30082B05D8584B1B6993F8E7
:108468002C30FB6001E00123FB60FB68DAB27B8AF9
:10847800591C7982194602F13003DAB24E4B5A542C
:108488004E4B1B69D3F8063003F02003002B07D0AE
:108498007B8A5A1C7A821A46474B3021995406E047
:1084A8007B8A5A1C7A821A46434B312199547B8A1B
:1084B800414A9818414B1B691B6A1A46424940F0C9
:1084C80007F97B8A06337B827B8A3B4A98183B4BA9
:1084D8001B695B6A1A463C4940F0FAF837492B2079
:1084E800FDF7E4FB344840F0CDFB03469AB2354B28
:1084F8001A80AAE0FB7D002B40F0A2807B681B78E5
:10850800532B40F09F807B6801337B607B681B782E
:10851800312B02D10123FB750FE07B681B78322BCE
:1085280002D10923FB7508E07B681B78332B02D145
:108538001123FB7501E01923FB7500237B820023BF
:10854800BB826EE0FB7D1D4AD3601C492820FDF7E5
:10855800ADFB0346002B5ED1184B1B6993F82C30FA
:10856800002B0BD0154B1B6993F82C30082B05D822
:10857800124B1B6993F82C30FB6001E00123FB6070
:10858800FB68DAB27B8A591C7982194602F13003FA
:10859800DAB2094B5A54094B1B69D3F8063003F079
:1085A8002003002B12D07B8A5A1C7A821A46024B6F
:1085B8003021995411E000BF54400020844300202A
:1085C800642E0508E4410020542E05087B8A5A1CB5
:1085D8007A821A461F4B312199547B8A1D4A981872
:1085E8001D4B1B691B6A1A461C4940F071F87B8AAF
:1085F8000A337B827B8A174A9818174B1B695B6A78
:108608001A46164940F064F87B8A0A337B8212497D
:108618002B20FDF74BFBFB7D0133FB75BB8A013338
:10862800BB82BB8A072B8DD90A4840F02BFB034637
:108638009AB20B4B1A8008E000BF04E000BF02E0CA
:1086480000BF00E000BF022300E0002318461C37EB
:10865800BD46F0BD5440002084430020442E050848
:10866800E441002080B584B000AF78607B680133B6
:108678007B60786800F0CAFB0346BB73BB7B202B8A
:1086880056D8BB7B002B31D12C4B1B7843F0010310
:10869800DAB22A4B1A700023FB7323E0FB7B013309
:1086A800274AD36026492820FDF700FB0346002B04
:1086B80015D1234B1B69D3F8063003F48073002BC4
:1086C80009D01F4B1B69D3F80A201D4B1B6942F0C8
:1086D8000202C3F80A201A492B20FDF7E7FAFB7BB0
:1086E8000133FB73FB7B1F2BD8D91FE0BB7B144ADC
:1086F800D36013492820FDF7D9FA0346002B15D17A
:108708000F4B1B69D3F8063003F48073002B09D094
:108718000B4B1B69D3F80A20094B1B6942F0020274
:10872800C3F80A2006492B20FDF7C0FA002300E011
:10873800022318461037BD4680BD00BFA2ED0020B9
:108748008443002080B584B000AF78607B68013333
:108758007B60786800F05AFB0346BB73BB7B202B19
:1087680000F28480444B1B7823F00103DAB2424BB9
:108778001A70BB7B002B4FD10023FB7348E0FB7BB7
:1087880001333E4AD3603D492820FDF78FFA03465E
:10879800002B3AD1394B1B69D3F8063003F0080394
:1087A800002B07D1354B1B69D3F80A3003F00203BD
:1087B800002B26D0314B1B69D3F8063003F48063B5
:1087C800002B0AD02D4B1B69D3F80A202B4B1B69B1
:1087D80042F00802C3F80A2013E0284B1B69D3F8BB
:1087E8000620264B1B6922F00802C3F80620234BFB
:1087F8001B69D3F80A20214B1B6922F00202C3F837
:108808000A201E492B20FDF751FAFB7B0133FB732D
:10881800FB7B1F2BB3D927E0BB7B184AD3601749D2
:108828002820FDF743FA0346002B1DD1134B1B6983
:10883800D3F8063003F00803002B07D10F4B1B6950
:10884800D3F80A3003F00203002B09D00B4B1B6945
:10885800D3F80A20094B1B6942F00802C3F80A2022
:1088680006492B20FDF722FA002300E002231846D0
:108878001037BD4680BD00BFA2ED00208443002014
:1088880080B598B002AF78607B6801337B603B4B62
:1088980000221A807B681B78432B04D10021C82052
:1088A80002F02AFD64E07B681B78572B04D1002175
:1088B800CB2002F021FD5BE07B681B78522B14D1A2
:1088C80007F140031946CA2002F016FDBA6CFB6C8A
:1088D800DBB22B492B483FF0FBFE2A4840F0D2F987
:1088E80003469AB2254B1A8042E07B681B78452BD9
:1088F80018D107F140031946CA2002F0FDFCBA6CF2
:10890800FB6CD9B23B6DDBB200930B461E491D4888
:108918003FF0DEFE1B4840F0B5F903469AB2174B0C
:108928001A8025E07B681B78532B21D107F140037F
:108938001946CA2002F0E0FC07F10C03322200219C
:1089480018463FF095FF7B6D07F10C000F4A19217F
:108958003FF07CFEBA6C07F10C030D4909483FF063
:10896800B7FE084840F08EF903469AB2034B1A80C6
:10897800002318465837BD4680BD00BFE44100209B
:108988007C2E050854400020882E0508982E0508DE
:108998009C2E050880B584B000AF78607B680133F1
:1089A8007B60786800F032FA0346FB737B68023319
:1089B8007B607B681B78303BBB737B6801337B60D3
:1089C8007968032000F03EFA03467B73FB7B002B9B
:1089D80025D0FB7B202B22D8BB7B002B1FD0BB7B59
:1089E800082B1CD8FB7B104AD3600F492820FDF7C1
:1089F8005DF90346002B10D10B4B1969BB7B5A1E3E
:108A080013465B0113440B4445337A7B1A700649BD
:108A18002B20FDF74BF9002302E0022300E002239C
:108A280018461037BD4680BD8443002080B594B0F9
:108A380004AF78607B6801337B60786800F0E6F902
:108A4800034687F83E307B6802337B607B681B787F
:108A5800303B87F83D3097F83E30002B00F095808A
:108A680097F83E30202B00F2908097F83D30002B8D
:108A780000F08B8097F83D30082B00F2868097F83D
:108A88003E30444AD36043492820FDF70FF9034696
:108A9800002B7AD13F4B1B691B7C2F2B04D93D4BF4
:108AA8001B691B7C332B03D9302387F83F3004E044
:108AB800384B1B691B7C87F83F30364B196997F890
:108AC8003D305A1E13465B0113440B444033D3F820
:108AD8000600D3F80A1007F12C02002301930A2399
:108AE80000930F2305F0BAFA2A4B196997F83D301D
:108AF8005A1E13465B0113440B445033D3F8060047
:108B0800D3F80A1007F11C02002301930A230093EB
:108B18000F2305F0A3FA1F4B196997F83D305A1E29
:108B280013465B0113440B444833D3F80600D3F8CB
:108B38000A1007F10C02002301930A2300930F2364
:108B480005F08CFA13492B20FDF7B0F897F83E1082
:108B580097F83D0097F83F3007F10C02039207F1B0
:108B68001C02029207F12C020192009303460A4666
:108B780009490A483FF0ACFD084840F083F803462D
:108B88009AB2074B1A80002300E0022318464037A8
:108B9800BD4680BD84430020A42E05085440002013
:108BA800E4410020B0B588B002AF78607B6801333B
:108BB8007B60786800F02AF90346FB757B6802330E
:108BC8007B607B681B78303BBB757B6801337B60BF
:108BD8007B685A1C7A601B787B757968062000F0E0
:108BE80031F938617B6806337B607968062000F0CC
:108BF80029F9F860804B00221A80FB7D002B00F0D9
:108C0800F380FB7D202B00F2EF80BB7D002B00F072
:108C1800EB80BB7D082B00F2E780FB7D774AD360B1
:108C280076492820FDF742F80346002B40F0DF8004
:108C38007B7D522B2AD1F87DBC7D704B1969BB7D99
:108C48005A1E13465B0113440B443833D3F80930DA
:108C58009BB21D46694B1969BB7D5A1E13465B01C1
:108C680013440B443833D3F805309BB20193009575
:108C780023460246624963483FF02AFD614840F0B6
:108C880001F803469AB25C4B1A80A7E07B7D572B0C
:108C980006D07B7D452B03D07B7D442B40F098800C
:108CA800BB7D012B09D9554B1B69D3F81120534BB8
:108CB8001B6942F00102C3F81120BB7D012B27D1AB
:108CC800FA683B691344002B0AD14C4B1B69D3F853
:108CD80006204A4B1B6922F48072C3F806207DE007
:108CE80049490720FCF7E2FF474B1B6823F01003B4
:108CF800454A136044490620FCF7D8FF3F4B1B69DF
:108D0800D3F806203D4B1B6942F48072C3F8062055
:108D18003A4B1B69D3F80A20384B1B6942F004020E
:108D2800C3F80A203869F7F7FFFC02460B463349B7
:108D38000D69B97D4C1E10461946F8F747F80246EA
:108D480023465B0123442B443833C3F80920F868D1
:108D5800F7F7EAFC02460B4628490D69B97D4C1E17
:108D680010461946F8F732F8024623465B012344B9
:108D78002B443833C3F80520204B1B699B7B5AB220
:108D8800BB7D013B012101FA03F35BB213435AB2E5
:108D98001A4B1B69D2B29A737B7D452B0AD1174BAC
:108DA8001B69D3F80A20154B1B6942F48072C3F87B
:108DB8000A2012E07B7D442B0FD1104B1B69D3F89E
:108DC8000A200E4B1B6922F48072C3F80A2004E0C3
:108DD8000A492B20FCF76AFF07E000BF07492B2050
:108DE800FCF764FF002303E000BF022300E0022336
:108DF80018461837BD46B0BDE44100208443002022
:108E0800B42E0508544000209843002080B485B053
:108E180000AF78607B681B78303BFB73FB7B1A469E
:108E2800920013445B00FB737B6801331A78FB7B69
:108E38001344DBB2303BFB73FB7B18461437BD464B
:108E480080BC704780B485B000AF03463960FB71C1
:108E58000023FB600023FB7211E0FA6813469B00B5
:108E680013445B00FB60FB7A3A6813441B781A468C
:108E7800FB681344303BFB60FB7A0133FB72FA7AE0
:108E8800FB799A42E9D3FB6818461437BD4680BC83
:108E98007047000080B58EB000AF002387F83330EC
:108EA80024E097F933308C2202FB03F3154A13446C
:108EB800C7F81D3097F93330124A8C2101FB03F3B0
:108EC80013441833B3F801309BB218463B461A4690
:108ED800012103F06FF878637B6B002B0BD197F9B6
:108EE8003330DBB20133DBB287F8333097F93330F4
:108EF800012BD6DD00E000BF7B6BDBB218463837AC
:108F0800BD4680BD3C3F002080B58AB000AF034617
:108F1800FB8006233B7307F10C03C7F815300023C9
:108F280043F001037B760023BB760023FB76002306
:108F38003B77FB8807F110020321184603F03AF843
:108F480003469BB218462837BD4680BD80B58AB017
:108F580000AF0346FB8015233B7307F10C03C7F8EA
:108F68001530002343F001037B760023BB760023F2
:108F7800FB7600233B77FB8807F110020321184694
:108F880003F018F803469BB218462837BD4680BD43
:108F980080B58AB000AF0346FB800023BB84BB8C3E
:108FA8005A1CBA841A462E4B062199542D4B1B88FD
:108FB800002B3ED0BB8C5A1CBA841A46284B02217F
:108FC8009954022387F8273000237B8413E07A8C96
:108FD800BB8C591CB9841946234B9A5C204B5A54B4
:108FE8007B8C214AD25C97F82730134487F82730C6
:108FF8007B8C01337B841B4B1B887A8C9A42E6D38B
:10900800BB8C5A1CBA841A46154B0321995497F8FD
:109018002730033387F8273097F827305B42DAB2D6
:10902800BB8C591CB984194602F07F03DAB20C4B89
:109038005A540B4BC7F80D30BB8CC7F81130FB885E
:1090480007F108020321184602F0B4FF03463B84E7
:10905800044B00221A803B8C18462837BD4680BD39
:10906800E8410020E44100205440002080B58AB047
:1090780000AF03463960FB80FB8807F10C0204212E
:10908800184602F097FF0346FB84FB8C002B04D1A3
:109098007A7F3B681A70002300E0FF2318462837C0
:1090A800BD4680BD80B584B000AF0346FB7107F1B3
:1090B8000F03184601F01AFBFB79012B05D1FB7B46
:1090C80003F00303DBB2FB7306E0FB7B9B08DBB218
:1090D80003F00303DBB2FB73FB7B032B0FD0032BE3
:1090E8000ADC002B02D0012B03D005E04FF41663F5
:1090F80007E04FF4965304E04FF4165301E04FF4A1
:10910800964318461037BD4680BD80B582B000AF83
:1091180078607B689B889BB27A680421184602F0C5
:109128002DFD7B681B6818460837BD4680BD0000CA
:1091380080B582B000AF002037F038F87860144965
:10914800786837F0DBF878601249786837F011F8FA
:1091580078601149786837F00CF878604823032262
:109168000E49786837F032F878604D2303220C49AD
:10917800786837F02BF87860542303220949786817
:1091880037F024F878607B6818460837BD4680BDFC
:10919800C42E0508C82E0508E42E0508102F05085A
:1091A8002C2F0508442F050880B584B000AF7860DF
:1091B800FFF7BEFF0346184636F042FF0346542B1E
:1091C80057D0542BF4DC4D2B1ED04D2BF0DC1B2B31
:1091D80053D0482BECD12C4BB3F819309BB22A4A08
:1091E80019462A4836F038FC274BB3F8A5309BB20D
:1091F800254A1946264836F02FFC264836F06AFCE0
:10920800002036F0E0FC37E0234836F063FC07F135
:109218000C03184636F0D7FC3B7B7B737B7B013312
:109228001E4A13441B7803F00303022B02D17B7BF5
:10923800203B00E07B7BDBB23B733B7B1B2B1ED0D0
:109248003B7B312B05D1104B9B69C3F30F23FB816B
:1092580008E03B7B322BD7D10B4BD3F8A430C3F3B8
:109268000F23FB81FB8952224121184601F00EFE93
:1092780002E000F015F800BF9AE700BF00E000BF69
:109288001037BD4680BD00BF3C3F0020642F050855
:10929800842F0508A42F0508C02F050860FC0508C1
:1092A80080B584B000AF1A4836F014FC0023FB6088
:1092B8000023BB60FB1D184636F076FC0346002BE6
:1092C80002D1FB791B2B1ED0124BD3F88830FA68D9
:1092D8009A4205D10F4BD3F81431BA689A42E9D0B3
:1092E8000C4BD3F88830FB600A4BD3F81431BB60C1
:1092F800084BD3F88830074AD2F888201946064820
:1093080036F0AAFBD6E700BF1037BD4680BD00BFC8
:10931800DC2F05083C3F002008300508B0B584B0B4
:1093280000AF03463960FB71FB791846FAF750FC29
:109338000346184600F080FFF860FB681B784E2B48
:109348000ED1FB6801331B786F2B09D13B68244988
:109358001A460B4603CB106051601B7813723AE033
:10936800FB681B78572B0DD13B681E4A1D461446D7
:109378000FCC28606960AA60EB6020682861A38828
:10938800AB8228E03B685A1C3A60FA6812781A7077
:109398003B685A1C3A60FA6852781A703B685A1C43
:1093A8003A60FA6892781A703B6800221A70386836
:1093B8003FF068FC03461A463B6813440A4A1D46B8
:1093C80014460FCC28606960AA60EB602388A278F5
:1093D8002B821346AB7400BF1037BD46B0BD00BF2B
:1093E80024300508303005084830050880B483B0BB
:1093F80000AF00237B6017E010497A681346DB0052
:109408009B1A5B000B447A68C3F80A200B497A68F8
:109418001346DB009B1A5B000B4400221A710022E2
:109428005A717B6801337B607B68012BE4DD002384
:1094380018460C37BD4680BC704700BFA8ED002019
:1094480080B400AFBFF34F8F00BFBD4680BC7047EC
:1094580080B500AF054BDB6803F4E0620349044BB9
:109468001343CB60FFF7ECFF00BFFDE700ED00E022
:109478000400FA0580B500AF074B1B68002B07D125
:10948800064A074907483FF023F9034B01221A60AF
:10949800044B184680BD00BF5844002074320508AC
:1094A800803205085C440020B0B58AB000AF214B7B
:1094B80007F108041D460FCD0FC42B68238038F030
:1094C80057FDF86100237B6201233B620AE038F014
:1094D8004FFD0246FB69D31A40F2ED22934201D9AF
:1094E800002322E0FB1D184636F05EFB0346002BE6
:1094F800EDD17B6A102B07D807F108027B6A134469
:109508001A78FB799A4201D000233B627B6A0133C7
:109518007B62FB791E2BD9D13B6A002B04D07B6A76
:10952800112B01D1012300E0002318462837BD463E
:10953800B0BD00BF9032050880B582B000AF0346C9
:10954800FB71FB791D2B01D000230DE0FFF7ACFF69
:109558000346002B07D0064B1B68002B03D00121C4
:109568000448F6F743FE012318460837BD4680BD78
:1095780050440020B043002080B500AF9A22034930
:10958800002036F057FA00BF80BD00BF8C3B0508AD
:1095980080B582B000AF786036F03CFA0346002B05
:1095A80008D0FFF767FF03461A46094978683FF075
:1095B8008FF807E0FFF75EFF03461A46054978680B
:1095C8003FF086F87B6818460837BD4680BD00BF67
:1095D800A4320508CC32050880B5A0B000AF002041
:1095E80036F0E4FDF8674F49F86F36F087FEF86704
:1095F8003B1D1846FFF7CCFF03461946F86F36F0B7
:10960800B8FDF8674849F86F36F0B3FDF8674123AD
:1096180003224649F86F36F0D9FDF8674423032240
:109628004349F86F36F0D2FDF867492303224149D0
:10963800F86F36F0CBFDF867532303223E49F86FE5
:1096480036F0C4FDF867562303223C49F86F36F01C
:10965800BDFDF867572303223949F86F36F0B6FD88
:10966800F86736F0D7F90346002B4FD03549F86F25
:1096780036F07FFDF867432303223349F86F36F04D
:10968800A5FDF867522303223049F86F36F09EFD96
:10969800F8672C49F86F36F06CFDF8673023032221
:1096A8002B49F86F36F092FDF867312303222949D8
:1096B800F86F36F08BFDF867322303222649F86FDE
:1096C80036F084FDF867332303222449F86F36F017
:1096D8007DFDF867342303222149F86F36F076FDC3
:1096E800F867352303221F49F86F36F06FFDF867D6
:1096F800362303221C49F86F36F068FDF8673723D4
:1097080003221A49F86F36F061FDF8672E23032209
:109718001749F86F36F05AFDF867FB6F184680371F
:10972800BD4680BDE0320508E4320508F832050878
:10973800183305083433050850330508683305081D
:1097480078330508883305088C330508B0330508D5
:10975800C4330508E433050800340508383405081F
:109768006C34050888340508A0340508B4340508A5
:10977800C834050880B59EB000AFCB48F6F730FD79
:1097880003463B67C94B01221A603B6F002B1CD074
:10979800C74B01221A60EB22C649002036F04AF96D
:1097A800C54836F097F936F0EFF803469BB2012129
:1097B8001846FDF741FD36F0E7F803469BB2002254
:1097C8000121184602F076F8C3E1B94B1B68002B5B
:1097D80018D1B74B01221A6036F0D6F803469BB26F
:1097E80000220121184602F065F8B44836F034F931
:1097F800B34B1B68002B05D0B24B1B681946B24807
:1098080036F02AF9FFF7E8FE0346184636F018FC4A
:1098180003462E3B292BB0D801A252F823F000BFF3
:10982800F99A000883970008F59800081599000828
:1098380021990008479900086D990008519A000875
:10984800739A00089B99000883970008839700087B
:109858008397000883970008839700088397000878
:10986800839700088397000883970008F5990008F4
:10987800839700089B9A0008D798000883970008E8
:10988800839700088397000883970008239A0008A5
:109898008397000883970008839700088397000838
:1098A8008397000883970008839700088397000828
:1098B800959A0008DD9800088397000883970008A8
:1098C800D1980008A199000800F0AEF941E100F034
:1098D8002FFE3EE136F058F803469BB200220121E4
:1098E800184601F0E7FF39F0EBFF32E100237B6710
:1098F80008E07B6F7A6F7549042038F093FF7B6F1F
:1099080001337B677B6F632BF3DD22E10023FB666A
:10991800FB6E21221A701CE136F036F803469BB222
:1099280000220121184601F0C5FF0F2102203AF05C
:1099380069F8674836F0CEF839F0AEFE09E136F03E
:1099480023F803469BB200220121184601F0B2FF1A
:109958000F2101203AF056F85D4836F0BBF839F08F
:109968009BFEF6E036F010F803469BB20022012178
:10997800184601F09FFF5749012039F06FFD5649FD
:10998800022039F06BFD524836F0A4F839F084FE15
:10999800DFE000F021FBDCE035F0F6FF03469BB288
:1099A80000220121184601F085FF4C4836F092F854
:1099B8004B4836F08FF807F16903184600F096FE19
:1099C80097F86930DB43DBB23A1D1146184600F0C0
:1099D80023FD3B1D184636F07DF8424836F07AF8EC
:1099E8003B4836F077F839F057FEB2E035F0CCFF57
:1099F80003469BB200220121184601F05BFF3A485A
:109A080036F02AF800220121022039F075FC30488E
:109A180036F060F839F040FE9BE035F0B5FF0346BC
:109A28009BB200220121184601F044FF2F4836F06E
:109A380013F800220121012039F05EFC244836F099
:109A480049F839F029FE84E035F09EFF03469BB2C1
:109A580000220121184601F02DFF39F0F9FD1C48BC
:109A680036F038F839F018FE73E035F08DFF03460C
:109A78009BB200220121184601F01CFF39F0C8FDF5
:109A8800134836F027F839F007FE62E0FFF7E0FCEC
:109A98005FE000F0B7FA134836F01CF80C4836F0CF
:109AA80019F839F0F9FD54E0B04300205044002083
:109AB80054440020B43B0508CC340508F0340508AC
:109AC8007CED00201400002008350508283505081D
:109AD800503505086C3505087835050884350508BE
:109AE8009C35050888330508AC350508C0350508D8
:109AF80039F0D2FD034687F86B3097F86B3087F85A
:109B08006A3097F86A300133124A13441B7803F01D
:109B18000303022B03D197F86A30203B01E097F842
:109B28006A3087F86B3097F86B30562B07D0562B76
:109B38003FF723AE502B05D0542B06D01DE600F07E
:109B4800A1F906E000F0D0F803E000F005F800BF46
:109B580013E612E660FC050880B58CB000AF2C480F
:109B680035F0B8FF39F098FD034687F82B3097F8A1
:109B78002B301B2B47D043F69821264835F06CFF35
:109B88003B46002219460020FCF740F8D7E900239D
:109B980013467B627B6AFB6209E03B46002219465A
:109BA8000020FCF733F8D7E900231346FB627A6AF2
:109BB800FB6A9A42F1D007F1140343F6982118463C
:109BC80037F016FD38F0D4F93862134835F082FFC3
:109BD80007F11403184637F07DFD0346002B00D12A
:109BE800F6E700BF38F0C4F9F8610C4835F072FFA9
:109BF800FA693B6AD31A1946094835F02DFF094816
:109C080035F068FFABE700BF3037BD4680BD00BF09
:109C1800D0350508FC3505081C3605082C3605081E
:109C2800443605085836050890B583B002AF35F0BC
:109C3800ABFE03469BB200220121184601F03AFE12
:109C4800FFF718FC1A4B1A681A4B19681A4B1B684D
:109C58001A4C019400930B460146194835F0FCFE56
:109C680039F0A0FD174835F035FF1449164835F08E
:109C7800F3FE0421154835F0EFFE0421144835F0B1
:109C8800EBFE0421134835F0E7FE134B1B68002B4D
:109C980005D0124B1B681946114835F0DDFE1148F6
:109CA80035F018FF39F0F8FC00BF0437BD4690BD09
:109CB8009C000020940000209800002088360508A9
:109CC8006C36050898360508B4360508CC360508FC
:109CD800E4360508FC3605087CED00201400002059
:109CE800083505081437050880B59EB000AF002375
:109CF80087F8773039F0D0FC034687F86B3097F84F
:109D08006B3087F86A3097F86A3001335B4A13443E
:109D18001B7803F00303022B03D197F86A30203B2A
:109D280001E097F86A3087F86B3097F86B301B2B97
:109D380000F09E80572B3DD1514835F0CBFE39F0CD
:109D4800ABFC034687F86B3097F86B301B2B00F0A1
:109D58009180C92387F8583001237B65C92387F888
:109D68005D30002343F0010387F85930002387F85A
:109D78005A30002387F85B30002387F85C303B1D9E
:109D88003B671123FB660023A7F8743009E03B6F9B
:109D98001A1D3A6701221A60B7F874300133A7F820
:109DA8007430B7F87430FA6E9A42F0D8012387F805
:109DB800773000BF97F87730002B5CD00023A7F8E6
:109DC80060300023A7F8623000237B6607F1600348
:109DD8001946032003F040FD0023A7F860300A234A
:109DE800A7F8623007F154037B6607F16003194650
:109DF800022003F031FD0123A7F860300023A7F803
:109E0800623000237B6607F160031946032003F0E4
:109E180023FD0223A7F860300023A7F8623000234F
:109E28007B6607F160031946032003F015FD012343
:109E3800A7F86030FB6E9BB2A7F862303B1D7B66CB
:109E480007F160031946022003F006FD0223A7F874
:109E58006030FB6E9BB2A7F862303B1D7B6607F152
:109E680060031946022003F0F7FC03F0BBFF02E091
:109E780000BF00E000BF7837BD4680BD60FC050824
:109E88002437050880B584B000AF39F005FC0346D7
:109E9800FB73FB7BBB73BB7B01331C4A13441B78EE
:109EA80003F00303022B02D1BB7B203B00E0BB7B0A
:109EB800FB73FB7B412B04D04A2B05D00023BB81CD
:109EC80005E00123BB8102E00223BB8100BFBA8900
:109ED8000F4B1A800323BB800023FB800023BB6049
:109EE8003B1D1946032003F0B7FC0323BB80012365
:109EF800FB8007F10C03BB603B1D1946022003F0F1
:109F0800ABFC00BF1037BD4680BD00BF60FC050834
:109F1800A4ED002080B582B000AF274835F09CFD45
:109F2800264B7B607B6819687B685A687B685B682E
:109F3800234835F091FD7B6808337B607B6819689E
:109F48007B685A687B685B681E4835F085FD7B68CE
:109F580008337B607B6819687B685A687B685B6834
:109F6800194835F079FD7B6808337B607B68196890
:109F78007B685A687B685B68144835F06DFD7B68C0
:109F880008337B607B6819687B685A687B685B6804
:109F98000F4835F061FD7B6808337B607B68196882
:109FA8007B685A687B685B680A4835F055FD00BFD6
:109FB8000837BD4680BD00BF88330508AC3E05089C
:109FC80088370508C4370508003805083C380508EF
:109FD80078380508B438050880B582B002AF4FF06C
:109FE80001630093044B054A4FF00051044839F0CF
:109FF80049FD00BFBD4680BD00F80E0800001820CE
:10A008001D9F000880B58AB000AF00233B820A2359
:10A018007B823B1D7B6107F110031946012003F089
:10A028001BFC3B7ADC2B0AD03B7AD92B07D03B7A36
:10A03800C72B04D93B7AE52B01D8012300E0002384
:10A04800002B02D07B680D2B04DDC8233B72002354
:10A058007B6002E03B7AC83B7B607B7BDC2B0AD0D1
:10A068007B7BD92B07D07B7BC72B04D97B7BE52B4C
:10A0780001D8012300E00023002B03D0D7F80930D2
:10A088000D2B0ADDC8237B7300237B720023BB7270
:10A098000023FB7200233B7302E07B7BC83B7B60A1
:10A0A80000237B6200233B6235F06EFC03469BB2C3
:10A0B80000220121184601F0FDFB544835F00AFD45
:10A0C800534835F007FD534835F004FD3B7A1846F0
:10A0D80000F0B2F8034619464F4835F0BDFC7B7BCB
:10A0E800184600F0A9F8034619464C4835F0B4FC68
:10A0F80000F09CFA0346FB76FB7EBB76BB7E013301
:10A10800474A13441B7803F00303022B02D1BB7E9A
:10A11800203B00E0BB7EFB76FB7E1B2B5BD17B6A82
:10A12800002B02D13B6A002B6BD03E4835F094FCE3
:10A1380000233B8200237B8200237B6107F110030D
:10A148001946032003F088FB00233B820A237B8205
:10A158003B1D7B6107F110031946022003F07CFBCD
:10A168007B6A002B0ED0304835F076FC01233B8209
:10A1780000237B8200237B6107F11003194603202B
:10A1880003F06AFB3B6A002B0ED0284835F064FCCC
:10A1980002233B8200237B8200237B6107F11003AB
:10A1A8001946032003F058FB214835F055FC0323DA
:10A1B800FB610AE0F9691F4835F04EFC4FF47A70EC
:10A1C80037F09AFEFB69013BFB61FB69002BF1DC70
:10A1D80003F008FE15E0FB7E412B06D13B1D184617
:10A1E80000F0A4F801237B625EE7FB7E422B7FF43C
:10A1F8005BAF3B1D0533184600F098F801233B621E
:10A2080052E700BF2837BD4680BD00BFF0380508BB
:10A2180010390508883305083C39050860390508F0
:10A2280060FC050884390508A0390508BC3905080B
:10A23800D8390508003A050880B483B000AF034652
:10A24800FB71FB79C93B182B34D801A252F823F0D3
:10A25800C1A20008BDA20008BDA20008C5A200084E
:10A26800BDA20008BDA20008BDA20008C9A200083E
:10A27800BDA20008F1A20008CDA20008D5A20008DE
:10A28800D9A20008DDA20008E1A20008E5A20008A2
:10A29800BDA20008BDA20008EDA20008BDA20008EA
:10A2A800E9A20008BDA20008BDA20008BDA20008DE
:10A2B800D1A200080F4B18E00F4B16E00F4B14E02B
:10A2C8000F4B12E00F4B10E00F4B0EE00F4B0CE062
:10A2D8000F4B0AE00F4B08E00F4B06E00F4B04E072
:10A2E8000F4B02E00F4B00E00F4B18460C37BD46F2
:10A2F80080BC70470C3A0508183A0508243A050846
:10A308002C3A0508343A05083C3A0508483A050845
:10A31800503A0508583A0508683A0508703A050899
:10A32800783A05087C3A0508883A050880B483B06D
:10A3380000AF78607B681B685A1C7B681A607B6872
:10A348001B680D2B08DD7B6800221A7000225A70EA
:10A3580000229A700022DA707B681B68013B0C2B84
:10A368001CD801A252F823F0ADA30008B5A3000839
:10A37800BDA30008C5A30008CDA30008D5A3000805
:10A38800DDA30008E5A30008EDA30008F5A3000875
:10A39800FDA3000805A400080DA400087B68C822D6
:10A3A8001A7133E07B68C9221A712FE07B68CC22CE
:10A3B8001A712BE07B68D0221A7127E07B68D322C0
:10A3C8001A7123E07B68E1221A711FE07B68D422AE
:10A3D8001A711BE07B68D7221A7117E07B68DB22B1
:10A3E8001A7113E07B68DD221A710FE07B68D522B1
:10A3F8001A710BE07B68D8221A7107E07B68D622B5
:10A408001A7103E07B68D2221A7100BF00BF0C37B3
:10A41800BD4680BC704700BF80B485B000AF03461E
:10A428003960FB710023FB7319E0FB7903F001032A
:10A43800DBB2002B05D03B685A1C3A6031221A70F7
:10A4480004E03B685A1C3A6030221A703B680022CC
:10A458001A70FB795B08FB71FB7B0133FB73FB7B99
:10A46800072BE2D900BF00BF1437BD4680BC704738
:10A4780080B59AB000AF002035F098FE786625497F
:10A48800786E35F03BFF78662349786E35F071FEBB
:10A4980078662249786E35F06CFE7866442303228C
:10A4A8001F49786E35F092FE7866502303221D49C5
:10A4B800786E35F08BFE78660020F9F789FB034645
:10A4C8001846FFF7B9FE03463846252216493EF0DE
:10A4D800FFF8394631230322786E35F077FE786627
:10A4E8000120F9F775FB03461846FFF7A5FE03465A
:10A4F800384625220D493EF0EBF83946322303222F
:10A50800786E35F063FE78667B6E18466837BD4610
:10A5180080BD00BF903A0508983A0508B03A05088A
:10A52800E83A0508003B0508143B0508443B0508C4
:10A5380080B500AFFFF79CFF0346184635F080FD55
:10A548000346702B54D0702BF4DC642B56D0642B4C
:10A55800F0DC1B2B68D01B2BECDB502BEADC312BFF
:10A56800E8DB313B1F2BE5D801A252F823F000BFEE
:10A5780011A600081FA600083DA500083DA5000873
:10A588003DA500083DA500083DA500083DA500081B
:10A598003DA500083DA500083DA500083DA500080B
:10A5A8003DA500083DA500083DA500083DA50008FB
:10A5B8003DA500083DA500083DA5000805A6000822
:10A5C8003DA500083DA500083DA500083DA50008DB
:10A5D8003DA500083DA500083DA500083DA50008CB
:10A5E8003DA500083DA500083DA50008F9A50008FF
:10A5F800002140F2EA30FCF79FF914E0002140F214
:10A60800EA30FBF753FB0EE0002240F2EA3100206B
:10A6180003F0E6FE07E0002240F2EA31012003F0F1
:10A62800DFFE00BF86E785E700BF80BD80B500AFCD
:10A6380039F032F803461A46134B1A70124B1B783E
:10A648002E2B03D1104B1B785BB21BE00E4B1B78F3
:10A65800202B03D80C4B1B785BB213E00A4B1B78FA
:10A668007E2B06D9084B1B781946084835F0F4F9B3
:10A6780005E0054B1B781946054835F0EDF9024B06
:10A688001B785BB2184680BDA8430020803B0508B4
:10A69800883B050880B582B000AF01214120F8F75A
:10A6A80071FC4FF47F43BB804823FB710223BB71CD
:10A6B8003B1D19460B48F8F775F801210920F8F7F2
:10A6C80061FC4FF44043BB801023FB710223BB7134
:10A6D8003B1D19460448F8F765F800BF0837BD4622
:10A6E80080BD00BF00180140000C014080B584B057
:10A6F80000AF78600748F8F77DF90346FB81FB89CE
:10A708001B0A9BB2DAB27B681A7000BF1037BD46CD
:10A7180080BD00BF0018014080B400AF72B600BF12
:10A72800BD4680BC7047000080B483B000AF0346CC
:10A738003960FB7197F90730002B0BDA3B68DAB206
:10A748000C49FB7903F00F03043B1201D2B20B440E
:10A758001A7609E03B68DAB2074997F9073012011F
:10A76800D2B20B4483F8002300BF0C37BD4680BC2F
:10A77800704700BF00ED00E000E100E080B582B066
:10A7880000AF78607B68B3F1807F01D3012327E0B5
:10A798007B6823F07F43144A013B53600F214FF03D
:10A7A800FF30FFF7C1FF104B1A7A00221A725A7A4B
:10A7B80000225A729A7A00229A72DA7A0022DA729F
:10A7C800094B1A78002242F007021A705A780022C0
:10A7D8005A709A7800229A70DA780022DA70002388
:10A7E80018460837BD4680BD10E000E080B400AFD1
:10A7F800034B1B8803F001031846BD4680BC704715
:10A808009C44002080B582B000AFFFF785FF2F4B36
:10A818001B685B092E4AA2FB0323DB091846FFF7D6
:10A82800ADFF0346002B01D000BFFDE72948F7F72D
:10A8380025FF2948F7F722FF2848F7F71FFF284880
:10A84800F7F71CFF2748F7F719FF03F0F5FA034657
:10A858007B807B8845F2AA52934206D07B8843F2DC
:10A86800CC32934201D003F0F1FA1F4B1B8843F01E
:10A8780001039AB21C4B1A8000237B6010E01B4A2C
:10A888007B6813441B78552B07D0174B1B8823F084
:10A8980001039AB2144B1A8005E07B6801337B6090
:10A8A8007B68072BEBDD00237B6007E00F4A7B68A2
:10A8B800134455221A707B6801337B607B68072B31
:10A8C800F4DD37F0FBFD00BFFDE700BF14000020FA
:10A8D800C55A7C0A00080140000C014000100140E4
:10A8E80000140140001801409C44002094100120ED
:10A8F80080B485B000AFF860B9607A6000BF1437E3
:10A90800BD4680BC7047000080B584B000AF786059
:10A918003960584807605848C0F800E04B4B1B683E
:10A928001A464B4B1A604B4B00221A700CE0494BED
:10A938001B781946484B002243F82120454B1B78C9
:10A948000133DAB2434B1A70424B1B78092BEED90C
:10A95800404B00221A7020E03D4B1B68C3F30B03E9
:10A96800B3F57F6F1ED23A4B1B681B6803F07F4319
:10A97800B3F1006F0CD1364B1A68364B1B78591C53
:10A98800C8B23449087019461368334A42F821306E
:10A998002F4B1B6810332E4A13602E4B1B78092B44
:10A9A800DAD900E000BF294B1B681A462B4904205E
:10A9B80037F038FF2A4B1B681A462A49042037F01B
:10A9C80031FF244B00221A7012E0224B1B785A1CCC
:10A9D800204B1B781946204B53F82130224904207C
:10A9E80037F020FF1B4B1B780133DAB2194B1A7072
:10A9F800184B1B78092BE8D97B68FB60FB68002B98
:10AA080019D00DE07B681B785C2B03D07B681B7822
:10AA18002F2B02D17B680133FB607B6801337B609D
:10AA28007B681B78002BEDD13B68FA680F4904203E
:10AA380037F0F8FE05E03B68FA680D49042037F066
:10AA4800F1FE03F0CFF900BFFDE700BF8447002007
:10AA5800904700208C4700205C470020C83B050831
:10AA680088470020DC3B0508F03B0508043C050846
:10AA7800203C0508844700208847002080B400AFA8
:10AA880062B600BFBD4680BC704780B400AF72B6E6
:10AA980000BFBD4680BC704780B586B000AF786007
:10AAA8007B68002B03D12F213048FFF72DFF7B68EF
:10AAB8001B682F4A934203D030212C48FFF724FF0C
:10AAC8007B685B6A1B68002B01D100234AE07B6826
:10AAD8009B6AFB607B689A6A7B680C339A4202D156
:10AAE8007B68183301E07B680C333B61FB681A789C
:10AAF80000221A705A7800225A709A7800229A70A6
:10AB0800DA780022DA70FB681A7900221A715A7909
:10AB180000225A719A7900229A71DA790022DA7140
:10AB2800FB689B68BB6000237B6107E0BA687B69B0
:10AB3800134400221A707B6901337B617B685B6870
:10AB48007A68926802FB03F37A699A42EEDBFFF7B0
:10AB58009CFF7B68FA685A627B683A699A62FFF7D9
:10AB68008DFF012318461837BD4680BD3C3C0508BB
:10AB7800EFADDAFE80B588B000AFF860B9607A60F2
:10AB88003B60FB68002B03D16B215448FFF7BCFEE8
:10AB9800BB68002B03D16C215048FFF7B5FE7B68DA
:10ABA800002B03D16D214D48FFF7AEFE3B68002B0B
:10ABB80003DC6E214948FFF7A7FEBB6A002B03DCC4
:10ABC8006F214648FFF7A0FEFB683A685A60FB68A9
:10ABD800BA6A9A60BB687B610023FB6107E07A6907
:10ABE800FB69134400221A70FB690133FB613B685F
:10ABF800BA6A02FB03F3FA699A42F0DBFB68BA68A7
:10AC08005A61FB681A7B00221A735A7B00225A7316
:10AC18009A7B00229A73DA7B0022DA73FB681A7C2B
:10AC280000221A745A7C00225A749A7C00229A7460
:10AC3800DA7C0022DA747B683B610023BB6107E0A1
:10AC48003A69BB69134400221A70BB690133BB61BE
:10AC58003B68BA6A02FB03F3BA699A42F0DBFB6805
:10AC68007A681A62FB681A7E00221A765A7E0022D7
:10AC78005A769A7E00229A76DA7E0022DA76FB6885
:10AC88001A7F00221A775A7F00225A779A7F002269
:10AC98009A77DA7F0022DA77FA68FB680C329A62D0
:10ACA800FA68FB6818325A62FB681A78002262F068
:10ACB80010021A705A78002262F052025A709A787A
:10ACC800002262F025029A70DA78002262F001020E
:10ACD800DA7000BF2037BD4680BD00BF3C3C050888
:10ACE80080B584B000AF78607B68002B03D19721D2
:10ACF8001948FFF709FE7B681B68184A934203D07E
:10AD080098211548FFF700FE7B689B6A5A687B68A4
:10AD18009B6A1B689A4208DB7B681846FFF7BCFEF3
:10AD28000346002B01D1002311E07B689B6ABB60BE
:10AD3800BB689B68BA6852687968496801FB02F287
:10AD48001344FB60BB685A6801325A60FB681846B6
:10AD58001037BD4680BD00BF3C3C0508EFADDAFEAC
:10AD680080B584B000AFF860B9607A60BB683C2BEE
:10AD78001CD0BB683C2B1EDCBB68042B0ED0BB6808
:10AD8800042B18DCBB68002B03D0BB68012B07D051
:10AD980011E00B4B00221A6000230DE000230BE0AA
:10ADA8007968F86800F034F8034605E0786800F040
:10ADB80009F8034600E0042318461037BD4680BD55
:10ADC8009447002080B485B000AF78607B68FB6052
:10ADD8000D4B1B68002B04D00C4B1A68FB681A60DB
:10ADE8000CE0FB684FF0FF321A704FF0FF325A70D8
:10ADF8004FF0FF329A704FF0FF32DA700023184696
:10AE08001437BD4680BC704794470020A00000203E
:10AE180080B586B002AF786039603B68FB60FB683C
:10AE28009B68442B1AD0452B1FD1134B1B68002B52
:10AE380001D00A231BE0C823009302230F4A1049BC
:10AE48001048FFF797FE0F49786802F0C7FB0A4BD6
:10AE580001221A600C4A7B68136007E0064B002247
:10AE68001A60786802F0F0FB00E000BF0023184683
:10AE78001037BD4680BD00BF9447002028490020F8
:10AE880098470020F4ED0020A000002080B58AB08B
:10AE980000AF0346FB800B467B7113463B7145238D
:10AEA8007B61FB8807F10C0201211846FFF758FF68
:10AEB8000346002B40F06481FB88013319468D4816
:10AEC80034F0CAFD002387F827308B4B00221A7014
:10AED800894B3B620023FB6107F10A0207F10B0370
:10AEE8001146184600F056F90346FB76FB7E642BA4
:10AEF80009D144237B61FB8807F10C020121184624
:10AF0800FFF72EFF3DE1FB7E002B11D07A4B1B781B
:10AF1800002B00F03381784834F0DCFD64220021F6
:10AF280075483DF0A5FC744B3B620023FB6125E1AD
:10AF380097F92730FA7A93424CD0FB7A87F8273072
:10AF48006D4B1B78002B0BD06B4834F0C3FD64228B
:10AF5800002169483DF08CFC674B3B620023FB6194
:10AF6800FB7A742B1AD197F90430542B0AD13B6A17
:10AF780062491A460B4603CB106051603B6A07339F
:10AF88003B6225E03B6A5E4A1068186091889279B6
:10AF980099809A713B6A06333B6219E097F904304D
:10AFA800522B0AD13B6A57491A460B4603CB10600D
:10AFB80051603B6A07333B620AE03B6A524A1068B9
:10AFC80018609188927999809A713B6A06333B623E
:10AFD8000523FB6197F90530412B78D1BB7A013302
:10AFE8004A4A13441B7803F09703002B2ED0FB69C1
:10AFF8004E2B1DDD404B1B78002B0BD03E4834F008
:10B0080069FD642200213C483DF032FC3A4B3B622A
:10B018000023FB613B6A3E4A106818609188927968
:10B0280099809A713B6A06333B62FB690533FB6181
:10B03800BA7A3B6A1A703B6A013300221A703B6A7B
:10B0480001333B62FB690133FB6145E7FB694B2B2D
:10B058000FDCFB694A2B0CDDBB7A1A462D49386A8E
:10B068003DF036FB3B6A04333B62FB690433FB610A
:10B0780085E0FB694A2B1DDD1F4B1B78002B0BD08D
:10B088001D4834F027FD642200211B483DF0F0FBE9
:10B09800194B3B620023FB613B6A1D4A106818602C
:10B0A8009188927999809A713B6A06333B62FB6971
:10B0B8000533FB61BB7A1A461749386A3DF008FB2D
:10B0C8003B6A05333B62FB690533FB6104E7FB69B7
:10B0D8004D2B25DCFB694C2B22DDBB7A1A460F4928
:10B0E800386A3DF0F5FA3B6A02333B62FB6902338A
:10B0F800FB6144E0983C0508B84A0020AC3C0508D0
:10B10800B43C0508BC3C0508C43C050860FC0508BF
:10B11800CC3C0508D43C0508DC3C0508E43C0508A3
:10B12800FB694C2B1DDD184B1B78002B0BD01648E8
:10B1380034F0D0FC6422002113483DF099FB124BF7
:10B148003B620023FB613B6A104A106818609188D3
:10B15800927999809A713B6A06333B62FB690533A1
:10B16800FB61BB7A1A460A49386A3DF0B1FA3B6A74
:10B1780003333B62FB690333FB61ADE600BFABE61B
:10B1880000BF2837BD4680BDB84A0020CC3C050822
:10B19800EC3C050880B584B000AF7860396007F1F1
:10B1A8000B03184634F000FD0346002B1AD1FB7A36
:10B1B800722B0CD0722B15DC522B08D0522B11DCC1
:10B1C8001B2B02D0202B04D00CE064231DE052235B
:10B1D8001BE0002034F0F7FC03461B2B01D164234D
:10B1E80013E000BF0B48FFF77BFDF860FB68002BFE
:10B1F80009D0FB681A787B681A70FB685A783B6834
:10B208001A70002301E04FF0FF3318461037BD468F
:10B2180080BD00BFF4ED002080B485B000AF786039
:10B228000B46FB70164B1B687A689A4202D040F2B4
:10B23800E9331FE0134B5B6AFB60FB681A68114B2C
:10B248009B689A4214DA72233B72FB787B72FB6824
:10B258009A68FB681B685B0013441A4607F10803E9
:10B268001B881380FB681A6801321A60002301E00A
:10B2780040F2E93318461437BD4680BC704700BF1A
:10B28800A0000020F4ED002080B485B000AF786005
:10B298000B46FB70164B1B687A689A4202D040F244
:10B2A800E9331FE0134B5B6AFB60FB681A68114BBC
:10B2B8009B689A4214DA74233B72FB787B72FB68B2
:10B2C8009A68FB681B685B0013441A4607F1080379
:10B2D8001B881380FB681A6801321A60002301E09A
:10B2E80040F2E93318461437BD4680BC704700BFAA
:10B2F800A0000020F4ED002080B582B000AF786097
:10B3080039607B68A3F2E933032B1ED801A252F8F7
:10B3180023F000BF35B300083FB3000849B3000865
:10B328002DB3000800F03EF8034635E0386800F019
:10B33800C3F9002330E0386800F004FA00232BE05A
:10B34800386800F0CBF9002326E07B68C83B042B63
:10B3580021D801A252F823F075B300087DB3000884
:10B3680087B3000891B3000899B3000800F01AF8F1
:10B37800034611E0386800F075F803460CE03868B9
:10B3880000F00AF9034607E000F076F9034603E007
:10B39800034B1B6800E0012318460837BD4680BDF3
:10B3A8007C52002080B483B000AF2A4B00221A6080
:10B3B800294B00221A60294B00221A60284B7B6017
:10B3C80000233B603DE07B68002283F83A2000229E
:10B3D80083F83B20002283F83C20002283F83D209C
:10B3E8007B68002283F83620002283F83720002269
:10B3F80083F83820002283F839207B68002283F8FC
:10B408003A20002283F83B20002283F83C200022C7
:10B4180083F83D207B68002283F83E20002283F8D1
:10B428003F20002283F84020002283F841207B68D7
:10B43800002283F842207B6876337B603B680133C7
:10B448003B603B680F2BBEDD002318460C37BD461A
:10B4580080BC70477C52002080520020845200201B
:10B468001C4B002080B584B000AF78607B68FB601F
:10B47800464B1B680F2B7FDC454B1B68002B03DBFF
:10B48800434B1B680F2B02DD414B00221A60404BD7
:10B498001B68762202FB03F33E4A9818FB681B6878
:10B4A800322219463DF0BCFA394B1B68394A7621DD
:10B4B80001FB03F31344313300221A70344B1B6829
:10B4C800FA6852683349762000FB03F30B443033A3
:10B4D800C3F802202E4B1B68FA6892682D49762023
:10B4E80000FB03F30B443033C3F80620284B1B68DA
:10B4F800FA68D2682749762000FB03F30B443833F7
:10B50800C3F80220224B1B68FA6812692149762089
:10B5180000FB03F30B443833C3F806201C4B1B68AD
:10B52800762202FB03F340331A4A1344981CFB6843
:10B538005B69322219463DF073FA154B1B68154AB0
:10B54800762101FB03F31344733300221A707868E1
:10B5580002F000FE0D4B1B6801330C4A13600C4BC4
:10B568001B6801330A4A1360094B1B680F2B08DD5F
:10B57800074B00221A6004E036F062FF034B1022EA
:10B588001A60002318461037BD4680BD7C52002043
:10B59800805200201C4B002080B485B000AF78603A
:10B5A8007B68FB60314B1B68002B03DB2F4B1B6850
:10B5B8000F2B02DD2D4B00221A602C4B1B687622C4
:10B5C80002FB03F32A4A1344BB602A4B1B68002B77
:10B5D80019D0BB68D3F83220FB685A60BB68D3F82F
:10B5E8003620FB689A60BB68D3F83A20FB68DA60BB
:10B5F800BB68D3F83E20FB681A61BB6803F14202BE
:10B60800FB685A612CE0FB6800221A7100225A710B
:10B6180000229A710022DA71FB6800221A72002255
:10B628005A7200229A720022DA72FB6800221A7398
:10B6380000225A7300229A730022DA73FB680022F0
:10B648001A7400225A7400229A740022DA74FB6871
:10B6580000221A7500225A7500229A750022DA759E
:10B66800002318461437BD4680BC7047845200201A
:10B678001C4B00207C52002080B400AF0C4B1B6890
:10B68800002B10D00A4B1B68013B094A1360094B79
:10B698001B680133074A1360064B1B680F2B02DD3A
:10B6A800044B00221A6000231846BD4680BC704730
:10B6B8007C5200208452002080B483B000AF7860B0
:10B6C8007B68002B02D07B68034A1A6000BF0C37E6
:10B6D800BD4680BC704700BFF43C050880B483B009
:10B6E80000AF786000BF0C37BD4680BC70470000D3
:10B6F80080B582B000AF002034F058FD78600D4965
:10B70800786834F0FBFD78600B49786834F031FDD7
:10B7180078600A49786834F02CFD78605323032256
:10B728000749786834F052FD78607B681846083716
:10B73800BD4680BD043D0508083D05081C3D0508BB
:10B74800303D050880B582B000AF7860FFF7D0FFC4
:10B758000346184634F074FC03461B2B05D0532BC4
:10B7680002D100F007F800BFF0E700BF0837BD4678
:10B7780080BD0000B0B5B0B004AF484B1B68002BCB
:10B788005AD0464B1B68C7F8AC300023C7F8A8301E
:10B798004BE0D7F8A830762202FB03F3404A134463
:10B7A800C7F8A430D7F8A430D3F83230002B0FD123
:10B7B800D7F8A430002242F0300283F83220002269
:10B7C80083F83320002283F83420002283F83520C0
:10B7D800D7F8A430D3F83230DBB21D46D7F8A430FE
:10B7E800D3F836305C1CD7F8A430D3F83A30D7F801
:10B7F800A420D2F83E20D7F8A4104231381D029177
:10B808000192009323462A4626493CF061FF3B1DDE
:10B81800184634F05FF9D7F8AC30013BC7F8AC30C4
:10B82800D7F8A8300133C7F8A830D7F8A820D7F838
:10B83800AC309A42ADDB02E01B4834F04BF91B48B0
:10B8480034F048F9002034F0BEF90346C7F8A030B8
:10B85800D7F8A030C7F89C30D7F89C300133144A89
:10B8680013441B7803F00303022B03D1D7F89C3051
:10B87800203B01E0D7F89C30C7F8A030D7F8A030BB
:10B888001B2B07D0D7F8A030432B02D1FFF78AFD36
:10B8980000BF72E700BFB037BD46B0BD7C52002084
:10B8A8001C4B0020443D0508743D0508883D0508EB
:10B8B80060FC050880B582B000AF03463A60FB80A3
:10B8C8000B46BB80BB88062B2AD801A252F823F06E
:10B8D800F5B80008FBB8000829B9000805B9000840
:10B8E80029B9000811B900081DB9000800F020F8AE
:10B8F80018E0FB88184600F021F813E0FB88396847
:10B90800184600F03DF80DE0FB883968184600F04D
:10B91800B7F807E0FB88184600F0FAF8034602E09B
:10B92800012300E0002318460837BD4680BD00BF4C
:10B9380080B400AF00BFBD4680BC704780B584B0FE
:10B9480000AF0346FB800023FB600C4B1B221A70E0
:10B958000A4B5B225A70094B32229A70074B4A22D3
:10B96800DA700423FB60FB88044AF968184600F083
:10B97800E2F800BF1037BD4680BD00BF88520020E6
:10B9880080B584B000AF03463960FB803B68FB603C
:10B99800394BBB60BB685A1CBA601B221A70BB6863
:10B9A8005A1CBA605B221A70FB68DB889BB20133B1
:10B9B800324A82FB03129210DB17D31ADAB2BB6841
:10B9C800591CB9603032D2B21A70FB68DB889BB25E
:10B9D8005A1C2A4B83FB02139910D317C91A0B461A
:10B9E8009B000B445B00D11ACAB2BB68591CB960F2
:10B9F8003032D2B21A70BB685A1CBA603B221A7035
:10BA0800FB681B899BB201331C4A82FB031292100C
:10BA1800DB17D31ADAB2BB68591CB9603032D2B21C
:10BA28001A70FB681B899BB25A1C144B83FB0213C8
:10BA38009910D317C91A0B469B000B445B00D11A07
:10BA4800CAB2BB68591CB9603032D2B21A70BB682E
:10BA58005A1CBA6048221A70BB6800221A7006483D
:10BA68003DF010F90146FB88034A184600F063F8D8
:10BA780000BF1037BD4680BD8852002067666666E5
:10BA880080B586B000AF03463960FB803B68FB6039
:10BA9800FB681B687B61FB689B889BB2002B30D0DE
:10BAA80000237B827B8A194A0021D1541AE07B69E2
:10BAB8001B780A2B06D17B8A5A1C7A821A46134BAA
:10BAC8000D2199547B695A1C7A617A8A511C7982B2
:10BAD80019780E4B99547B8A0C4A0021D1547B8AE1
:10BAE800DE2B04D87B691B78002BE0D100E000BF77
:10BAF80006483DF0C7F80146FB88044A184600F09E
:10BB08001AF800BF1837BD4680BD00BF8852002014
:10BB180080B58AB000AF0346FB80FB8807F10C02B2
:10BB28000821184600F046FA0346FB84FB8C1846A9
:10BB38002837BD4680BD80B58AB000AF0346B960DE
:10BB48007A60FB8101E0FAF72FF8FB891846FFF7C6
:10BB5800DFFF0346002BF6D17B68C7F81530BB68BA
:10BB6800C7F81930FB8907F110020321184600F0C5
:10BB780021FA00BF2837BD4680BD000080B582B0DD
:10BB880000AF03463A60FB800B46BB80BB88B3F529
:10BB98007B7F1CD0B3F57B7F3FDC052B12DC002BB1
:10BBA8003BDB052B39D801A252F823F0D7BB00089C
:10BBB800DFBB0008EDBB0008F9BB000807BC0008A4
:10BBC80015BC0008A3F2E933012B26D823E000F0C6
:10BBD80071F8034628E0FB883968184600F0ACF88D
:10BBE800034621E0FB88184600F0E8F803461BE00E
:10BBF800FB883968184600F01DF9034614E0FB88F5
:10BC08003968184600F042F903460DE0386800F03C
:10BC180081F8034608E0002306E0B988FB883A6803
:10BC28001846F9F7C7FF034618460837BD4680BDD2
:10BC380080B586B000AF4FF4A060F7F7B9F80121DE
:10BC48000120F7F7D9F91C233B7400237B740123E7
:10BC5800BB740123FB7407F110031846F6F76AF961
:10BC6800124B1B68124AA2FB0323DB097B617B6929
:10BC78009BB23B810023BB8000237B810023FB8098
:10BC88003B1D19464FF08040F7F72AFA012201219F
:10BC98004FF08040F7F7B4FB01214FF08040F7F7F1
:10BCA8001BFB00BF1837BD4680BD00BF1400002035
:10BCB800D34D621080B582B000AF0023FB8016E040
:10BCC800FA88134913465B0013445B000B440022B7
:10BCD8001A80FA880E4913465B0013445B000B4434
:10BCE80000225A8000229A80FB880133FB80FB885F
:10BCF800092BE5D9FFF79CFF00224FF47B71002048
:10BD0800F9F758FF002318460837BD4680BD00BF25
:10BD18007053002080B485B000AF78607B68FB600A
:10BD2800044B1A68FB681A60002318461437BD468E
:10BD380080BC70476C53002080B487B000AF0346C6
:10BD48003960FB80FB88002B01D002232FE03B6881
:10BD5800FB60194B3B610023FB821FE03B691B889A
:10BD68009BB2002B14D1FB681B681A463B69C3F8C9
:10BD780002203B69002242F001021A7000225A7028
:10BD8800FB8A03F5FA739AB2FB689A8000230EE0E7
:10BD98003B6906333B61FB8A0133FB82FB8A092B33
:10BDA800DCD9FB6800221A7100225A710123184657
:10BDB8001C37BD4680BC70477053002080B485B0E6
:10BDC80000AF0346FB80FB88002B01D1022329E04A
:10BDD800FB88B3F5FA7F03D3FB88B3F5FF7F01D95E
:10BDE80002231FE0FB88A3F5FA73FB80FB88092B6D
:10BDF80017D8FA8813465B0013445B000C4A1344B7
:10BE0800FB60FB6800221A7000225A70FB6800224F
:10BE18009A700022DA7000221A7100225A710023E7
:10BE280000E0022318461437BD4680BC704700BFA7
:10BE38007053002080B485B000AF03463960FB80A2
:10BE4800FB88A3F5FA73FB803B68FB60FB88092B32
:10BE580014D8FA8813465B0013445B000A4A13445B
:10BE6800BB60BB681B889BB2012B07D1FB681B68B2
:10BE78001A46BB68C3F80220002300E002231846D4
:10BE88001437BD4680BC70477053002080B485B01D
:10BE980000AF03463960FB80FB88A3F5FA73FB808B
:10BEA8003B68FB60FB88092B14D8FA8813465B00B3
:10BEB80013445B000F4A1344BB60BB681B889BB2EA
:10BEC800012B07D1BB68D3F802301A46FB681A6009
:10BED800002309E0FB6800221A7000225A70002231
:10BEE8009A700022DA70022318461437BD4680BCC7
:10BEF800704700BF7053002080B582B000AF0121A9
:10BF08004FF08040F7F722FB204B1B6801331F4A94
:10BF180013600023FB802AE0FA881D4913465B0062
:10BF280013445B000B441B88012B1DD1FA88184968
:10BF380013465B0013445B000B44D3F80230002B1C
:10BF480012D0FA88124913465B0013445B000B4475
:10BF5800D3F80230FA88591E0D4813465B00134483
:10BF68005B000344C3F80210FB880133FB80FB88A5
:10BF7800092BD1D9F9F72CFE064B1B680133054A6A
:10BF8800136000BF0837BD4680BD00BF20EE00200B
:10BF9800705300206C53002080B400AF62B600BF1D
:10BFA800BD4680BC704780B400AF72B600BFBD46C6
:10BFB80080BC704780B584B000AFF860B9607A6023
:10BFC800BB68B3F57B7F03D100F08CF8034683E0B0
:10BFD800BB68002B07D1FB689BB27968184600F054
:10BFE8004BFB034678E0FB68002B02DBFB68042B65
:10BFF80001DD032370E0BB68013B082B6BD801A26D
:10C0080052F823F031C00008DFC000084FC0000814
:10C01800BFC00008DFC00008CFC00008DFC00008AC
:10C0280041C000085FC00008FB689BB279681846E9
:10C0380000F04AFD03464FE0FB689BB2184600F04B
:10C0480067FE034648E0FB689BB27968184601F032
:10C0580041F8034640E0FFF7A6FF2149FA68134676
:10C068001B0113449A01D21A8B1828331B889BB2E0
:10C07800012B11D1FB689BB2184601F099F81849B9
:10C08800FA6813461B0113449A01D21A8B183033ED
:10C0980000221A7100225A711149FA6813461B01CD
:10C0A80013449A01D21A8B18443300221A70FFF7EE
:10C0B80073FF002310E0FB689BB27968184601F013
:10C0C80089F8034608E0FB689BB27968184600F0D7
:10C0D80093FE034600E0012318461037BD4680BD95
:10C0E80024EE002080B58EB000AFE04B7B637B6B05
:10C0F80000221A707B6B00225A70002242F038022C
:10C108009A70002242F00102DA70002242F04002E6
:10C118001A717B6B002242F0250283F82620002248
:10C1280083F827207B6B00225A72002242F04002DB
:10C138009A720022DA7200221A737B6B002242F094
:10C1480004025A7100229A717B6B00225A730022F2
:10C1580042F008029A73002242F00102DA730022C8
:10C1680042F040021A747B6B002242F00402DA713A
:10C1780000221A727B6B0022DA74002242F0080255
:10C188001A75002242F001025A75002242F040025C
:10C198009A757B6B00225A74002242F002029A744C
:10C1A8007B6B0022DA75002242F004021A767B6B60
:10C1B80000225A767B6B00229A760022DA767B6B15
:10C1C80000221A7700225A7700229A770022DA771B
:10C1D8007B6B002283F82020002283F82120532340
:10C1E8003B60A34BC7F81D303B461946002000F0C2
:10C1F800B5FAA04B7B637B6B00221A707B6B002225
:10C208005A70002242F044029A700022DA7000222A
:10C2180042F040021A717B6B002242F0260283F83A
:10C228002620002283F827207B6B00225A720022E6
:10C238009A72002242F00202DA7200221A737B6BB1
:10C2480000225A7200229A72002242F00202DA7226
:10C2580000221A737B6B002242F004025A710022FA
:10C268009A717B6B00225A73002242F008029A737B
:10C27800002242F00102DA73002242F040021A74EE
:10C288007B6B002242F00402DA7100221A727B6B87
:10C298000022DA74002242F008021A75002242F0E5
:10C2A80001025A75002242F040029A757B6B002207
:10C2B80042F004025A7400229A747B6B002242F006
:10C2C8000802DA7500221A767B6B01225A767B6B9C
:10C2D800002242F040029A760022DA767B6B002236
:10C2E8001A77002242F018025A77002242F001021F
:10C2F8009A77002242F04002DA777B6B002242F004
:10C30800010283F82020002283F8212053233B6078
:10C31800574BC7F81D303B461946012000F01EFA5E
:10C32800554B7B637B6B00221A707B6B00225A7023
:10C33800002242F048029A700022DA70002242F08D
:10C3480040021A717B6B002242F0270283F82620F4
:10C35800002283F827207B6B00225A7200229A72EF
:10C36800002242F00402DA7200221A737B6B002268
:10C3780042F008025A7100229A717B6B00225A73AC
:10C38800002242F00C029A73002242F00102DA7392
:10C39800002242F040021A747B6B002242F008022D
:10C3A800DA7100221A727B6B0022DA74002242F0E2
:10C3B8000C021A75002242F001025A75002242F05E
:10C3C80040029A757B6B00225A74002242F00402E4
:10C3D8009A747B6B0022DA75002242F008021A7602
:10C3E8007B6B01225A767B6B002242F040029A76E0
:10C3F8000022DA767B6B00221A77002242F01802BC
:10C408005A77002242F001029A77002242F0400255
:10C41800DA777B6B002242F0020283F820200022A8
:10C4280083F8212053233B60114BC7F81D303B464E
:10C438001946022000F092F9104B7B637B6B0022B7
:10C448001A707B6B00225A70002242F04C029A70DC
:10C458000022DA70002242F040021A717B6B00223F
:10C4680042F0340283F82620002209E024EE00205E
:10C47800B03D050853F2002082F60020B1FA0020F2
:10C4880083F827207B6B00225A7200229A720022BE
:10C4980042F00802DA7200221A737B6B002242F023
:10C4A80010025A7100229A717B6B00225A73002283
:10C4B80042F010029A73002242F00102DA7300225D
:10C4C80042F040021A747B6B002242F01002DA71CB
:10C4D80000221A727B6B0022DA74002242F01002EA
:10C4E8001A75002242F001025A75002242F04002F9
:10C4F8009A757B6B00225A74002242F004029A74E7
:10C508007B6B0022DA75002242F008021A767B6BF8
:10C5180000225A767B6B00229A760022DA767B6BB1
:10C5280000221A7700225A7700229A770022DA77B7
:10C538007B6B002283F82020002283F821205323DC
:10C548003B604A4BC7F81D303B461946032000F0B4
:10C5580005F9474B7B637B6B00221A707B6B0022CB
:10C568005A70002242F050029A700022DA700022BB
:10C5780042F040021A717B6B002242F0350283F8C8
:10C588002620002283F827207B6B00225A72002283
:10C598009A72002242F01002DA7200221A737B6B40
:10C5A800002242F010025A7100229A717B6B00221D
:10C5B8005A73002242F010029A73002242F00102DC
:10C5C800DA73002242F040021A747B6B002242F0B8
:10C5D8002002DA7100221A727B6B0022DA740022C0
:10C5E80042F014021A75002242F001025A75002224
:10C5F80042F040029A757B6B00225A74002242F086
:10C6080010029A747B6B002242F00402DA75002251
:10C618001A767B6B00225A767B6B00229A76002270
:10C62800DA767B6B00221A7700225A7700229A77F3
:10C638000022DA777B6B002283F82020002283F81F
:10C64800212053233B60094BC7F81D303B46194650
:10C65800042000F083F8074B01221A60FFF79CFCC6
:10C66800002318463837BD4680BD00BFB03D0508D9
:10C67800E0FE0020B053002080B584B000AF034630
:10C688003960FB803B68FB60FB681B79653B042BCA
:10C6980046D801A252F823F0B5C60008C9C600085A
:10C6A800E1C60008F9C6000811C70008FB680022A7
:10C6B8005A7100229A710022DA7100221A7246E039
:10C6C800FB68002242F001025A7100229A7100228E
:10C6D800DA7100221A723AE0FB68002242F0020284
:10C6E8005A7100229A710022DA7100221A722EE021
:10C6F800FB68002242F003025A7100229A7100225C
:10C70800DA7100221A7222E0FB68002242F0040269
:10C718005A7100229A710022DA7100221A7216E008
:10C72800FB68D3F8052005230B49042036F07AF876
:10C73800FB684FF0FF325A714FF0FF329A714FF099
:10C74800FF32DA714FF0FF321A72042300E000233F
:10C7580018461037BD4680BDBC3D050880B58CB075
:10C7680002AF03463960FB803B687B62FA88134658
:10C778001B0113449A01D21AD24B13443B623B6A01
:10C7880003F2FF303B6A03F179013B6A03F23B2273
:10C79800962300930323FEF7EDF93B6A002283F802
:10C7A80044203B6A002283F845203B6A002283F834
:10C7B80046203B6A002283F82B24002283F82C248D
:10C7C800002283F82D24002283F82E243B6A0022BD
:10C7D80083F83420002283F835203B6A002283F84E
:10C7E8003620002283F83720002283F838200022E0
:10C7F80083F839203B6A002283F83A20002283F824
:10C808003B20002283F83C20002283F83D203B6A2D
:10C81800002283F83E20002283F83F20002283F87C
:10C828004020002283F841207B6A1A683B6AC3F8DB
:10C8380022203B6A002283F82820002283F829203E
:10C848003B6A00221A7007F110031846F5F7AAF898
:10C85800FB88042B00F2C58001A252F823F000BF28
:10C868007DC80008BFC8000801C9000843C90008FE
:10C8780085C90008FA88934913461B0113449A0195
:10C88800D21A8B18D3F8093001211846F6F77AFB2B
:10C89800FA888C4913461B0113449A01D21A8B1843
:10C8A800B3F805309BB243F001039BB2012118464F
:10C8B800F6F768FB97E0FA88824913461B01134490
:10C8C8009A01D21A8B18D3F8093001211846F6F7C5
:10C8D80093FBFA887B4913461B0113449A01D21A29
:10C8E8008B18B3F805309BB243F001039BB20121CA
:10C8F8001846F6F747FB76E0FA88724913461B019B
:10C9080013449A01D21A8B18D3F80930012118461A
:10C91800F6F772FBFA886B4913461B0113449A0118
:10C92800D21A8B18B3F805309BB243F001039BB2BF
:10C9380001211846F6F726FB55E0FA8861491346A7
:10C948001B0113449A01D21A8B18D3F8093001211C
:10C958001846F6F751FBFA885A4913461B01134447
:10C968009A01D21A8B18B3F805309BB243F0010331
:10C978009BB201211846F6F705FB34E0FA885149C5
:10C9880013461B0113449A01D21A8B18D3F80930A5
:10C9980001211846F6F730FBFA884A4913461B016D
:10C9A80013449A01D21A8B18B3F805309BB243F09E
:10C9B80001039BB201211846F6F7E4FAFA884149C7
:10C9C80013461B0113449A01D21A8B18B3F8073087
:10C9D8009BB243F001039BB201211846F6F7D2FA45
:10C9E80001E0002369E0FA88364913461B01134425
:10C9F8009A01D21A8B180833B3F809309BB23B81DD
:10CA08001823FB720223BB72FA882E4913461B01B6
:10CA180013449A01D21A8B180833D3F8053007F15A
:10CA2800080211461846F5F7BDFEFA88254913464F
:10CA38001B0113449A01D21A8B181033B3F807302C
:10CA48009BB23B810423FB72FA881E4913461B01E3
:10CA580013449A01D21A8B180833D3F80B3007F114
:10CA6800080211461846F5F79DFE3B6ADB8C9BB21F
:10CA7800DBB23B7300237B730023BB730123FB737F
:10CA880007F10C031846F5F755FA3B6AD3F801305D
:10CA980007F1100211461846F4F726FE3B6AD3F850
:10CAA800013001211846F4F799FF3B6A1B7843F0DF
:10CAB8000103DAB23B6A1A70002318462837BD46CC
:10CAC80080BD00BF24EE002080B58AB000AF0346C9
:10CAD8003960FB803B683B62FA8813461B011344AC
:10CAE8009A01D21A894B1344FB61FB6900221A7020
:10CAF800FB69002283F83420002283F83520FB6983
:10CB0800002283F84420FB69002283F84520FB6952
:10CB1800002283F846203B6A1A68FB69C3F8222082
:10CB2800FB69002283F82820002283F829203B6A29
:10CB3800D3F81D307B62FB69002283F82A2000228B
:10CB480083F82B20002283F82C20002283F82D2044
:10CB580018E0FB69D3F82A2013469B0013445B00B6
:10CB68001A46FB69C3F82A20FB69D3F82A307A6A87
:10CB780012781344A3F13002FB69C3F82A207B6AB8
:10CB880001337B627B6A1B782C2BE2D17B6A0133F1
:10CB98007B627B6A1A78FB6983F82F207B6A0233F1
:10CBA8007B627B6A1A78FB6983F82E207B6A0233E2
:10CBB8007B627B6A1A78FB6983F830207B6A0233D0
:10CBC8007B627B6A1B78342B08D1FB69002242F018
:10CBD800010283F82820002283F82920FB69D3F872
:10CBE8002A30FB60FB6993F83030322B02D00023E7
:10CBF8007B8203E04FF400537B8200BFFB6993F80C
:10CC08002E30372B0BD0FB6993F82F304E2B02D1E7
:10CC180000233B8206E04FF480533B8202E000236E
:10CC28003B8200BFFB6993F82F30452B04D04F2B74
:10CC380006D00023BB8207E04FF48063BB8203E089
:10CC48004FF4C063BB8200BFFB69DB69002B1AD0BD
:10CC5800FB695B8B9BB201211846F6F793F9FB69D8
:10CC68001B8C9BB23B811023FB720223BB72FB69B6
:10CC7800DB6907F1080211461846F5F793FDFB88B2
:10CC8800184600F095FA00233B830C23FB82FB69CE
:10CC9800D3F8013007F10C0211461846F4F724FDC9
:10CCA800FB69D3F8013001211846F4F797FEFB69B8
:10CCB800D3F80130012240F225511846F4F7DCFE82
:10CCC800FA88124913461B0113449A01D21A8B1889
:10CCD800D3F801309B8999B2FA880C4813461B0196
:10CCE80013449A01D21A8318D3F8013021F0400274
:10CCF80092B29A81FB691B7843F00103DAB2FB69AF
:10CD08001A70002318462837BD4680BD24EE00203F
:10CD180080B582B000AF0346FB80FA8835491346D8
:10CD28001B0113449A01D21A8B1844331B78002B29
:10CD38000CD1FA882F4913461B0113449A01D21AC1
:10CD48008B181B7803F00203002B4ED0FA88294970
:10CD580013461B0113449A01D21A8B1840335B887F
:10CD68009BB2002B26D1FA88224913461B01134493
:10CD78009A01D21A8B181B78FA8823F00203D8B2CA
:10CD88001C4913461B0113449A01D21A8B180246F8
:10CD98001A70FA88174913461B0113449A01D21ACC
:10CDA8008B18D3F80130002240F227711846F4F7A7
:10CDB80063FE17E0FA880F4913461B0113449A01D2
:10CDC800D21A8B1840335B889BB2FA88013B98B221
:10CDD800084913461B0113449A01D21A8B18403391
:10CDE80002465A8040F2FB1300E000231846083739
:10CDF800BD4680BD24EE002080B584B000AF034658
:10CE08003960FB80FB88002B42D0FB88042B3FD87D
:10CE18003B68FB60FB685B69312B18D1FA881F49B6
:10CE280013461B0113449A01D21A8B181033D86881
:10CE3800FA881A4913461B0113449A01D21A8B180F
:10CE480018331B899BB21946F5F796FE1EE0FB685E
:10CE58005B69302B18D1FA88104913461B0113441B
:10CE68009A01D21A8B181033D868FA880B491346DE
:10CE78001B0113449A01D21A8B1818331B899BB2D1
:10CE88001946F5F7BFFE01E0022302E0002300E0A7
:10CE9800032318461037BD4680BD00BF24EE00208E
:10CEA80080B588B000AF0346FB803123FB6107F1F2
:10CEB8000802FB8811461846FFF79EFF00BF20377F
:10CEC800BD4680BD80B584B000AF03460A46FB80EE
:10CED80013467B7101E035F08FFBFA884849134609
:10CEE8001B0113449A01D21A8B1844331B78312B37
:10CEF800F1D8FFF758F8FA88414913461B01134443
:10CF08009A01D21A8B1845331B78FB73FA883C496F
:10CF180013461B0113449A01D21A8B1828331B8815
:10CF28009BB2012B1BD1FA88354913461B011344C8
:10CF38009A01D21A8B1830339B889BB2FA88013336
:10CF480098B22F4913461B0113449A01D21A8B1821
:10CF5800303302469A80FB881846FFF7A1FFFA880B
:10CF6800274913461B0113449A01D21A8B184033E0
:10CF7800002262F037029A700022DA70FA88F97B90
:10CF88001F4813461B0113449A01D21A83180B44F5
:10CF980047337A791A70FB7B0133FB73FB7B194AA1
:10CFA800A2FB03121209322101FB02F29B1AFB7346
:10CFB800FA88134913461B0113449A01D21A8B1895
:10CFC80044331B78FA880133D8B20D4913461B0144
:10CFD80013449A01D21A8B18443302461A70FA88FD
:10CFE800074913461B0113449A01D21A8B1845337B
:10CFF800FA7B1A70FEF7D0FF00BF1037BD4680BD20
:10D0080024EE00201F85EB5180B485B000AF0346A5
:10D018003960FB80FA882D4913461B0113449A0195
:10D02800D21A8B1844331B78002B49D0FA88274929
:10D0380013461B0113449A01D21A8B1846331B78E6
:10D04800FB73FA88F97B214813461B0113449A01A4
:10D05800D21A83180B4447331A783B681A70FB7B43
:10D068000133FB73FB7B1A4AA2FB0312120932211C
:10D0780001FB02F29B1AFB73FA88144913461B0141
:10D0880013449A01D21A8B1844331B78FA88013B4F
:10D09800D8B20E4913461B0113449A01D21A8B18B1
:10D0A800443302461A70FA88084913461B01134490
:10D0B8009A01D21A8B184633FA7B1A70012300E0C2
:10D0C800002318461437BD4680BC704724EE002064
:10D0D8001F85EB5180B586B000AF03463960FB80F1
:10D0E8003B683B613B69D3F80930FB753B69D3F872
:10D0F8000530FB600023BB754FE0BB7DFA68134425
:10D108001A78FB8811461846FFF7DCFEBB7D013311
:10D11800BB75FB7D013BFB75FA88244913461B014F
:10D1280013449A01D21A8B181B7803F00203002BC0
:10D1380033D1FEF738FFFA881C4913461B01134404
:10D148009A01D21A8B18D3F801309B8999B2FA88C0
:10D15800164813461B0113449A01D21A8318D3F8B0
:10D16800013041F0800292B29A81FA880F49134641
:10D178001B0113449A01D21A8B181B78FA8843F0C2
:10D188000203D8B2094913461B0113449A01D21A63
:10D198008B1802461A70FEF7FFFEFB7D002BACD100
:10D1A800002318461837BD4680BD00BF24EE002076
:10D1B80080B588B000AF0346FB803023FB6107F1E0
:10D1C8000802FB8811461846FFF716FE00BF2037F5
:10D1D800BD4680BD80B586B000AF03463960FB8090
:10D1E8003B687B61FB88184600F068FA38613B6948
:10D1F800002B02D14FF4FA7344E03B691A787B693B
:10D208005A743B695A789B781B021343FB817B69EC
:10D2180000229A74FB8903F00103002B06D07B6976
:10D228009B7C43F00103DAB27B699A74FB8903F0B3
:10D238000203002B06D07B699B7C43F00203DAB221
:10D248007B699A74FB8903F00403002B06D07B6981
:10D258009B7C43F00403DAB27B699A74FB8903F080
:10D268000803002B0DD0FB8831331A4607490420E8
:10D2780035F0D8FA7B699B7C43F00803DAB27B6906
:10D288009A74002318461837BD4680BDDC3D050852
:10D2980080B500AF002000F01FF800BF80BD80B54A
:10D2A80000AF012000F018F800BF80BD80B500AFC6
:10D2B800022000F011F800BF80BD80B500AF032048
:10D2C80000F00AF800BF80BD80B500AF042000F070
:10D2D80003F800BF80BD000080B584B000AF0346EE
:10D2E800FB80FEF760FE0023FB60FB88032B23D046
:10D2F800FB88042B20D0FA88784913461B01134475
:10D308009A01D21A8B18D3F8013040F66A111846E0
:10D31800F4F7DAFC0346012B0ED1FA886F4913465D
:10D328001B0113449A01D21A8B18D3F8013040F626
:10D338006A111846F4F78EFDFA88684913461B01EE
:10D3480013449A01D21A8B18D3F801304FF458714C
:10D358001846F4F7B9FC0346012B0ED1FA885F4949
:10D3680013461B0113449A01D21A8B18D3F80130C3
:10D378004FF458711846F4F76DFDFA88574913466B
:10D388001B0113449A01D21A8B18D3F8013040F6C6
:10D3980046011846F4F798FC0346012B0ED1FA888B
:10D3A8004E4913461B0113449A01D21A8B18D3F81D
:10D3B800013040F646011846F4F74CFDFA88474913
:10D3C80013461B0113449A01D21A8B18D3F8013063
:10D3D8009B899BB203F080039BB2002B16D0FA887E
:10D3E8003E4913461B0113449A01D21A8B18D3F8ED
:10D3F80001301B889BB203F080039BB2002B05D041
:10D40800FB88184600F06CF80123FB60FA88334962
:10D4180013461B0113449A01D21A8B18D3F8013012
:10D428001B889BB203F020039BB2002B05D0FB881E
:10D43800184600F06DF90123FB60FA882749134666
:10D448001B0113449A01D21A8B18D3F801301B8898
:10D458009BB203F01F039BB2002B38D0FA881F49F8
:10D4680013461B0113449A01D21A8B18D3F80130C2
:10D478001B889BB203F00103002B26D015E0FA8825
:10D48800164913461B0113449A01D21A8B18D3F874
:10D4980001301B88FA88114913461B0113449A016D
:10D4A800D21A8B18D3F801309B88FA880B49134697
:10D4B8001B0113449A01D21A8B18D3F801301B8828
:10D4C8009BB203F00103002BD9D10123FB60FB6859
:10D4D800FEF762FD00BF1037BD4680BD24EE002078
:10D4E80080B584B000AF0346FB8007F10F02FB88CC
:10D4F80011461846FFF788FD0346002B30D1FA88FD
:10D508002B4913461B0113449A01D21A8B181B7816
:10D51800FA8823F00203D8B2254913461B011344A5
:10D528009A01D21A8B1802461A70FA8820491346B3
:10D538001B0113449A01D21A8B18D3F801309B8926
:10D5480099B2FA881A4813461B0113449A01D21A51
:10D558008318D3F8013021F0800292B29A8123E037
:10D56800FA88134913461B0113449A01D21A8B18DF
:10D57800D3F80130FA7B11461846F4F733FBFA88E2
:10D588000B4913461B0113449A01D21A8B184033D6
:10D59800002262F037029A700022DA70FB88FA7B68
:10D5A80011461846FDF770FE00BF1037BD4680BD16
:10D5B80024EE002080B500AF0B4600E001331A7856
:10D5C8000A2AFBD01A780D2AF8D01A78002A03D034
:10D5D8001946042035F026F900BF80BD80B582B019
:10D5E80000AF786039607B68002B02DD7B68042B14
:10D5F80001DD032320E012497A6813461B01134416
:10D608009A01D21A8B1803F58563D3F80330002BDF
:10D6180004D04FF461710B48FDF776F93968084872
:10D628007A6813461B0113449A01D21A831803F52A
:10D638008563C3F80310002318460837BD4680BD2C
:10D6480024EE0020F83D050880B582B000AF786070
:10D658007B68002B02DD7B68042B01DD032325E0BA
:10D6680014497A6813461B0113449A01D21A8B187D
:10D6780003F58563D3F80330002B04D140F28E31D3
:10D688000D48FDF741F90B497A6813461B0113440D
:10D698009A01D21A8B1803F585630022DA700022EA
:10D6A8001A7100225A7100229A710023184608370D
:10D6B800BD4680BD24EE0020F83D050880B584B045
:10D6C80000AF78607A6813461B0113449A01D21A96
:10D6D80002F57E730C4A134407331846FDF700FB26
:10D6E800F8607B68002B09D1FB68002B03D0074B3F
:10D6F80001221A6002E0054B63221A60FB68184693
:10D708001037BD4680BD00BF24EE0020B453002072
:10D7180080B588B002AF0346FB80FA8813461B0128
:10D7280013449A01D21A484B13447B617B69D3F89E
:10D7380001301B889BB2A7F809307B69D3F8013008
:10D748001846F4F78DFA0346DBB23B727B6903F2A5
:10D75800FF333B613D4B1B68002B0ED13B695B6A75
:10D768001B68FB60FA883B7A1946FB6800930B46F6
:10D778003749022035F056F859E07B6993F82E3086
:10D78800372B04D13B7A03F07F03DBB23B72FB8873
:10D79800002B1AD07B691B8D9BB2012B15D17B699D
:10D7A8009B8E9BB2002B10D07B699B8E9BB2013B5A
:10D7B8009AB27B699A867B699B8E9BB2002B33D188
:10D7C800FB881846FFF7F4FC2EE03B695B6A1A6891
:10D7D8003B699B689A421DDA3B695B6A9A683B69B8
:10D7E8005B6A1B6819460B465B000B4413441A46D8
:10D7F80007F1080319889B78118093703B695B6A6D
:10D808001A6801321A60FB883A7A11461846FDF701
:10D8180003FD0CE0FB88002B08D0FA883B7A0D4901
:10D82800022034F0FFFF02E000BF00E000BF7B6988
:10D83800D3F8013040F225511846F4F70BFB00BF2E
:10D848001837BD4680BD00BF24EE0020B05300202D
:10D85800683E0508903E050880B582B000AF0346D3
:10D868003960FB80FB88092B1ADC002B37DD013B74
:10D87800082B34D801A252F823F000BFCFD80008F3
:10D88800D7D80008DFD80008E7D80008E7D800088C
:10D89800E7D80008E7D80008B7D80008C3D80008B8
:10D8A800B3F57B7F1BD1386800F020F819E03868A1
:10D8B80000F028F803469BB214E0386800F04AF8F4
:10D8C80003469BB20EE0386800F0A2F809E0386819
:10D8D80000F036F905E0386800F074F901E001233A
:10D8E80000E0002318460837BD4680BD80B500AF6C
:10D8F8001020F4F7C9FB0220F4F79CFB002318461C
:10D9080080BD000080B485B000AF78607B68FB60A4
:10D91800FB681B889BB20B2B06D8FB681B889BB245
:10D92800DB000B4A134400E00023BB60BB68002BFC
:10D9380002D140F2BD2305E0BB681A68FB68C3F852
:10D948000220002318461437BD4680BC704700BF2C
:10D95800AC3E050880B588B000AF78607B683B6155
:10D968003B691B889BB20B2B06D83B691B889BB273
:10D97800DB00264A134400E00023FB60FB68002B11
:10D9880002D140F2BD233DE0FB681B68FB613B69A7
:10D99800D3F80230BB60B8683BF074F90346013332
:10D9A8007B617B6903F00103002B02D07B690133A3
:10D9B8007B610023BB610CE0BB695A1CBA61FA6841
:10D9C8005268934202D94FF464731BE0FB69023337
:10D9D800FB61FB691B884FF6FF729342ECD1BA6971
:10D9E8007B691A44FB685B689A4202D94FF46473F6
:10D9F80008E07B695B087B617A69B968F86900F0BF
:10DA08005AF8034618462037BD4680BDAC3E050887
:10DA180080B586B000AF78607B687B617B695B8886
:10DA28009BB23B617B695B68FB607B691B889BB22F
:10DA38000B2B06D87B691B889BB2DB000B4A13446F
:10DA480000E00023BB60BB68002B02D140F2BD237D
:10DA580007E0BB681B683A691946F868F2F7ACFC3E
:10DA6800002318461837BD4680BD00BFAC3E0508E8
:10DA780080B584B000AF78600B467B800023FB60E4
:10DA880011E07B687A8811461846F4F727FC0346AC
:10DA9800FB727B681B887A889A4201D1FB7A06E080
:10DAA800FB680133FB60FB68032BEADD02231846A1
:10DAB8001037BD4680BD80B588B000AFF860B9604A
:10DAC8007A6000237B610023BB6100F0E7F8352012
:10DAD800F4F7F4FC0423FB7723E07B68013B7B60CD
:10DAE800BB681B887B827B8A1946F868FFF7C0FFF2
:10DAF8000346FB77FB681B887A8A9A4204D07B69C5
:10DB0800002B01D101237B61BB680233BB60FB7F23
:10DB1800042B03D04FF43173BB6109E0FB68023377
:10DB2800FB607B68002B02D0FB7F042BD5D000BFA5
:10DB380000F0BAF8BB6918462037BD4680BD000022
:10DB480080B588B000AF78607B68FB61FB691B8893
:10DB58009BB20B2B06D8FB691B889BB2DB00164ACD
:10DB6800134400E00023BB61BB69002B02D140F2E3
:10DB7800BD231CE0FB695B889BB25B089BB2013349
:10DB88007B61FB695B683B61BB691B68FB607A6909
:10DB98003969F868FFF78FFFB860BB68002B04D0BD
:10DBA800FA68064906483AF093FDBB689BB21846E6
:10DBB8002037BD4680BD00BFAC3E05080C3F0508B8
:10DBC8009446002080B58AB000AF78607B68BB615E
:10DBD800BB691B889BB20B2B06D8BB691B889BB201
:10DBE800DB002D4A134400E000237B617B69002B96
:10DBF80002D140F2BD234AE07B695B683B613B6927
:10DC0800DB0AFB603520F4F759FC3B695B08FB61D4
:10DC18003B6903F00103002B02D0FB690133FB6170
:10DC280000237B627B691B683B620BE03B6A1B88B5
:10DC38004FF6FF7293420BD17B6A01337B623B6ADA
:10DC480002333B627B6AFA699A42EFD800231EE0EE
:10DC580000BF00F023F800237B620FE07B6ADB0241
:10DC68001A467B691B681344BB60B868F4F75CFA12
:10DC78000346042B07D17B6A01337B627B6AFA680F
:10DC88009A42EBD800E000BF00F00EF800231846D7
:10DC98002837BD4680BD00BFAC3E050880B500AF43
:10DCA800F4F716FA00BF80BD80B500AFF4F728FA84
:10DCB80000BF80BD80B400AF72B600BFBD4680BC57
:10DCC800704780B400AFBFF34F8F00BFBD4680BC24
:10DCD8007047000080B500AF054BDB6803F4E062D5
:10DCE8000349044B1343CB60FFF7EBFF00BFFDE78D
:10DCF80000ED00E00400FA0580B400AF084B1B6893
:10DD08000133074A1360074B1B68002B04D0054BEF
:10DD18001B68013B034A136000BFBD4680BC7047C7
:10DD2800C0530020C453002080B500AF0D2000F080
:10DD380027F800BF80BD80B500AFFEF7DDF800BF53
:10DD480080BD80B500AFFFF7A3FA00BF80BD80B5E6
:10DD580000AFFFF7A4FA00BF80BD80B500AFFFF7A2
:10DD6800A5FA00BF80BD80B500AFFFF7A6FA00BFD7
:10DD780080BD80B500AFFFF7A7FA00BF80BD0000E7
:10DD880080B584B000AF0346FB71FFF793FF114ADB
:10DD9800FB791370FB791A460F4910483AF098FC42
:10DDA8000E490020FFF706FC0D4BFB6000BFFB6827
:10DDB8005A1EFA60002BFAD100F074F8084BFB6089
:10DDC80000BFFB685A1EFA60002BFAD100F06AF80F
:10DDD800EAE700BFBC530020443F050810030120B8
:10DDE800FFFF040080B500AFFFF764FFFFF772FF85
:10DDF80000BFFDE780B483B000AF78600A4B1A8893
:10DE08007B681A80094B1A887B685A80084B1A6805
:10DE18007B685A60074B1A687B689A6000BF0C37AA
:10DE2800BD4680BC704700BFE8F7FF1FEAF7FF1F39
:10DE3800ECF7FF1FF0F7FF1F80B400AF024B1B8801
:10DE48001846BD4680BC704700F8FF1F80B500AF7C
:10DE5800F4F73EF9F4F7D8F90120F4F79FFAF4F74C
:10DE68004FF900BF80BD000080B582B000AF01212E
:10DE78001120F5F787F80823BB801023FB710223D4
:10DE8800BB713B1D19460648F4F78CFC012208219A
:10DE98000348F4F7FDFE00BF0837BD4680BD00BF4C
:10DEA8000010014080B500AF114B1B88002B17D123
:10DEB80008211048F4F7DAFD0346002B08D10821A1
:10DEC8000C48F4F759FE0A4B4FF47A721A800DE0A9
:10DED80008210848F4F796FE054B0A221A8005E047
:10DEE800034B1B88013B9AB2014B1A8000BF80BDCF
:10DEF800C85300200010014080B59EB000AFC7E9AC
:10DF080002017A60FB7097F88030002B13D1FA7801
:10DF180007F11003302118463AF0AAFCFB781A469C
:10DF2800302178683AF0A4FCFB7878333B4400222F
:10DF380003F8682C16E0FB7801331A4607F1100342
:10DF4800302118463AF094FCFB7801331A46302108
:10DF580078683AF08DFCFB78013378333B44002233
:10DF680003F8682C002387F87530002387F877308A
:10DF780026E0D7E902014FF00A024FF00003F3F759
:10DF880019F997F87510481C87F875000846324942
:10DF98008B181A7800F178033B4403F8682C97F83B
:10DFA8007730013387F87730D7E902014FF00A025A
:10DFB8004FF00003F3F7FEF802460B46C7E90223C9
:10DFC800D7E90223134304D097F87720FB789A42C5
:10DFD800CFD3002387F87630002387F877302CE0FA
:10DFE800FA7897F87730D31A013B78333B4413F823
:10DFF800683C87F87430FA7897F87730D21A97F82F
:10E0080080309A4209D197F876305A1C87F87620E2
:10E018001A467B6813442E221A7097F876305A1CD9
:10E0280087F876201A467B68134497F874201A708C
:10E0380097F87730013387F8773097F87720FB78AF
:10E048009A42CDD397F876307A68134400221A7032
:10E0580000BF7837BD4680BD843F050880B586B0CF
:10E0680002AFC7E902017A603B60BB69DAB2FB69BB
:10E07800DBB20A210191009313467A68D7E90201BD
:10E08800FFF73AFF7B6818461037BD4680BD80B55C
:10E0980086B000AFF860B9601346FB80FB68002BC0
:10E0A80002D101233B8204E0FB68012B16D1022335
:10E0B8003B82FB887B82BB687B6107F110031946B2
:10E0C8000320FFF7C9FBFB887B82BB687B6107F1F4
:10E0D800100319460220FFF7BFFB00E000BF183706
:10E0E800BD4680BD80B588B000AFF860B960134602
:10E0F800FB80FB68002B02D10123BB8208E0FB6890
:10E10800012B02D10223BB8202E04FF6FF731DE010
:10E11800FB88FB82BB68BB6107F114031946012029
:10E12800FFF79AFB0023FB830AE0FB8BBA681344D2
:10E138001B78FF2B01D0002308E0FB8B0133FB8306
:10E14800FA8BFB889A42F0D34FF6FF7318462037B4
:10E15800BD4680BD80B483B000AF786000BF0C3787
:10E16800BD4680BC7047000080B483B000AF034652
:10E178003960FB711346BB71FB79A3F1C8020B49E7
:10E1880013469B0013440B443A681A60FB79A3F1C9
:10E19800C802064913469B0013440B440433BA795A
:10E1A8001A7000BF0C37BD4680BC7047D0530020A2
:10E1B80080B582B000AFC8237B6009E07B68DBB222
:10E1C800002225491846FFF7CFFF7B6801337B60A3
:10E1D8007B68E52BF2DD01222049D220FFF7C4FF3E
:10E1E80003221F49CC20FFF7BFFF04221D49C92085
:10E1F800FFF7BAFF05221C49D020FFF7B5FF06221A
:10E208001A49D420FFF7B0FF07221949D720FFF792
:10E21800ABFF09221749D520FFF7A6FF0A221649A6
:10E22800D320FFF7A1FF0B221449E120FFF79CFF41
:10E238000C221349D820FFF797FF0D221149DB2044
:10E24800FFF792FF0F221049DD20FFF78DFF00BF77
:10E258000837BD4680BD00BF79000108C9CA030858
:10E2680069F8010869760208550A010859ED02089B
:10E27800E54B040881890308996D0108B76D010809
:10E2880009C90108CD2A0308C556030880B586B018
:10E2980000AF78603960174B1B68002B04D1FFF77B
:10E2A80087FF144B01221A603B687B617B695B69BD
:10E2B8003B613B69DC2B17D03B69D92B14D03B69F8
:10E2C800C72B11DD3B69E52B0EDC3B69C83BFB60C6
:10E2D8000949FA6813469B0013440B441B683968C4
:10E2E80078689847034601E04FF4167318461837C4
:10E2F800BD4680BD68540020D053002080B58AB048
:10E3080000AF7860396007F10C03042279680120B6
:10E31800F7F79CFB0346002B04D040F209229342F6
:10E3280007D009E07A7F3B681A704FF0FF337B62B1
:10E3380005E001237B6202E000237B6200BF7B6A69
:10E3480018462837BD4680BD80B588B000AFF86054
:10E35800B9607A6033F00CFEF861FA697B6813449F
:10E36800BB61B968F868FFF7C9FF78617B69B3F1E9
:10E37800FF3F01D1002315E033F0FAFD38613A6917
:10E38800FB699A4203D1012033F0B6FD01E03B69F5
:10E39800FB617B69012B03D03A69BB699A42E0D3E0
:10E3A8004FF4FC7318462037BD4680BD80B586B053
:10E3B80000AFF860B9607A6007F113037A6819460C
:10E3C800F868FFF7C1FF78617B69002B03D1FB7CFC
:10E3D8001A46BB681A607B6918461837BD4680BD67
:10E3E80080B586B000AFF860B9607A60BB683B6101
:10E3F80000237B613B69442B48D03B69442BC0F226
:10E408008E803B69B3F57C7F00F389803B69B3F567
:10E418007A7F40F384803B69A3F2E933072B7ED8E7
:10E4280001A252F823F000BF5DE40008B3E400083D
:10E43800BDE4000851E4000827E50008D9E4000815
:10E44800F5E4000879E400087968F86800F074F8E1
:10E45800786167E03649FA681346DB009B1A5B006F
:10E468000B44D3F80A307968184601F031FA59E0BC
:10E478002F49FA681346DB009B1A5B000B44D3F85C
:10E488000A307968184601F085FA4BE02849FA689D
:10E498001346DB009B1A5B000B44D3F80A307968FB
:10E4A800184601F055FA78613CE07968F86801F09F
:10E4B80069FB37E01E49FA681346DB009B1A5B00CC
:10E4C8000B44D3F80A307968184601F08BFA29E032
:10E4D8001749FA681346DB009B1A5B000B44D3F814
:10E4E8000A307968184601F0B3FC1BE0F868104957
:10E4F800FA681346DB009B1A5B000B44D3F80A301A
:10E5080044F2404202FB03F303F51473094A13442F
:10E5180003334FF461621946FFF7B9FD02E00123A6
:10E528007B6100BF7B6918461837BD4680BD00BFB8
:10E53800A8ED00206C540020B0B58EB002AF786012
:10E5480039603B683B623B6A5B683A6A9268019251
:10E5580000937B68AF4AB0494FF4806034F062F9A9
:10E56800AE497A681346DB009B1A5B000B44D3F86C
:10E578000A3044F2404202FB03F3A94A1344FB6108
:10E58800A6497A681346DB009B1A5B000B44D3F854
:10E598000A20FB691A60FB697A685A603B6A9B68C3
:10E5A8001A46FB69C3F8B9203B6A5A68FB69C3F885
:10E5B800B520FB6903F583530333FA69C2F8A93020
:10E5C800FB6903F25322FB69C3F8AD20FB69002203
:10E5D80083F8B120002283F8B220002283F8B32008
:10E5E800002283F8B420FB699D334FF47A711846F2
:10E5F80032F0FEFFFB6903F29313FB620023BB6258
:10E6080020E0FB6A00221A7100225A7100229A71D6
:10E618000022DA71FB6A00221A7000225A70002266
:10E628009A700022DA70FB6A00221A7200225A726B
:10E6380000229A720022DA72FB6A0C33FB62BB6A10
:10E648000133BB62BB6A0F2BDBDDFB6900221A7248
:10E6580000225A7200229A720022DA72FB690022A2
:10E668001A7300225A7300229A730022DA73FB6924
:10E6780000221A7400225A7400229A740022DA7452
:10E688007868FB6903F253234FF461621946FFF778
:10E6980029FD0346002B08D0FB6903F253234FF4EE
:10E6A8006162002118463AF0E3F80523BB615D4B2F
:10E6B8001B68002B07D0574A5B494FF4806034F041
:10E6C800B1F80023E7E2534A58494FF4806034F028
:10E6D800A9F8F9694FF47B7001F066F8B861BB6975
:10E6E800002B32D005237B6164233B617B69494A57
:10E6F8004F494FF4806034F095F87B694FF47A7293
:10E7080002FB03F37B62474B1B68002B07D0414A8F
:10E7180045494FF4806034F085F80023BBE23B693B
:10E72800184633F0E9FB7A6A3B69D31A7B623B49A6
:10E738007A681346DB009B1A5B000B449B889BB2EC
:10E74800022B02D17B6A002BDDDC364B1B68002BC9
:10E7580007D0304A34494FF4806034F063F800231E
:10E7680099E22E497A681346DB009B1A5B000B443A
:10E778009B889BB2022B02D1BB69002B97D12749FA
:10E788007A681346DB009B1A5B000B449B889BB29C
:10E79800022B0AD07868FB6903F253234FF46162B5
:10E7A8001946FFF774FC002375E240F24D23194A1D
:10E7B80020494FF4806034F035F8F9694FF47B70E4
:10E7C80001F03EF8174B1B68002B07D0114A164979
:10E7D8004FF4806034F026F800235CE2FB690022E5
:10E7E80042F0100283F89920002283F89A20002230
:10E7F80083F89B20002283F89C200A4B1B68002B7F
:10E808001AD0044A08494FF4806034F00BF800230A
:10E8180041E200BF7846050840400508A8ED002001
:10E828006C540020CC53002074400508984005081B
:10E83800C840050804410508F86900F0F9FBF860CC
:10E84800FB68002B40F06781FB691833B94A1C4606
:10E8580015460FCD20606160A260E360FB6900226D
:10E8680042F0010283F89520002283F896200022C6
:10E8780083F89720002283F89820FB69002242F051
:10E88800030283F89520002283F89620002283F85B
:10E898009720002283F89820A74B1B68002B07D0ED
:10E8A800A64AA7494FF4806033F0BCFF0023F2E189
:10E8B800F86900F00DFCF8609F4B1B68002B07D02F
:10E8C8009E4A9F494FF4806033F0ACFF0023E2E199
:10E8D800FB68002B40F0D380974B1B68002B07D0B8
:10E8E800964A97494FF4806033F09CFF0023D2E1A9
:10E8F800F969172000F0A4FF8F4B1B68002B07D085
:10E908008E4A8F494FF4806033F08CFF0023C2E1B8
:10E91800FB69D3F8C120F96913465B0013449B00D7
:10E928000B4403F5C873D3F80730FA69D2F8C1204D
:10E9380023F04001F86913465B0013449B0003442D
:10E9480003F5C873C3F80710FB69D3F8C120F96948
:10E9580013465B0013449B000B4403F5C873D3F8BC
:10E96800073003F08003002B67D1FB69002242F0D7
:10E97800040283F89520002283F89620002283F869
:10E988009720002283F898206B4B1B68002B07D038
:10E998006A4A6B494FF4806033F044FF00237AE100
:10E9A800F86900F043FE644B1B68002B07D0634AEC
:10E9B80063494FF4806033F035FF00236BE1FB6956
:10E9C800D3F8C120F96913465B0013449B000B443C
:10E9D80003F5C873D3F80730FA69D2F8C12043F0B9
:10E9E8008001F86913465B0013449B00034403F558
:10E9F800C873C3F80710FB69002242F0050283F8C8
:10EA08009520002283F89620002283F89720002280
:10EA180083F89820F969172000F012FF0346002BAD
:10EA28007BD1454B1B68002B07D0444A44494FF41F
:10EA3800806033F0F7FE00232DE1FB69002242F0ED
:10EA4800060283F89520002283F89620002283F896
:10EA58009720002283F89820F86900F0CDFBFB6925
:10EA6800002242F0070283F89520002283F89620BE
:10EA7800002283F89720002283F898204EE02E4B3E
:10EA88001B68002B07D02D4A2D494FF4806033F0C6
:10EA9800C9FE0023FFE0FB69D3F8C120F9691346DA
:10EAA8005B0013449B000B4403F5C873D3F807308D
:10EAB80003F04003002B2ED1FB69D3F8C120F9697C
:10EAC80013465B0013449B000B4403F5C873D3F84B
:10EAD8000730FA69D2F8C12043F04001F8691346BB
:10EAE8005B0013449B00034403F5C873C3F8071085
:10EAF800FB69002262F06F021A75002242F00102DF
:10EB08005A7500229A750022DA75FA690D49F86873
:10EB180000F022FE02E000BF00E000BF064B1B68C9
:10EB2800002B11D0054A06494FF4806033F07AFE75
:10EB38000023B0E024410508CC530020784605089E
:10EB48007440050834410508FB691833544A1C46CB
:10EB5800134607CB20606160A2601A889B78A28167
:10EB6800A373FB69002242F0010283F8952000227A
:10EB780083F89620002283F89720002283F89820B3
:10EB8800FB69002242F0020283F89520002283F8F4
:10EB98009620002283F89720002283F89820FB69AA
:10EBA8009D33184632F096FD0346002B40D03D4B6E
:10EBB8001B68002B07D03C4A3C494FF4806033F077
:10EBC80031FE002367E0FB69002242F0030283F86C
:10EBD8009520002283F89620002283F897200022AF
:10EBE80083F89820FB699D334FF47A71184632F008
:10EBF800FFFCFB69002242F0040283F89520002202
:10EC080083F89620002283F89720002283F8982022
:10EC1800F9690E2000F0C8FD224B1B68002B07D0B5
:10EC2800214A22494FF4806033F0FCFD002332E092
:10EC3800FB69002242F00A0283F89520002283F83B
:10EC48009620002283F89720002283F89820F6F770
:10EC5800ABFF144B1B68002B07D0134A13494FF422
:10EC6800806033F0DFFD002315E011497A68134610
:10EC7800DB009B1A5B000B449B889BB2022B3FF482
:10EC8800BCAD7868FB6903F253234FF461621946FF
:10EC9800FFF7FDF9002318463037BD46B0BD00BF69
:10ECA80044410508CC5300207846050874400508FF
:10ECB800A8ED002080B584B000AF78600023FB6029
:10ECC8007B685A680D491346DB009B1A5B000B44AE
:10ECD8009B889BB2032B0CD17B685B6818467B68CA
:10ECE80003F253234FF461621946FFF7D0F9012369
:10ECF800FB60FB6818461037BD4680BDA8ED0020B4
:10ED080080B582B000AF786079680F2000F04CFDC4
:10ED18007B68D3F8D530012B04D07B68D3F8D53085
:10ED2800022B2AD17B6803F253207B68D3F8DD10CD
:10ED38007B68D3F8D9301A46F1F73EFB7B68D3F8E5
:10ED4800993003F08003002B04D07B68D3F8D530CA
:10ED5800022B12D17B68D3F8993043F080027B688C
:10ED6800C3F899207B685B6818467B6803F25323D5
:10ED78004FF461621946FFF78AF900BF0837BD46AC
:10ED880080BD80B584B000AF78607B68D3F89930D7
:10ED980023F010027B68C3F899207B681B69002B5D
:10EDA80054D10023FB604DE07B68DB685A1C7B680C
:10EDB800DA607B68DB680F2B08DD7B6800221A733A
:10EDC80000225A7300229A730022DA737B68DA6889
:10EDD8007B68C3F8C1207B68002283F86F2100227A
:10EDE80083F87021002283F87121002283F87221B0
:10EDF8007968012000F024FD0346002B01D002238E
:10EE08003FE07B68D3F86F3103F00103002B13D088
:10EE18007B68D3F86F3103F02003002B0FD07B6899
:10EE2800002242F010021A7400225A7400229A74C6
:10EE38000022DA74012324E0786800F082F8FB6885
:10EE48000133FB60FB680F2BAEDD17E07B681B69A5
:10EE5800102B03DC7B681B69002B0ADA7B68002215
:10EE680042F010021A7400225A7400229A74002286
:10EE7800DA747B681B695A1E7B681A61F6F794FE80
:10EE8800002318461037BD4680BD80B584B000AF5A
:10EE980078607B68D3F8993043F010027B68C3F838
:10EEA80099200023FB6042E07B689B685A1C7B68C2
:10EEB8009A607B689B680F2B08DD7B6800221A72BA
:10EEC80000225A7200229A720022DA727B689A68CB
:10EED8007B68C3F8C1207B68002283F86F21002279
:10EEE80083F87021002283F87121002283F87221AF
:10EEF8007968012000F0A4FC0346002B01D002230E
:10EF08001BE07B68D3F86F3103F00103002B08D0B6
:10EF18007B68D3F86F3103F02003002B04D1012361
:10EF28000BE0786800F00DF8FB680133FB60FB68C4
:10EF38000F2BB9DDF6F738FE002318461037BD460B
:10EF480080BD80B584B000AF78600023FB607B682B
:10EF5800D3F86F31022B43D17B68D3F8C12079688D
:10EF680013465B0013449B000B4403F5C87300224F
:10EF7800DA7000221A7100225A7100229A717B6895
:10EF8800D3F8C120796813465B0013449B000B44F7
:10EF980003F5C873D3F807307A68D2F8C12003F0B4
:10EFA8004001786813465B0013449B00034403F553
:10EFB800C873C3F807107B68002242F0020283F886
:10EFC8009520002283F89620002283F897200022BB
:10EFD80083F8982079680D2000F0E6FB0123FB6098
:10EFE800FB6818461037BD4680BD80B584B000AFB9
:10EFF80078607B68002242F0030283F895200022A3
:10F0080083F89620002283F89720002283F898201E
:10F018007B68D3F86F31FB607968032000F0C4FB8C
:10F028007B68FA68C3F86F2100BF1037BD4680BD02
:10F0380080B584B000AF78600023FB737B68BB6049
:10F048001CE0B868FFF736FE0346002B01D000230A
:10F0580039E0B868FFF754FEBB68D3F8993003F07D
:10F068001003002B05D0B868FFF78BFE0346FB732F
:10F0780004E0B868FFF709FF0346FB73FB7B002B2E
:10F08800DFD0FB7B022B02D140F25F231BE0BB6881
:10F09800002242F0010283F89520002283F896208E
:10F0A800002283F89720002283F89820B868FFF799
:10F0B80048FF0346002B02D040F25F2303E0B86804
:10F0C800FFF793FF002318461037BD4680BD0000A8
:10F0D800B0B584B000AF78607B68FB60FB68002245
:10F0E80042F02C021A75002242F001025A750022E1
:10F0F8009A750022DA75FB6818333D4A1C46154696
:10F108000FCD20606160A260E360F968042000F020
:10F118004BFBB860FB68D3F86F31002B4ED0FB680F
:10F12800D3F86F3140F2612293420BD0FB68D3F8D9
:10F138006F3140F25F22934204D0FA682D49B868D3
:10F1480000F00AFB7968212000F07AFB0346002BC7
:10F1580002D040F25F2346E0FB68D3F8C120F9688B
:10F1680013465B0013449B000B4403F5C873D3F8A4
:10F178000730FA68D2F8C12003F04001F868134656
:10F188005B0013449B00034403F5C873C3F80710DE
:10F19800FB68D3F8C120F96813465B0013449B0051
:10F1A8000B4403F5C8730022DA7000221A7100229A
:10F1B8005A7100229A7140F25F2314E0FB68D3F879
:10F1C800C120FB68D3F8D110F86813465B001344DC
:10F1D8009B00034403F5C873C3F80310F9680220C1
:10F1E80000F02EFB034618461037BD46B0BD00BFE1
:10F1F800544105086441050880B584B000AF7860C3
:10F208007B68FB6079680B2000F01AFB0346002B33
:10F2180008D1FB68D3F86F31002B03D1786800F070
:10F228009FF89AE079680D2000F00AFB0346002B4E
:10F2380008D1FB68D3F86F31002B03D1786800F050
:10F24800D7F88AE079680E2000F0FAFA0346002B16
:10F2580008D1FB68D3F86F31002B03D1786800F030
:10F2680047F97AE079680F2000F0EAFA0346002BA4
:10F2780008D1FB68D3F86F31002B03D1786800F010
:10F28800ADF86AE07968102000F0DAFA0346002B3E
:10F298001CD1FB68D3F86F31002B17D1FB68D3F86A
:10F2A800C120F96813465B0013449B000B4403F527
:10F2B800C873D3F8033003F00203002B02D0786838
:10F2C80000F0B4F9786800F0D3F846E0FB68D3F8AA
:10F2D800C120F96813465B0013449B000B4403F5F7
:10F2E800C873D3F8033003F00203002B12D07968F7
:10F2F800112000F0A5FA0346002B2BD1FB68D3F8A8
:10F308006F31002B02D1786800F03AF9786800F084
:10F318008DF91FE079680A2000F092FA0346002B65
:10F3280008D1FB68D3F86F31002B03D1786800F05F
:10F3380027F912E079680C2000F082FA0346002BC6
:10F348000AD1FB68D3F86F31002B05D1786800F03B
:10F35800BFF901E000BF00E000BF1037BD4680BD27
:10F3680090B585B000AF78607B68FB60FB680022D1
:10F3780042F064021A7500225A7500229A7500221A
:10F38800DA75FB681833134A1C46134607CB20600E
:10F398006160A2601B7823737968052000F004FA85
:10F3A800B860BB68002B05D0FA680B49B86800F054
:10F3B800D3F90BE0F968142000F042FAFB68D3F89F
:10F3C800993043F00102FB68C3F8992000BF143755
:10F3D800BD4690BD704105088041050880B483B0E2
:10F3E80000AF786000BF0C37BD4680BC7047000096
:10F3F800B0B584B000AF7860194A1A494FF48060FC
:10F4080033F010FA7B68FB60FB68002262F0370279
:10F418001A7500225A7500229A750022DA75FB685F
:10F428001833114A1C4615460FCD20606160A26052
:10F43800E3607968072000F0B7F9B860BB68002B73
:10F4480005D0FA680949B86800F086F903E0F96858
:10F45800152000F0F5F900BF1037BD46B0BD00BF5C
:10F468008C4605088C41050898410508A8410508FF
:10F47800B0B584B000AF78607B68FB60FB680022A1
:10F4880062F036021A7500225A7500229A75002217
:10F49800DA75FB681833144A1D4614460FCC2860E9
:10F4A8006960AA60EB6023882B827968082000F0E5
:10F4B8007BF9B860BB68002B05D0FA680B49B868BF
:10F4C80000F04AF90BE0FB68D3F8993023F0010209
:10F4D800FB68C3F89920F9681F2000F0B1F900BF54
:10F4E8001037BD46B0BD00BFB4410508C841050886
:10F4F800B0B584B000AF78607B68FB60FB68002221
:10F5080062F035021A7500225A7500229A75002297
:10F51800DA75FB681833184A1D4614460FCC286064
:10F528006960AA60EB6020682861FB68012283F8A3
:10F538000921F968322000F083F90346002B18D11D
:10F548007968092000F030F9B860BB6840F262229F
:10F5580093420DD0BB68002B04D1F968292000F034
:10F568006FF906E0FA680549B86800F0F5F800E0B8
:10F5780000BF1037BD46B0BDD4410508E8410508B5
:10F58800B0B586B000AF78607B687B617B6900228C
:10F5980062F034021A7500225A7500229A75002208
:10F5A800DA757B6918331F4A1D4614460FCC28604C
:10F5B8006960AA60EB60206828617969342000F0EE
:10F5C8003FF90346002B2AD179680A2000F0ECF8AD
:10F5D80038613B6940F25E22934204D17969202068
:10F5E80000F02EF908E03B69002B05D07A690E4936
:10F5F800386900F0B1F812E07B69D3F86F31002B5D
:10F608000CD17969182000F01BF9F860FB68002B11
:10F6180005D17969202000F013F900E000BF183700
:10F62800BD46B0BDF441050808420508B0B584B030
:10F6380000AF78607B68FB60FB68002262F03302F1
:10F648001A7500225A7500229A750022DA75FB682D
:10F6580018331C4A1D4614460FCC28606960AA60FE
:10F66800EB6003CC2861696123782B76FB68012263
:10F6780083F8092179680B2000F096F8B860BB6818
:10F68800002B04D0FA681049B86800F065F8F968EA
:10F69800282000F0D5F80346002B0FD1FB68D3F8DB
:10F6A800C53003F08003002B08D0FB68D3F86F3116
:10F6B800FA680649184600F04FF800BF00BF103737
:10F6C800BD46B0BD18420508344205084442050845
:10F6D80090B585B000AF78607B68FB60FB6800225E
:10F6E80062F032021A7500225A7500229A750022B9
:10F6F800DA75FB681833164A1C46134607CB206098
:10F708006160A2601B88A381F968352000F098F831
:10F718000346002B18D179680C2000F045F8B86032
:10F72800BB6840F2622293420DD0BB68002B05D023
:10F73800FA680849B86800F00FF805E0F96822206F
:10F7480000F07EF800E000BF1437BD4690BD00BF52
:10F75800544205086442050880B58CB000AFF860D3
:10F76800B9607A607B68FB620E4B7B615023BB619A
:10F77800FB6AD3F8C1305A1CFB6A1B681B0113448F
:10F78800FB61FB6A5B697B62FB683B62BB68BB62CF
:10F7980007F1140319462A20F4F76AFA00BF303734
:10F7A800BD4680BD7042050880B584B000AF786062
:10F7B80039603B68FB60FB687C331F4A106818603F
:10F7C800FB68002283F86F21002283F87021002251
:10F7D80083F87121002283F87221FB6803F2532217
:10F7E800FB68C3F8AD20FB68002242F0100283F8E2
:10F7F800D920002242F00E0283F8DA20002283F892
:10F80800DB20002283F8DC20FB68A53319467868E2
:10F81800FEF73CFDB860FB687C3308491A460B4686
:10F8280003CB1060516019889B7811819372BB6873
:10F8380018461037BD4680BD804205088442050839
:10F8480080B586B000AF786039603B687B617B69C2
:10F858007C331D4A106818607B69002283F86F2189
:10F86800002283F87021002283F87121002283F896
:10F8780072217B69D3F8C1303B617B69D3F8C12021
:10F888007B691B681B011A447B69C3F8C1207B692B
:10F89800A53319467868F4F7EBF9F8607B693A699B
:10F8A800C3F8C1207B697C3308491A460B4603CB51
:10F8B8001060516019889B7811819372FB68184613
:10F8C8001837BD4680BD00BF904205089442050820
:10F8D80080B586B000AF786039603B68002B2ED0C9
:10F8E8007B68002B2BDB7B68012B28DC7B6844F2D0
:10F8F800404202FB03F3144A13447B617B69A5333E
:10F908003B613B69E63308220021184638F0B0FF16
:10F91800396940F2E930FEF7B9FCF860FB68002B62
:10F9280004D13B69D3F8E630002B03D13B68074A82
:10F938001A6004E03B69D3F8E6203B681A6000BF10
:10F948001837BD4680BD00BF6C540020A042050892
:10F9580080B586B000AF786039603B687B617B68B2
:10F9680044F2404202FB03F3094A13443B613B69FA
:10F97800A533FB60FB687A691A60F9684420FEF7D2
:10F9880085FCB860BB6818461837BD4680BD00BF07
:10F998006C54002080B586B000AF786039603B6851
:10F9A8007B617B6844F2404202FB03F30C4A134438
:10F9B8003B613B69A533FB607B691A68FB68C3F848
:10F9C800E6207B695A68FB68C3F8EA20F9684FF4B7
:10F9D8007C70FEF75BFC00BF1837BD4680BD00BFDA
:10F9E8006C54002080B586B000AF786039607B68C1
:10F9F80044F2404202FB03F3294A13443B613B694A
:10FA0800A533FB60FB68D3F8E630002B43D0FB68D6
:10FA1800D3F8E630BB607B6801331A462149B868E1
:10FA280032F07CFBFB6800221A7700225A7700220A
:10FA38009A770022DA7700237B6124E07B6901331F
:10FA48001A461949B86832F069FBFB687A69DA61C5
:10FA5800F9680120F4F70CF9FB68D3F8CA3003F011
:10FA68000103002B05D0F96840F2EB30FEF70EFCDD
:10FA780006E07B6901331A460C49B86832F04EFB40
:10FA88007B6901337B617B690F2BD7DD0849B86837
:10FA980032F0ECFA00E000BF1837BD4680BD00BF69
:10FAA8006C540020B4420508D4420508F442050805
:10FAB8001443050880B58AB006AF7860294BBB604F
:10FAC80007F108031A4640F2E9317868FEF788FC26
:10FAD800002030F06BFBF8602349F86830F00EFC2A
:10FAE800F860BB68184621497A681346DB009B1A00
:10FAF8005B000B44D3F80A301A467B680133194679
:10FB08000023059300230493039102230293019297
:10FB180002230093034602221549F86830F0D2FA0E
:10FB2800F860492303221349F86830F04FFBF86066
:10FB38004F2303221049F86830F048FBF86050233F
:10FB480003220E49F86830F041FBF8605323032282
:10FB58000B49F86830F03AFBF860FB681846103734
:10FB6800BD4680BD344305083C430508A8ED002088
:10FB780040430508A8430508C8430508E0430508AD
:10FB8800FC43050880B586B000AF786039602C4921
:10FB98007A681346DB009B1A5B000B44D3F80A30E3
:10FBA8007B617B6944F2404202FB03F3254A13441C
:10FBB8003B613B69A533FB607868FFF77BFF034631
:10FBC800184630F03DFA03461B2B35D01B2BE8DBDB
:10FBD800532BE6DC492BE4DB493B0A2BE1D801A295
:10FBE80052F823F019FC0008ABFB0008ABFB000837
:10FBF800ABFB0008ABFB0008ABFB000821FC0008CE
:10FC080031FC0008ABFB0008ABFB000829FC00082E
:10FC1800F86800F0DDF80EE0386900F015F80AE041
:10FC2800386900F06FF806E0F96840F2EA30FEF74C
:10FC38002DFB00BFB5E7B4E700BF1837BD4680BD50
:10FC4800A8ED00206C54002080B584B000AF786027
:10FC58007B68FB600E482FF0FFFEFB6818331946DF
:10FC68000C482FF0F9FEFB687C3319460A482FF040
:10FC7800F3FEFB68D3F89530194608482FF0ECFEE0
:10FC880000202FF0F7FF00BF1037BD4680BD00BF32
:10FC9800204405083C4405085C4405087C440508E4
:10FCA80080B584B000AF7860002030F07FFAF8604B
:10FCB8000F49F86830F022FBF8607B6802220D4992
:10FCC800F86830F083FAF8600B49F86830F051FAB8
:10FCD800F8600A49F86830F04CFAF8600849F868A2
:10FCE80030F047FAF860FB6818461037BD4680BD0B
:10FCF8009C440508A8440508D0440508F8440508AC
:10FD08000C45050880B584B000AF78607B68BB609F
:10FD18000123FB60F868FFF7C3FF0346184630F07D
:10FD28009CF926482FF098FEFB685A1EB9681346BE
:10FD38005B0013449B000B4403F5C873D3F80730EA
:10FD480019461F482FF088FEFB685A1EB9681346EB
:10FD58005B0013449B000B4403F5C873D3F80330CE
:10FD6800194618482FF078FE14482FF075FE1649EA
:10FD780016482FF0FBFF03462D2B0FD02D2BC9DC87
:10FD88001B2B16D02B2B13D1FB680F2B02DD012365
:10FD9800FB600DE0FB680133FB6009E0FB68012BA9
:10FDA80002DC1023FB6002E0FB68013BFB6000BF44
:10FDB800B0E700BF1037BD4680BD00BF204505082D
:10FDC80024450508384505084C45050850450508EB
:10FDD80080B584B000AF78607B68FB6015482FF071
:10FDE8003BFE15482FF038FEFB685B681946134840
:10FDF8002FF032FEFB681B69194611482FF02CFEC4
:10FE0800FB685B6919460F482FF026FEFB68DB6923
:10FE180019460D482FF020FEFB68D3F8CA30194662
:10FE28000A482FF019FE00202FF024FF00BF1037DA
:10FE3800BD4680BD544505082044050858450508B9
:10FE48007845050898450508B8450508D8450508C2
:10FE580080B483B000AF7860396000BF0C37BD460E
:10FE680080BC704780B485B000AF78607B68002B99
:10FE780001D1124B1CE07B68FB600023BB600CE0E7
:10FE8800FB681B785C2B03D0FB681B782F2B01D1F8
:10FE9800FB68BB60FB680133FB60FB681B78002BC9
:10FEA800EED1BB68002B02D0BB68013300E07B6851
:10FEB80018461437BD4680BC704700BFF845050892
:10FEC80080B5AAB004AFF860B9607A600023C7F8BB
:10FED800943043F2DD33C7F890307A68D7F8903021
:10FEE8009A420FD8F868FFF7BDFF0246D7F890305E
:10FEF80001937B680093BB6811494FF0005032F0C2
:10FF080091FC19E0F868FFF7ADFF024607F1100011
:10FF1800D7F8903002937B680193BB68009313462F
:10FF2800084A802138F092FB002387F88F3007F1C8
:10FF38001003184631F00CFC9837BD4680BD00BF51
:10FF4800FC4505083446050880B487B000AFF86062
:10FF5800B9607A603B607B6800221A7000225A7090
:10FF680000229A700022DA707B6800221A7100223F
:10FF78005A7100229A710022DA7100237B611AE01B
:10FF88007B69DB003A68134400221A7000225A7019
:10FF980000229A700022DA707B69DB003A68134409
:10FFA80000221A7100225A7100229A710022DA7115
:10FFB8007B6901337B617B690F2BE1DDBB68094AF3
:10FFC8001A60BB68084A5A60BB68084A9A60BB68EE
:10FFD800074ADA60BB68074A1A6100BF1C37BD468A
:10FFE80080BC7047A4000020AC000020B0000020B6
:08FFF800B8000020D000002039
:020000040801F1
:1000000080B485B000AFF860B9607A6000BF143783
:10001000BD4680BC7047000080B584B000AF7860FA
:10002000074BBB60074BFB6007F108031A46102122
:100030007868FAF761FC00BF1037BD4680BD00BF8D
:1000400051FF00080100010880B584B000AF78605E
:10005000074BBB60074BFB6007F108031A461021F2
:10006000786834F00FF800BF1037BD4680BD00BF80
:1000700051FF00080100010880B586B000AF78602C
:1000800039603B687B617B68B3F57C7F6ADC7B68A9
:10009000B3F57A7F06DC7B680F2B46D07B68442B58
:1000A00041D05FE07B68A3F2E933072B5AD801A265
:1000B00052F823F0D9000108E3000108ED0001081F
:1000C000D5000108650101081D010108650101084D
:1000D000F7000108002363E0386800F067F80023A8
:1000E0005EE0386800F08EF8002359E0386800F0D0
:1000F0006FF8002354E03B683B613B69002B30D034
:100100003B69D3F8E630002B2BD03B69D3F8E630BF
:10011000FB602549F86831F0ADFF22E03868FFF751
:100120007BFF00233CE004233AE07B69002283F854
:100130003020002283F83120002283F83220002270
:1001400083F833207B69002283F8CA20002283F8D9
:10015000CB20002283F8CC20002283F8CD2000237E
:100160001EE000BF7B68042B05D07B68B3F57B7F66
:1001700015D1002314E07B69002242F05F0283F86E
:10018000CA20002242F0020283F8CB20002283F82A
:10019000CC20002283F8CD2040F25F2300E0012331
:1001A00018461837BD4680BDB046050880B483B0F8
:1001B00000AF78607B68002B03D07B68034AC3F8EC
:1001C000E62000BF0C37BD4680BC7047C44605081A
:1001D00080B584B000AF78607B68FB60FB68D3F8C3
:1001E000E630002B08D0FB68D3F8E630BB6004494A
:1001F000B86831F03FFF00E000BF1037BD4680BD5A
:10020000D446050880B584B000AF78607B68FB6099
:10021000FB68DB68002B03D113482FF021FC02E0C0
:1002200012482FF01DFC124A3F2112482FF018FCF3
:1002300011482FF015FC114911482FF09BFD034682
:10024000432B08D0432BF3DC1B2B09D03F2B06D1CB
:1002500000F018F803E07868FFF7F6FE00BFE7E764
:1002600000BF1037BD4680BDEC460508184705089D
:10027000444705085447050888470508944705087A
:10028000D400002080B500AF05482FF0E9FB3F21E6
:1002900004482FF0E5FB04482FF0E2FB00BF80BDCF
:1002A00098470508BC470508D84705082DE9B04F11
:1002B0009AB000AF78643964FA63FB6B002B06DCFC
:1002C0004F4BFB656423BB6501237B651BE0FB6B28
:1002D000012B06D14B4BFB650A23BB6501237B65D4
:1002E00011E0FB6B022B07D142F21073FB65012377
:1002F000BB6501237B6506E04FF47A73FB65012340
:10030000BB650A237B657B6C00223B637A633B6C95
:1003100000229A469346D7E90C010B460AFB03F2EA
:10032000034603FB0BF313440246A2FB0A452B448E
:100330001D46C7E91245C7E91245FB6D0022BB62A5
:10034000FA62D7E90A23D7E91201F0F737FF02462C
:100350000B46C7E91823FB6D00223B627A62D7E99E
:100360001201D7E90823F0F729FFF96D49080020A9
:10037000B961F861D7E906010446A2428B410AD36C
:10038000D7E91823511C396043F100037B60D7E99A
:100390000034C7E91834BB6D00223B617A617B6E83
:1003A000D7E90445224602FB03F23B6E294601FBD6
:1003B00003F313443A6E2146A2FB01894B4499464C
:1003C000C7E91889C7E918897B6D0022BB60FA600C
:1003D000D7E90223D7E91801F0F7F0FE02460B46F1
:1003E000C7E91823D7E91823012B01D23B6E01E09E
:1003F0004FF0FF3318466837BD46BDE8B08F00BFE9
:1004000040420F00A086010080B489B000AFF860C0
:10041000B9607A603B60FB687B617B695B683B61CC
:100420007B6800221A7000225A7000229A70002203
:10043000DA707B6800221A7100225A7100229A71C8
:100440000022DA710023FB6137E0FB69DB003A68C8
:10045000D1183869FA6913465B0013449B000344C2
:1004600003F688631B680B600023BB6116E03969E3
:10047000FA6913465B0013449B00CA18BB69134416
:1004800003F68C631B7818461749FB69DA00BB69D1
:10049000134441F82300BB690133BB61BB69052BE1
:1004A000E5DDFB69DB003A681344FA6952010E4945
:1004B0000A445A60FB690133FB61FB690F2BC4DD01
:1004C000BB680A4A1A60BB68094A5A60BB68094A95
:1004D0009A60BB68084ADA60BB68084A1A6100BFC4
:1004E0002437BD4680BC7047ECDC0020D8000020DB
:1004F000F800002030010020500100209002002070
:1005000080B58CB000AFF860B9607A6000233B62C0
:10051000FB68FB61FB695B68BB6131F0F3FB7861F1
:100520007B69002B00F0C6800121786931F01EFC48
:100530000346002B40F0BA800023FB62ABE00023AF
:100540007B62FB6ADB007A6813441968B869FA6A4F
:1005500013465B0013449B00034403F688631B6847
:10056000994248D0FB6ADB007A6813441968B8697D
:10057000FA6A13465B0013449B00034403F6886346
:100580001960FB6ADB007A6813441B6803F47C5330
:10059000002B16D0B969FA6A13465B0013449B001E
:1005A0000B4403F688631B6843F40041B869FA6A98
:1005B00013465B0013449B00034403F688631960F1
:1005C00015E0B969FA6A13465B0013449B000B44BB
:1005D00003F688631B6823F40041B869FA6A13467E
:1005E0005B0013449B00034403F6886319600123F6
:1005F0007B6201233B620023BB622FE0B969FA6A88
:1006000013465B0013449B00CA18BB6A134403F6ED
:100610008C631A783648FB6AD900BB6A0B4450F8E1
:100620002330DBB29A4201D001237B623049FB6A5E
:10063000DA00BB6A134451F82330D8B2B969FA6AB8
:1006400013465B0013449B00CA18BB6A134403F6AD
:100650008C6302461A70BB6A0133BB62BB6A052B0E
:10066000CCDD7B6A002B13D001233B62BA69FB6AA5
:10067000E82101FB03F3134428339B6823F00102B4
:10068000B969FB6AE82000FB03F30B4428339A6046
:10069000FB6A0133FB62FB6A0F2B7FF750AF00212F
:1006A000786931F0A9FBF86800F0B8F9786931F0A1
:1006B00031FB06E04FF4A7730E4A0F49042032F0D5
:1006C000B5F83B6A002B0ED0BB69002242F0020253
:1006D00083F8842E002283F8852E002283F8862E4C
:1006E000002283F8872E00BF3037BD4680BD00BF93
:1006F000ECDC002090600508A049050880B584B0B6
:1007000000AF7860074BBB60074BFB6007F1080345
:100710001A4610217868FAF7EFF800BF1037BD4687
:1007200080BD00BF090401080105010880B584B03F
:1007300000AF7860074BBB60074BFB6007F1080315
:100740001A461021786833F09DFC00BF1037BD4673
:1007500080BD00BF090401080105010880B588B00B
:1007600000AFF860B9607A6000237B61BB681B68EA
:1007700003F47C53B3F5807F02D10123FB6137E0A2
:10078000BB681B6803F47C53B3F5007F02D10223DE
:10079000FB612DE0BB681B6803F47C53B3F5806FED
:1007A00002D10323FB6123E0BB681B6803F47C5385
:1007B000B3F5006F02D10423FB6119E0BB681B682D
:1007C00003F47C53B3F5805F04D101237B610523DF
:1007D000FB610DE0BB681B6803F47C53B3F5005F5D
:1007E00004D101237B610623FB6101E00023FB614F
:1007F0004E49F86831F03EFC4D4B5B681946F8688D
:1008000031F038FC4B49F86831F034FC4A4AFB6956
:1008100052F823301946F86831F02CFCBB681B688D
:1008200003F00103002B01D0082300E00723FB6144
:100830003E49F86831F01EFC3D4B9B681946F8684C
:1008400031F018FC3B49F86831F014FC3A4AFB6976
:1008500052F823301946F86831F00CFCBB681B686D
:1008600003F00203002B01D00B2300E00C23FB61FB
:100870002E49F86831F0FEFB2D4B1B691946F868CC
:1008800031F0F8FB2B49F86831F0F4FB2A4AFB6998
:1008900052F823301946F86831F0ECFB7B69002BE5
:1008A00040D02649F86831F0E5FB0023BB6116E033
:1008B000BA68BB69134404331B78FB74FB7CC82BF8
:1008C00004D11F49F86831F0D5FB05E0FB7C1A46DE
:1008D0001C49F86831F026FCBB690133BB61BB6978
:1008E000052BE5DD1849F86831F0C4FB0023BB6136
:1008F00015E07A68BB6913441B78FB74FB7CC82B3A
:1009000004D10F49F86831F0B5FB05E0FB7C1A46CD
:100910000C49F86831F006FCBB690133BB61BB6967
:10092000052BE6DD00BF2037BD4680BDD049050858
:1009300030010020D449050850010020D84905089D
:10094000EC490508F4490508FC49050880B483B062
:1009500000AF78607B6803F00203002B01D1032312
:1009600000E0022318460C37BD4680BC704780B5B6
:1009700082B000AF786039603868FFF7E7FF034660
:10098000022B05D17A6813469B0013445B007B6001
:100990007B6818460837BD4680BD80B485B000AF7F
:1009A000786039607B68E82202FB03F33A681344FD
:1009B0000433BB600023FB6027E039687A68134684
:1009C0005B0013449B00CA18FB68134403F68C6356
:1009D0001978BA68FB6813440A461A70FB68DBB2E0
:1009E0000133D9B2BA68FB685B0013440A469A71B6
:1009F000BA68FB6813441978BA68FB685B00134453
:100A00000A46DA71FB680133FB60FB68052BD4DD15
:100A100000BF00BF1437BD4680BC704780B586B0AC
:100A200000AF78607B683B613B695B68FB600023DB
:100A30007B6106E0F9687869FFF7AFFF7B690133F6
:100A40007B617B690F2BF5DD00BF00BF1837BD460A
:100A500080BD000080B586B000AF786039600023AB
:100A60007B617B68442B3CD07B68442B3BDB7B6801
:100A7000B3F57C7F37DC7B68B3F57A7F33DD7B6849
:100A8000A3F2E933072B2ED801A252F823F000BFBE
:100A9000B10A0108BB0A0108C50A0108E70A0108F2
:100AA000E70A0108D90A0108E70A0108CF0A010884
:100AB000386804F0B3FF0023DEE0386805F022F95F
:100AC0000023D9E0386804F0FFFF0023D4E0386841
:100AD00004F0B6FF0023CFE03868FFF70FFE0023D5
:100AE000CAE00423C8E03B683B613B695B68FB608C
:100AF0003B69DB69E82202FB03F3FA681344043321
:100B0000BB607B680F2B25DC7B68032BC0F29D80CC
:100B10007B68033B0C2B00F2988001A252F823F073
:100B2000670B0108790B01088B0B01089D0B01086D
:100B3000AF0B0108C10B0108D30B0108E50B01083D
:100B4000EF0B0108010C0108130C0108250C01082A
:100B5000390C01087B68B3F57B7F76D1386800F0EB
:100B60008FF8786171E0386800F018FA78613B69B5
:100B70007A69C3F8CA2068E0386800F0A7FA78619B
:100B80003B697A69C3F8CA205FE0386801F0A8FFC2
:100B900078613B697A69C3F8CA2056E0386801F089
:100BA000F1FF78613B697A69C3F8CA204DE0386883
:100BB00002F022F878613B697A69C3F8CA2044E000
:100BC000386802F061F878613B697A69C3F8CA2035
:100BD0003BE0386803F078F878613B697A69C3F8DC
:100BE000CA2032E0386802F089F878612DE0386870
:100BF00002F03EFC78613B697A69C3F8CA2024E0C0
:100C0000386803F0CDFB78613B697A69C3F8CA2084
:100C10001BE0386801F0D4FE78613B697A69C3F85B
:100C2000CA2012E0386803F025F800237B613B6995
:100C30007A69C3F8CA2008E0386800F057F978618B
:100C40003B697A69C3F8CA2000BF7B69B3F5FC7FB2
:100C500011D1BB68DB6A03F00103002B0BD0BB682A
:100C6000DB6A03F04003002B05D1BB68DB6A23F08D
:100C70000102BB68DA627B6918461837BD4680BD41
:100C800080B58AB000AF786041F2835295499648AA
:100C9000FFF71AF97B68BB61BB695B687B61BB6965
:100CA000DB681A467B6903F58053C3F87F25BB696F
:100CB000DB68002B40F0DB8000233B62D3E03B6A23
:100CC000E82202FB03F37A69134404333B613B6976
:100CD000002283F82420002283F82520002283F8B4
:100CE0002620002283F827203B69002283F8282051
:100CF000002283F82920002283F82A20002283F88A
:100D00002B203B69002283F82C20002283F82D2021
:100D1000002283F82E20002283F82F203B69002236
:100D200083F83020002283F83120002283F832201B
:100D3000002283F833203B69002283F8342000220C
:100D400083F83520002283F83620002283F83720EC
:100D50003B69002283F85020002283F851200022B2
:100D600083F85220002283F853203B69002283F845
:100D70007C20002283F87D20002283F87E20002240
:100D800083F87F203B69002283F88020002283F8CB
:100D90008120002283F88220002283F883203B698F
:100DA000002283F88420002283F88520002283F823
:100DB0008620002283F887203B6900221A760022D1
:100DC0005A7600229A760022DA763B6900221A7758
:100DD00000225A7700229A770022DA770023FB61FB
:100DE0002FE0FA6913465B0013449B0088333A698D
:100DF0001344FB60FB68002242F07C021A7100225F
:100E00005A7100229A710022DA71FB68002242F0C6
:100E10007C021A7000225A7000229A700022DA7046
:100E2000FB68002262F04F021A7200225A720022FE
:100E30009A720022DA72FB680C33FB60FB690133A3
:100E4000FB61FB69072BCCDD3B69DB7C03F078039E
:100E5000DBB2182B04D03B69032118462EF044FB6B
:100E60003B6A01333B623B6A0F2B7FF728AF7B69FC
:100E700003F5A95314337B6200233B620EE07B6AC7
:100E800000221A7000225A7000229A700022DA7032
:100E90007B6A04337B623B6A01333B623B6A0F2B04
:100EA000EDDD7B6903F68860BB699B6840221946CB
:100EB000EFF786FA7868FFF7B1FD7B69002283F8C7
:100EC000842E002283F8852E002283F8862E0022AD
:100ED00083F8872E786804F013FA034618462837FB
:100EE000BD4680BD104A0508284A050880B584B073
:100EF00000AF78607B68FB60FB685B68BB60BB68C9
:100F0000D3F8843E002B35D023494FF4006031F0F4
:100F10008DFCBB68002283F8842E002283F8852E86
:100F2000002283F8862E002283F8872EFB68002299
:100F300042F0020283F83020002283F831200022A0
:100F400083F83220002283F83320BB6803F68862DE
:100F5000FB689A63FB68002242F0400283F8342069
:100F6000002283F83520002283F83620002283F8FF
:100F700037200CE0FB68002283F83020002283F841
:100F80003120002283F83220002283F8332000230E
:100F900018461037BD4680BD884A050880B489B020
:100FA00000AF78607B68FB61FB695B68BB61FB69D4
:100FB000DB69E82202FB03F3BA69134404337B6163
:100FC000FB69DA6913465B0013449B0003F68863F0
:100FD000BA6913443B61FB692033FB60FB6924332E
:100FE000BB607B69DB6A03F01003002B2BD13B69EC
:100FF0001B6803F40043002B12D1FB681B6803F04D
:101000000103002B06D07B695B6B43F001027B6917
:101010005A6305E07B695B6B23F001027B695A63CD
:10102000FB681B6803F00803002B06D07B69DB6AB2
:1010300043F020027B69DA6205E07B69DB6A23F01A
:1010400020027B69DA62FB681B6803F00203002B55
:1010500023D07B69DB6A43F480727B69DA62FB69C7
:10106000D3F8B2207B691A65BB681B6803F48073F0
:10107000002B05D07B69DB6A43F400727B69DA627E
:10108000BB681B6803F40073002B19D07B69DB6A13
:1010900023F400727B69DA6212E07B69002283F834
:1010A0005020002283F85120002283F85220002291
:1010B00083F853207B69DB6A23F480727B69DA62F0
:1010C000002318462437BD4680BC704780B58AB0DF
:1010D00002AF78607B68BB61BB695B687B61BB69A1
:1010E000DB69E82202FB03F37A69134404333B61B2
:1010F0000023FB613B69DB6A03F00103002B09D18C
:10110000786801F07DFA0346002B03D040F25F239C
:10111000FB6198E1A2230093F02301220221786869
:1011200005F054F9F861FB69002B25D03B695B6B36
:1011300003F40073002B0FD03B69D3F884305A1CA2
:101140003B69C3F884203B69D3F88430632B00F2F9
:1011500073810023FB616FE13B69D3F884305A1C33
:101160003B69C3F884203B69D3F88430312B00F20B
:1011700063810023FB615FE13B69002283F88420E7
:10118000002283F88520002283F88620002283F83D
:1011900087207B6903F5805393F83833FB60FB6845
:1011A0002F2B09D1786801F02BFA0346002B03D0CE
:1011B00040F25F23FB6146E13B69FA681A62FB6813
:1011C000912B00F03B81FB68952B00F03781FB6889
:1011D000DB1003F00103BB60BB68002B17D03B6939
:1011E000DB6A03F04003002B05D13B699B6943F0A8
:1011F00008023B699A61FB6803F00103002B1AD0D7
:101200003B699B6923F001023B699A6113E03B69EA
:101210009B6903F00803002B0DD0FB6803F001036A
:10122000002B02D1FB68202B05D13B699B6923F081
:1012300001023B699A61FB68202B53D13B699B6992
:1012400003F00203002B11D0786802F0E5FC03469E
:10125000052B0BDC3B69DB6A43F040023B69DA6239
:101260003B699B6923F008023B699A613B699B6972
:1012700003F00103002B02D0786803F036FD3B69D0
:101280009B6923F019023B699A613B69DB6A03F0B1
:101290000203002B40F0D4803B69DB6A03F48073C7
:1012A000002B06D0786803F0CDFD0346002B16D046
:1012B00016E13B69DB6A03F48063002B02D0786897
:1012C00003F0A8FC3B69002283F83820002283F851
:1012D0003920002283F83A20002283F83B207868E6
:1012E00003F060FDFB6803F01003002B0BD03B699B
:1012F0009B6903F00203002B05D13B699B6943F016
:1013000003023B699A61FB68242B2ED13B699B69E0
:1013100003F00203002B0BD03B69DB6A43F0400271
:101320003B69DA623B699B6923F008023B699A6179
:101330003B699B6943F001023B699A613B699B6988
:1013400023F010023B699A613B694FF0FF3283F84A
:1013500038204FF0FF3283F839204FF0FF3283F806
:101360003A204FF0FF3283F83B20FB6803F0FE0386
:10137000A02B54D1786803F015FD3B699B6943F0BD
:1013800011023B699A613B695B6B03F00203002B1E
:1013900011D0FB6803F00103002B06D03B699B6969
:1013A00043F080023B699A6105E03B699B6923F049
:1013B00080023B699A613B695B6B03F00103002B80
:1013C0001DD03B695B6B03F08003002B01D0C02371
:1013D00000E0D023A122009201220221786804F0CB
:1013E000F5FFF861FB69002B75D17B6903F580532C
:1013F00093F8383303F00F023B699A6323E03B69AB
:10140000002242F0010283F83820002283F83920BC
:10141000002283F83A20002283F83B2013E03B6946
:101420009B6903F00E03002B0CD13B699B6923F0F1
:1014300011023B699A6106E000BF04E000BF02E0D0
:1014400000BF00E000BF3B69DB6A03F00203002B32
:1014500012D13B695B6B03F08003002B1AD13B690F
:101460005B6B03F00103002B14D03B69DB6A03F0D4
:101470000103002B0ED000E000BF3B69D3F88C20A5
:101480001C4B1B689A4205D0786803F087F8034626
:10149000002B22D13B699B691A46BB69DA623B6922
:1014A0009A6BBB691A643B695A6ABB699A62BB69E9
:1014B000CE333969104A18462EF048FA3B69DB6A88
:1014C00003F00203002B0AD0BB69DB6A43F0400241
:1014D000BB69DA6204E000BF02E000BF00E000BFC9
:1014E000BB69FA69C3F8CA20FB6918462037BD46B4
:1014F00080BD00BF88E70508A060050880B588B0FA
:1015000002AF78607B687B617B695B683B617B696C
:10151000DB69E82202FB03F33A6913440433FB60FE
:101520007B69DB695A1C174B009340F272431649E2
:101530004FF4006031F07AF9FB685B6B03F0010354
:10154000002B0ED07B69DB695A1C104B009340F2D4
:1015500074430D494FF4006031F068F9786803F086
:10156000C4FB7B69DB695A1C094B009340F277434B
:1015700005494FF4006031F059F900231846183737
:10158000BD4680BDC44A0508AC4A0508DC4A0508CA
:10159000004B050880B58EB008AF78607B687B6132
:1015A0007B695B683B617B69DB69E82202FB03F3D3
:1015B0003A6913440433FB607B69DB695A1C364B80
:1015C000009340F2874335494FF4006031F02EF923
:1015D000FB685B6A962B11D17B69DB695A1C304B27
:1015E000009340F28A432D494FF4006031F01EF918
:1015F000FB685B6B23F00602FB685A6300230793CA
:1016000000230693002305930023049300230393F0
:101610000023029346230193AE230093F02301227B
:101620000921786804F0D2FEB860BB68002B12D1A3
:10163000FB685B6B43F00802FB685A637B69DB69FC
:101640005A1C184B009340F2944314494FF4006025
:1016500031F0ECF80BE07B69DB695A1C124B00930C
:1016600040F296430D494FF4006031F0DFF878689E
:10167000FFF744FFB8607B69DB695A1C0B4B009392
:1016800040F2994305494FF4006031F0CFF8BB6850
:1016900018461837BD4680BD144B0508AC4A0508EE
:1016A000304B0508544B05086C4B0508844B050866
:1016B00080B588B002AF786039607B687B617B69F8
:1016C0005B683B617B69DB69E82202FB03F33A69F3
:1016D00013440433FB607B69DB695A1C4D4B009358
:1016E00040F2A9434C494FF4006031F09FF8A92320
:1016F0000093F02311220221786804F067FEB8609D
:10170000BB68002B1FD1FB685B6B43F44072FB6826
:101710005A637B69DB695A1C404B009340F2AE432D
:101720003D494FF4006031F081F87B69DB695A1C58
:101730003B4B009340F2AF4337494FF4006031F028
:1017400075F8002362E0FB685B6B03F00103002B7C
:101750000CD17B69DB695A1C324B009340F2B443D5
:101760002D494FF4006031F061F80BE07B69DB69D3
:101770005A1C2D4B009340F2B64327494FF40060AA
:1017800031F054F8FB685B6B03F00103002B18D0B9
:101790007B69DB695A1C254B009340F2BB431E4911
:1017A0004FF4006031F042F83A68937C022161F313
:1017B000010393743A68937C032161F38403937467
:1017C00017E07B69DB695A1C194B009340F2BF4359
:1017D00011494FF4006031F029F83A68937C0121F7
:1017E00061F3010393743A68937C012161F38403EC
:1017F00093747B69DB695A1C094B009340F2C34325
:1018000005494FF4006031F011F8002318461837ED
:10181000BD4680BD9C4B0508AC4A0508B04B050889
:10182000C44B0508D84B0508EC4B0508004C0508CF
:101830002C4C050880B58AB008AF78600023079368
:1018400000230693002305930023049300230393AE
:101850000023029346230193AE230093F023012239
:101860000921786804F0B2FD0346002B0CBF012368
:101870000023DBB218460837BD4680BD80B588B06E
:1018800002AF786039607B687B617B695B683B6134
:101890007B69DB69E82202FB03F33A6913440433F2
:1018A000FB607B69DB695A1C664B009340F2DB43AB
:1018B00065494FF4006030F0B9FF7B69DA69396936
:1018C00013465B0013449B000B4403F688631B68BC
:1018D00003F47C53BB60BB6803F48073002B37D0E8
:1018E000FB685B6B43F04002FB685A633A68937C89
:1018F000012161F3010393743A68937C012161F340
:10190000840393747B69DB695A1C504B009340F24B
:10191000E4434D494FF4006030F088FF7B69DB6998
:101920005A1C4B4B009340F2E54347494FF400608B
:1019300030F07CFF7B69DB695A1C464B009340F218
:10194000E64341494FF4006030F070FF002348E364
:10195000BB6803F48063002B37D0FB685B6B43F0FC
:101960000102FB685A633A68937C022161F3010328
:1019700093743A68937C032161F3840393747B69C5
:10198000DB695A1C344B009340F2EE432E494FF46E
:10199000006030F04BFF7B69DB695A1C2F4B0093D2
:1019A00040F2EF4328494FF4006030F03FFF7B697D
:1019B000DB695A1C274B00934FF49E6322494FF476
:1019C000006030F033FF00230BE3BB6803F40073C7
:1019D000002B47D0FB685B6B43F44072FB685A6393
:1019E0003A68937C012161F3840393743A68937C91
:1019F000012161F3010393747B69DB695A1C184B65
:101A000000934FF49F6310494FF4006030F00EFFD5
:101A10007B69DB695A1C0E4B009340F2F9430A497B
:101A20004FF4006030F002FF7B69DB695A1C094B00
:101A3000009340F2FA4304494FF4006030F0F6FEA0
:101A40000023CEE2584C0508AC4A05087C4C05083A
:101A5000984C0508CC4C0508F44C0508104D0508B9
:101A6000444D0508BB6803F40063002B00F0388187
:101A7000FB685B6A03F01003002B11D17B69DB6903
:101A80005A1C8C4B00934FF4A0638B494FF40060B9
:101A900030F0CCFEFB685B6B43F00202FB685A63DC
:101AA000FB685B6A03F08003002B11D17B69DB6963
:101AB0005A1C824B009340F204537F494FF400605C
:101AC00030F0B4FEFB685B6B43F00402FB685A63C2
:101AD000FB685B6A062B40F082807B69DB695A1CDD
:101AE000774B009340F20C5373494FF4006030F091
:101AF0009DFE7B69DB695A1C724B009340F20D53CB
:101B00006D494FF4006030F091FE7B69DB695A1C2F
:101B10006D4B009340F20E5367494FF4006030F074
:101B200085FE7B69DB695A1C684B009340F20F53BA
:101B300061494FF4006030F079FE7B69DB695A1C23
:101B40005C4B00934FF4A2635B494FF4006030F0AC
:101B50006DFE7B69DB695A1C5D4B009340F21153AB
:101B600055494FF4006030F061FE3A68937C0221E1
:101B700061F3010393743A68937C022161F3840357
:101B80009374FB685B6B43F4C17343F00103FA6821
:101B900053637868FFF74EFE0346002B11D0FB68B5
:101BA0005B6B43F00802FB685A637B69DB695A1C74
:101BB000484B009340F21A533F494FF4006030F015
:101BC00035FE7B69DB695A1C434B009340F21C5382
:101BD00039494FF4006030F029FE002301E2FB6830
:101BE0005B6B43F4C07343F00103FA6853637B6992
:101BF000DB695A1C334B009340F223532E494FF4B8
